:100000000C94DD090C94050A0C94050A0C94050A5D
:100010000C94050A0C94050A0C94050A0C94050A24
:100020000C94050A0C94050A0C94050A0C94050A14
:100030000C94050A0C9477510C94050A0C94050A4B
:100040000C94050A0C94F3610C94DB2A0C94050AB9
:100050000C949D2C0C94050A0C94050A0C94050A2A
:100060000C94050A0C94050A0C94050A0C94050AD4
:100070000C94050A0C94050A0C94050A084AD73B0F
:100080003BCE016E84BCBFFDC12F3D6C74319ABD67
:1000900056833DDA3D00C77F11BED9E4BB4C3E918B
:1000A0006BAAAABE000000803F05A84CCDB2D44E7A
:1000B000B93836A9020C50B9918688083CA6AAAA7C
:1000C0002ABE000000803F6563686F3A00656E716C
:1000D0007565696E67202200220073746172740076
:1000E000506F7765725570002045787465726E6147
:1000F0006C205265736574002042726F776E206FBA
:100100007574205265736574002057617463686468
:100110006F672052657365740020536F6674776152
:100120007265205265736574004D61726C696E2052
:1001300000312E302E302052433200204C61737437
:1001400020557064617465643A2000323031322D7C
:1001500030372D323900207C20417574686F723A37
:10016000200069776A002046726565204D656D6FD5
:1001700072793A20002020506C616E6E6572427573
:100180006666657242797465733A200053746F72C3
:1001900065642073657474696E6773207265747228
:1001A00065697665643A006F6B00446F6E65207315
:1001B0006176696E672066696C652E004572726FA4
:1001C000723A004C696E65204E756D6265722069E9
:1001D00073206E6F74204C617374204C696E6520BF
:1001E0004E756D6265722B312C204C617374204CFE
:1001F000696E653A00636865636B73756D206D6940
:10020000736D617463682C204C617374204C696E4B
:10021000653A004E6F20436865636B73756D207798
:10022000697468206C696E65206E756D6265722CEC
:10023000204C617374204C696E653A004E6F204CFF
:10024000696E65204E756D626572207769746820ED
:10025000636865636B73756D2C204C617374204CFF
:10026000696E653A006F6B005072696E746572203A
:1002700073746F707065642064657520746F206599
:1002800072726F72732E20466978207468652065DB
:1002900072726F7220616E6420757365204D3939FA
:1002A0003920746F2072657374617274212E202856
:1002B00054656D7065726174757265206973207222
:1002C000657365742E2053657420697420626566B9
:1002D0006F72652072657374617274696E6729004C
:1002E000446F6E65207072696E74696E672066690E
:1002F0006C6500426567696E2066696C65206C6993
:10030000737400456E642066696C65206C69737453
:10031000006F6B20543A00202F0020423A00202F1B
:100320000020403A00543A0020453A0020573A0055
:10033000543A0020453A0020423A004649524D576F
:100340004152455F4E414D453A4D61726C696E2098
:1003500056313B20537072696E7465722F677262FA
:100360006C206D617368757020666F722067656EB2
:1003700036204649524D574152455F55524C3A68D6
:100380007474703A2F2F7777772E6D656E64656C75
:100390002D70617274732E636F6D2050524F544FE5
:1003A000434F4C5F56455253494F4E3A312E302001
:1003B0004D414348494E455F545950453A4D656E4D
:1003C00064656C2045585452554445525F434F551F
:1003D0004E543A310A00583A00593A005A3A004508
:1003E0003A0020436F756E7420583A00593A005A0B
:1003F0003A00785F6D696E3A00795F6D696E3A0018
:100400007A5F6D696E3A00556E6B6E6F776E206322
:100410006F6D6D616E643A220022000000000000E2
:1004200000000000000000000000000000000000CC
:100430000080BF00001B43000016430000B44200D0
:1004400000A0400000A0400000803FFFFFFF000030
:100450001B43000016430000B64253657474696E76
:1004600067732053746F72656400537465707320F2
:1004700070657220756E69743A0020204D39322003
:100480005800205900205A002045004D6178696DC0
:10049000756D2066656564726174657320286D6D85
:1004A0002F73293A0020204D323033205800205934
:1004B00000205A002045004D6178696D756D20411E
:1004C0006363656C65726174696F6E20286D6D2F52
:1004D0007332293A0020204D323031205800205903
:1004E00000205A00204500416363656C65726174A9
:1004F000696F6E3A20533D616363656C6572617428
:10050000696F6E2C20543D72657472616374206152
:100510006363656C65726174696F6E0020204D3293
:100520003034205300205400416476616E6365646A
:10053000207661726961626C65733A20533D4D6942
:100540006E20666565647261746520286D6D2F7319
:10055000292C20543D4D696E2074726176656C20A3
:10056000666565647261746520286D6D2F73292C32
:1005700020423D6D696E696D756D207365676D65AF
:100580006E742074696D6520286D73292C20583D88
:100590006D6178696D756D207859206A65726B2080
:1005A000286D6D2F73292C20205A3D6D6178696D5F
:1005B000756D205A206A65726B20286D6D2F732926
:1005C0000020204D323035205300205400204200BE
:1005D000205800205A00204500486F6D65206F6646
:1005E0006673657420286D6D293A0020204D3230E5
:1005F00036205800205900205A0050494420736585
:100600007474696E67733A002020204D33303120B6
:100610005000204900204400526573656E643A0022
:100620006F6B005072696E7465722068616C7465DE
:10063000642E206B696C6C28292063616C6C656486
:10064000202121005072696E7465722073746F707E
:100650007065642064657520746F206572726F72B6
:10066000732E2046697820746865206572726F72F7
:1006700020616E6420757365204D39393920746F9F
:100680002072657374617274212E202854656D7018
:100690006572617475726520697320726573657423
:1006A0002E20536574206974206265666F72652020
:1006B00072657374617274696E6729007C3C3E5E7A
:1006C0002B3D3F2F5B5D3B2C2A225C006563686FEE
:1006D0003A0020636F6C6420657874727573696F7B
:1006E0006E2070726576656E7465640020746F6F3D
:1006F000206C6F6E6720657874727573696F6E20F9
:1007000070726576656E746564006563686F3A0043
:10071000656E6473746F7073206869743A2000208A
:10072000583A0020593A00205A3A0024F404D920BB
:100730001BC40C5C0E9804C4095F0265077101F4C8
:1007400005F900FB04B30048048700C103690058A1
:1007500003550003034500BE023A008402310053F2
:10076000022A002902250004022000E4011C00C81E
:10077000011900AF011700980114008401130071E2
:100780000110006101100051010E0043010D0036FF
:10079000010B002B010B0020010B00150109000CBF
:1007A00001090003010800FB000800F3000800EB4A
:1007B000000700E4000600DE000600D8000600D2B4
:1007C000000600CC000500C7000500C2000500BD02
:1007D000000400B9000400B5000400B1000400AD3D
:1007E000000400A9000400A5000300A20003009F6C
:1007F0000004009B00030098000300950002009392
:10080000000300900003008D0002008B00030088AD
:100810000002008600020084000300810002007FC5
:100820000002007D0002007B0002007900020077D8
:1008300000010076000200740002007200010071E5
:100840000002006F0002006D0001006C0002006AEF
:1008500000010069000200670001006600010065F8
:1008600000010064000200620001006100010060FC
:100870000001005F0002005D0001005C0001005B00
:100880000001005A00010059000100580001005702
:100890000001005600010055000100540001005302
:1008A00000000053000100520001005100010050FF
:1008B0000001004F0001004E0000004E0001004DFD
:1008C0000001004C0001004B0000004B0001004AF9
:1008D00000010049000100480000004800010047F5
:1008E00000010046000000460001004500000045F0
:1008F00000010044000100430000004300010042E9
:1009000000000042000100410000004100010040E1
:100910000001003F0000003F0001003E0000003EDB
:100920000001003D0000003D0001003C0000003CD3
:100930000000003C0001003B0000003B0001003AC9
:100940000000003A000100390000003900010038C1
:1009500000000038000000380001003700000037B8
:1009600000010036000000360000003600010035AE
:1009700000000035000000350001003400000034A4
:100980000000003400010033000000330000003399
:10099000000100320000003200000032000100318E
:1009A0000000003100000031000100300000003084
:1009B000000000300001002F0000002F0000002F79
:1009C0000000002F0001002E0000002E0000002E6D
:1009D0000001002D0000002D0000002D0000002D62
:1009E0000001002C0000002C0000002C0000002C56
:1009F0000001002B0000002B0000002B0000002B4A
:100A00000001002A0000002A0000002A0000002A3D
:100A10000001002900000029000000290000002931
:100A20000000002900010028000000280000002824
:100A30000000002800000028000100270000002717
:100A4000000000270000002700000027000100260A
:100A500000000026000000260000002600000026FE
:100A600000010025000000250000002500000025F1
:100A700000000025000000250001002400000024E3
:100A800000000024000000240000002400010023D6
:100A900000000023000000230000002300000023CA
:100AA00000000023000000230001002200000022BB
:100AB00000000022000000220000002200000022AE
:100AC00000010021000000210000002100000021A1
:100AD0000000002100000021000000210001002092
:100AE0000000002000000020000000200000002086
:100AF0000000002000000020000000200001001F76
:100B00000000001F0000001F0000001F0000001F69
:100B10000000001F0000001F0001001E0000001E5A
:100B20000000001E0000001E00000024F4D430501D
:100B3000C38E20C2A24017828B7011127A910D8150
:100B40006CD90AA861E108C7586607615143061EBF
:100B50004B5D05C145A7041A411104093D98037175
:100B60003931034036DB0265339102D430540280C0
:100B70002E1D02632CEE01752AC501B028A00110BC
:100B80002781018F2564012B244B01E0223401AC25
:100B9000211F018D200D01801FFC00841EED009798
:100BA0001DDF00B81CD200E61BC600201BBC006481
:100BB0001AB200B219A8000A19A0006A189900D147
:100BC00017910040178B00B516840031167E00B3D4
:100BD0001579003A157300C7146F0058146A00EEB7
:100BE0001366008813630025135E00C7125B006C58
:100BF00012570015125400C111510070114F0021FD
:100C0000114B00D61049008D1047004610440002D9
:100C1000104200C00F4000800F3E00420F3C000613
:100C20000F3B00CB0E3800930E37005C0E350027CB
:100C30000E3400F30D3200C10D3100900D30006014
:100C40000D2E00320D2D00050D2C00D90C2B00AE01
:100C50000C2900850C29005C0C2700350C27000EA0
:100C60000C2600E80B2400C40B2400A00B23007DFD
:100C70000B23005A0B2100390B2100180B2000F820
:100C80000A1F00D90A1E00BB0A1E009D0A1D008013
:100C90000A1D00630A1C00470A1B002C0A1B0011D6
:100CA0000A1A00F7091A00DD091900C4091900AB76
:100CB000091900920917007B091800630917004CF5
:100CC00009160036091600200916000A091500F554
:100CD000081500E0081400CC081400B8081400A49B
:100CE000081400900813007D0812006B08130058C8
:100CF00008120046081200340811002308110012DF
:100D000008110001081100F0071000E0071000D0E2
:100D1000071000C0071000B0070F00A107100091D6
:100D2000070E0083070F0074070F0065070E0057BA
:100D3000070E0049070E003B070D002E070E00208E
:100D4000070D0013070D0006070D00F9060C00ED56
:100D5000060D00E0060C00D4060C00C8060C00BC12
:100D6000060C00B0060C00A4060B0099060C008DC2
:100D7000060B0082060B0077060B006C060B006169
:100D8000060A0057060B004C060A0042060A003805
:100D9000060A002E060A0024060A001A060A001097
:100DA00006090007060A00FD050900F4050900EB25
:100DB000050900E2050900D9050900D0050900C7A9
:100DC000050900BE050900B5050800AD050800A528
:100DD0000509009C050800940508008C050800849E
:100DE0000508007C050800740508006C050700650F
:100DF0000508005D050700560508004E0507004779
:100E00000507004005080038050700310507002ADE
:100E1000050700230507001C050600160507000F3F
:100E20000507000805060002050700FB040600F59B
:100E3000040700EE040600E8040600E2040700DBF5
:100E4000040600D5040600CF040600C9040600C34A
:100E5000040600BD040600B7040600B1040500AC9A
:100E6000040600A6040600A00405009B04060095E5
:100E7000040500900406008A04050085040500802E
:100E80000406007A04050075040500700405006B73
:100E900004050066040500610405005C04050057B4
:100EA000040500520405004D0405004804050043F4
:100EB0000405003E0404003A040500350405003032
:100EC0000404002C04050027040400230405001E6C
:100ED0000404001A04040016040500110404000DA3
:100EE000040400090405000404040000040400FCD8
:100EF000030400F8030400F4030400F0030400EC0E
:100F0000030400E8030400E4030400E0030400DC3D
:100F1000030400D8030400D4030400D0030400CC6D
:100F2000030400C8030300C5030300206269617362
:100F30003A200020643A2000206D696E3A2000209B
:100F40006D61783A2000204B753A20002054753AA4
:100F5000200020436C6173696320504944200020C5
:100F60004B703A2000204B693A2000204B643A2015
:100F700000504944204175746F74756E6520666138
:100F8000696C6564212054656D7065726174757259
:100F90006520746F2068696768006F6B20543A00A1
:100FA00020403A00504944204175746F74756E6555
:100FB000206661696C6564212074696D656F757464
:100FC00000504944204175746F74756E65206669E0
:100FD0006E6973686564202120506C6163652074BC
:100FE0006865204B702C204B6920616E64204B6437
:100FF00020636F6E7374616E747320696E20746801
:101000006520636F6E66696775726174696F6E2EB5
:1010100068004572726F723A00202D20496E766129
:101020006C6964206578747275646572206E756D84
:10103000626572210070012C0190012701B001222C
:1010400001C0011D01F00118011002130130020E50
:10105000016002090190020401C002FF000003FACE
:10106000004003F5008003F000D003EB002004E60D
:10107000007004E100E004DC004005D700C005D2A8
:10108000004006CD00D006C8008007C3003008BE6F
:1010900000F008B900C009B400B00AAF00B00BAA54
:1010A00000D00CA500000EA000500F9B00C01096B1
:1010B000005012910000148C00C0158700B01782F8
:1010C00000B0197D00D01B7800001E730040206E18
:1010D0000090226900F024640040275F0090295AA4
:1010E00000E02B5500102E500020304B00103246EF
:1010F00000E033410090353C001037370070383243
:1011000000A0392D00B03A2800A03B2300603C1E0F
:1011100000103D1900903D1400103E0F00703E0A73
:1011200000C03E0500003F0000202D20496E766182
:101130006C6964206578747275646572206E756D73
:101140006265722021003A20457874727564657278
:10115000207377697463686564206F66662E204D1E
:10116000415854454D5020747269676765726564D3
:101170002021003A20457874727564657220737777
:10118000697463686564206F66662E204D494E540D
:10119000454D50207472696767657265642021004F
:1011A00054656D70657261747572652068656174EF
:1011B0006564206265642073776974636865642080
:1011C0006F66662E204D415854454D50207472690B
:1011D000676765726564202121006563686F3A0066
:1011E000534420696E6974206661696C00457272AF
:1011F0006F723A00766F6C756D652E696E6974203A
:101200006661696C6564006F70656E526F6F742003
:101210006661696C65640053442063617264206F89
:101220006B006F70656E206661696C65642C20468A
:10123000696C653A20002E0046696C65206F706508
:101240006E65643A002053697A653A0046696C65B8
:101250002073656C6563746564006F70656E2066ED
:1012600061696C65642C2046696C653A20002E002B
:101270006F70656E206661696C65642C2046696CD0
:10128000653A20002E0057726974696E6720746F8A
:101290002066696C653A20006F70656E2066616932
:1012A0006C65642C2046696C653A20002E00466906
:1012B0006C652064656C657465643A0044656C65B2
:1012C00074696F6E206661696C65642C2046696C78
:1012D000653A20002E005344207072696E74696E66
:1012E00067206279746520002F004E6F742053448C
:1012F000207072696E74696E67006572726F722019
:1013000077726974696E6720746F2066696C650016
:1013100000000001020000000000000004030706B6
:1013200000000000000000000000000000000000BD
:1013300001020408102040800102040810204080AF
:10134000010204081020408080402010080402019F
:10135000020202020202020204040404040404045D
:10136000030303030303030301010101010101015D
:10137000002225282B002124272A494E46494E4980
:1013800054594E414E000020410000C84200401C0C
:101390004620BCBE4CCA1B0E5AAEC59D74CDCCCCEB
:1013A0003D0AD7233C17B7D13877CC2B329595E639
:1013B000241FB14F0A00D32AD72A11241FBECFEF12
:1013C000D0E1DEBFCDBF12E0A0E0B1E0ECEBF1EF89
:1013D00002C005900D92A63EB107D9F71EE0A6EE19
:1013E000B2E001C01D92A534B107E1F713E1C8EBEB
:1013F000D3E104C02297FE010E94DC72C63BD107F4
:10140000C9F70E94A52A0C94D1780C940000FC0125
:101410004591559165917491E52F362F272F642FB3
:101420007E2F832F922F08952F923F924F925F929B
:101430006F927F928F929F92AF92BF92CF92DF92E4
:10144000EF92FF920F931F93CF93DF9300D000D0C2
:1014500000D0CDB7DEB78C011C01220C331C220C4E
:10146000331CC1018B509D4F9A838983FC011082EC
:1014700011821282138221E033E04DEF52E069EFD6
:1014800072E085EF92E00E941F50C101825B9B4F8A
:101490000E94070A2B013C01F801E55BFB4F6491B8
:1014A00070E080E090E00E944A6F0E94196F7727F9
:1014B00067FD7095872F972F0E944C6F4B015C0141
:1014C000C10182579A4F9E838D8320E030E040EC2B
:1014D0005FE3C301B2010E947F71A50194010E94E4
:1014E0007F71ED81FE816083718382839383C1016B
:1014F000845E9E4F9C838B83FC016081718182811D
:10150000938160932C0170932D0180932E01909311
:101510002F0120E030E040E752E40E94B16E28EE57
:10152000C22E22E0D22E7B018C012AE935E046E969
:1015300055E062E975E08EE895E00E9490450E94D2
:10154000D457E981FA81108211821282138221E03C
:1015500033E04DEF52E069EF72E085EF92E00E94D8
:101560001F50C101815C9B4F0E94070A2B013C0167
:101570009058A50194010E947F71ED81FE816083E6
:1015800071838283938320E030E040E752E46091EE
:101590002C0170912D0180912E0190912F010E94BC
:1015A000B16E7B018C012AE935E046E955E062E93C
:1015B00075E08EE895E00E9490450E94D457A30103
:1015C0009201C301B2010E94D16DA50194010E9454
:1015D0007F71ED81FE81608371838283938320E03C
:1015E00030E040E05FE3EB81FC81608171818281CA
:1015F00093810E947F71FB01462F5F2F682F792F07
:1016000040932C0150932D0160932E0170932F0174
:1016100020E030E040E752E4BF010E94B16E7B0160
:101620008C012AE935E046E955E062E975E08EE88B
:1016300095E00E9490450E94D457C101855E9B4F62
:101640000E94070AF101E751FD4F80809180A2803E
:10165000B380A50194010E94D16D2B013C01982F0C
:10166000442D552D692F772DE981FA8140835183CF
:1016700062837383C101895D9B4F0E94070A8101C8
:10168000045F1E4FA50194010E94D16DF801608393
:10169000718382839383C1018D5C9B4F0E94070AF3
:1016A000810100501F4FA50194010E94D16DF801E6
:1016B0006083718382839383842D952DA62DB72D0E
:1016C000ED81FE8180839183A283B38310922C01EC
:1016D00010922D0110922E0110922F0126960FB616
:1016E000F894DEBF0FBECDBFDF91CF911F910F9158
:1016F000FF90EF90DF90CF90BF90AF909F908F9032
:101700007F906F905F904F903F902F900C94675117
:1017100007C03091C00035FFFCCF2093C600019672
:10172000FC0124912111F5CF22E030E081EC95E01D
:101730000C94E12E07C03091C00035FFFCCF209300
:10174000C6000196FC0124912111F5CF22E030E082
:1017500081EC95E00C94E12E07C03091C00035FF7C
:10176000FCCF2093C6000196FC0124912111F5CFF6
:101770002AE030E081EC95E00C94C42DCF93DF9308
:10178000C7ECD0E0FE0107C09091C00095FFFCCFF0
:101790008093C600319684918111F6CFEAE6F4E099
:1017A00007C09091C00095FFFCCF8093C600319692
:1017B00084918111F6CF8091C00085FFFCCF8AE033
:1017C0008093C600FE018491E7ECF0E008C09091A0
:1017D000C00095FFFCCF8093C600319684918111A3
:1017E000F6CF4091730D5091740D6091750D70910D
:1017F000760D8AE794E00E94880B4091770D509116
:10180000780D6091790D70917A0D82E894E00E94D4
:10181000880B40917B0D50917C0D60917D0D7091F6
:101820007E0D85E894E00E94880B40917F0D5091D9
:10183000800D6091810D7091820D88E894E00E9486
:10184000880B8091C00085FFFCCF8AE08093C600A2
:10185000FE018491E7ECF0E008C09091C00095FF94
:10186000FCCF8093C600319684918111F6CFEBE8CE
:10187000F4E007C09091C00095FFFCCF8093C600B4
:10188000319684918111F6CF8091C00085FFFCCF05
:101890008AE08093C600FE018491E7ECF0E008C086
:1018A0009091C00095FFFCCF8093C6003196849143
:1018B0008111F6CF4091830D5091840D6091850D7B
:1018C0007091860D85EA94E00E94880B4091870D07
:1018D0005091880D6091890D70918A0D8EEA94E087
:1018E0000E94880B40918B0D50918C0D60918D0D55
:1018F00070918E0D81EB94E00E94880B40918F0DCA
:101900005091900D6091910D7091920D84EB94E047
:101910000E94880B8091C00085FFFCCF8AE08093F5
:10192000C600FE018491E7ECF0E008C09091C00091
:1019300095FFFCCF8093C600319684918111F6CF3C
:10194000E7EBF4E007C09091C00095FFFCCF8093D7
:10195000C600319684918111F6CF8091C00085FF39
:10196000FCCF8AE08093C600FE018491E7ECF0E0B2
:1019700008C09091C00095FFFCCF8093C6003196BF
:1019800084918111F6CF4091630D5091640D609167
:10199000650D7091660D85ED94E00E94AC0B409151
:1019A000670D5091680D6091690D70916A0D8EED13
:1019B00094E00E94AC0B40916B0D50916C0D6091C6
:1019C0006D0D70916E0D81EE94E00E94AC0B409114
:1019D0006F0D5091700D6091710D7091720D84EECC
:1019E00094E00E94AC0B8091C00085FFFCCF8AE0A0
:1019F0008093C600FE018491E7ECF0E008C090916E
:101A0000C00095FFFCCF8093C60031968491811170
:101A1000F6CFE7EEF4E007C09091C00095FFFCCF51
:101A20008093C600319684918111F6CF8091C000D9
:101A300085FFFCCF8AE08093C600FE018491E7EC2D
:101A4000F0E008C09091C00095FFFCCF8093C600E5
:101A5000319684918111F6CF40915B0D50915C0DD0
:101A600060915D0D70915E0D8CE195E00E94880B98
:101A70004091570D5091580D6091590D70915A0D2C
:101A800085E295E00E94880B8091C00085FFFCCF25
:101A90008AE08093C600FE018491E7ECF0E008C084
:101AA0009091C00095FFFCCF8093C6003196849141
:101AB0008111F6CFE8E2F5E007C09091C00095FFF4
:101AC000FCCF8093C600319684918111F6CF80912E
:101AD000C00085FFFCCF8AE08093C600FE018491A0
:101AE000E7ECF0E008C09091C00095FFFCCF809338
:101AF000C600319684918111F6CF40915F0D5091CF
:101B0000600D6091610D7091620D81EC95E00E9415
:101B1000880B4091470D5091480D6091490D70918F
:101B20004A0D8AEC95E00E94880B4091930D5091EC
:101B3000940D6091950D7091960D8DEC95E00E943D
:101B4000AC0B4091530D5091540D6091550D709117
:101B5000560D80ED95E00E94880B40914F0D5091FD
:101B6000500D6091510D7091520D83ED95E00E94E2
:101B7000880B40914B0D50914C0D60914D0D709123
:101B80004E0D86ED95E00E94880B8091C00085FF88
:101B9000FCCF8AE08093C600FE018491E7ECF0E080
:101BA00008C09091C00095FFFCCF8093C60031968D
:101BB00084918111F6CFE9EDF5E007C09091C00066
:101BC00095FFFCCF8093C600319684918111F6CFAA
:101BD0008091C00085FFFCCF8AE08093C600FE01A3
:101BE0008491E7ECF0E008C09091C00095FFFCCF35
:101BF0008093C600319684918111F6CF4091E9021D
:101C00005091EA026091EB027091EC028BEE95E04C
:101C10000E94880B4091ED025091EE026091EF021C
:101C20007091F00284EF95E00E94880B4091F102E0
:101C30005091F2026091F3027091F40287EF95E007
:101C40000E94880B8091C00085FFFCCF8AE08093C2
:101C5000C600FE018491E7ECF0E008C09091C0005E
:101C600095FFFCCF8093C600319684918111F6CF09
:101C7000EAEFF5E007C09091C00095FFFCCF80939C
:101C8000C600319684918111F6CF8091C00085FF06
:101C9000FCCF8AE08093C600FE01C491E7ECF0E03F
:101CA00008C08091C00085FFFCCFC093C60031966C
:101CB000C491C111F6CF40915201509153016091EE
:101CC00054017091550188E096E00E94880B2DEB3D
:101CD00037E346E05EE360914E0170914F018091E1
:101CE0005001909151010E94B16EAB01BC0182E1A3
:101CF00096E00E949A0B2DEB37E346E05EE360919D
:101D00004A0170914B0180914C0190914D010E94CC
:101D10007F71AB01BC0185E196E00E949A0B809136
:101D2000C00085FFFCCF8AE08093C600DF91CF9191
:101D30000895CF93DF9300D0CDB7DEB780913F0EEB
:101D40009091400E9E012F5F3F4F009719F425544C
:101D50003E4002C0281B390B3A83298389819A812E
:101D60000F900F90DF91CF9108952091E60330916D
:101D7000E703243031050CF06AC04091E80350912C
:101D8000E90360E6649F9001659F300D1124BC015A
:101D9000C90186519C4F0E94A275E7ECF0E007C094
:101DA0009091C00095FFFCCF8093C600319684913E
:101DB0008111F6CFEDECF0E007C09091C00095FFE7
:101DC000FCCF8093C600319684918111F6CF80912B
:101DD000E8039091E90320E6289FF001299FF00D88
:101DE0001124E651FC4F06C09091C00095FFFCCF36
:101DF0008093C60081918111F7CFE8EDF0E007C034
:101E00009091C00095FFFCCF8093C60031968491DD
:101E10008111F6CF8091C00085FFFCCF8AE08093CE
:101E2000C6008091E8039091E903019664E070E0B8
:101E30000E9468729093E9038093E8038091E6031F
:101E40009091E70301969093E7038093E60308954A
:101E5000809174059091750560E070E001960C9496
:101E6000E07280917405909175054AE050E060E061
:101E700070E001960C94377440916E0550916F0597
:101E800090E6949F9001959F300D1124682F70E08B
:101E9000C90186519C4F0E94977590937505809358
:101EA000740521E0892B09F420E0822F08950E9417
:101EB000252B609386057093870580938805909302
:101EC0008905E0916E05F0916F05E659FA4F808122
:101ED000811114C0E0E2F6E007C09091C00095FFC8
:101EE000FCCF8093C600319684918111F6CF80910A
:101EF000C00085FFFCCF8AE08093C600089581EC86
:101F000095E00E94262DE8E1F6E007C09091C00020
:101F100095FFFCCF8093C600319684918111F6CF56
:101F200040917A0550917B0560917C0570917D050B
:101F30004F5F5F4F6F4F7F4F2AE030E081EC95E0BD
:101F40000E94D72D8091C00085FFFCCF8AE080934E
:101F5000C6000C94570F2F923F924F925F926F9250
:101F60007F928F929F92AF92BF92CF92DF92EF9229
:101F7000FF920F931F93CF93DF93CDB7DEB76F9789
:101F80000FB6F894DEBF0FBECDBFF0E67F2EA4E003
:101F90004A2E512CE8E6F2E08490BAE0BB2EE5E64A
:101FA000F2E0A49099249394809142069091430684
:101FB0002091440630914506821B930B8F77992719
:101FC000892B09F004C234C38D3051F08A3321F4D7
:101FD00090917105992321F02F3531050CF4DAC168
:101FE0002115310509F49FC28091E8039091E9031E
:101FF000789E7001799EF00C1124F701E20FF31F17
:10200000E651FC4F1082209171052111BEC1109242
:102010007105FC01E659FA4F1082870106511C4FE9
:102020006EE470E0C8010E949775009709F404C13E
:102030009093750580937405801B910B8E0D9F1DE9
:102040004AE050E060E070E085519C4F0E94377498
:102050006093760570937705809378059093790562
:10206000C0907A05D0907B05E0907C05F0907D05CE
:10207000970186010F5F1F4F2F4F3F4F601771076A
:1020800082079307C1F12091E8033091E903729E22
:10209000C001739E900D11246BE871E086519C4F36
:1020A0000E94C675892B39F5ECEBF1E007C09091E1
:1020B000C00095FFFCCF8093C600319684918111BA
:1020C000F6CFE3ECF1E007C09091C00095FFFCCFA4
:1020D0008093C600319684918111F6CF2AE030E0DA
:1020E000B701A60181EC95E00E94D72D8091C00038
:1020F00085FFFCCF8AC08091E8039091E903789E28
:102100001001799E300C1124810106511C4F6AE2A6
:1021100070E0C8010E949775009721F450C0F32623
:102120002F5F02C020E0F12CF101E20FF11DE6511A
:10213000FC4F30813A3299F790937505809374057E
:10214000801B910B820D931D60E070E085519C4FC8
:102150000E94E0720E94196F2F2D30E0261737077A
:1021600009F459C0ECEBF1E007C09091C00095FF75
:10217000FCCF8093C600319684918111F6CFE5EFB4
:10218000F1E007C09091C00095FFFCCF8093C6009E
:10219000319684918111F6CF40917A0550917B055B
:1021A00060917C0570917D052AE030E081EC95E03E
:1021B0000E94D72D8091C00085FFFCCF26C0ECEB9C
:1021C000F1E007C09091C00095FFFCCF8093C6005E
:1021D000319684918111F6CFE3E1F2E007C090914E
:1021E000C00095FFFCCF8093C60031968491811189
:1021F000F6CF2AE030E0B701A60181EC95E00E941D
:10220000D72D8091C00085FFFCCF8AE08093C60067
:102210000E947F0F47C08091760590917705A0912D
:102220007805B091790580937A0590937B05A0930A
:102230007C05B0937D053BC06AE270E0C8010E9456
:102240009775892BA1F1ECEBF1E007C09091C000EC
:1022500095FFFCCF8093C600319684918111F6CF13
:10226000ECE3F2E007C09091C00095FFFCCF8093B3
:10227000C600319684918111F6CF40917A05509134
:102280007B0560917C0570917D052AE030E081EC52
:1022900095E00E94D72D8091C00085FFFCCF8AE099
:1022A0008093C6001092730510927205EFC1809161
:1022B000E8039091E903789E8001799E100D112426
:1022C000EAEEEE2EE3E0FE2EE00EF11E67E470E093
:1022D000C7010E949775009709F442C09093750555
:1022E000809374058E199F09800F911F60E070E044
:1022F00085519C4F0E94E0720E94196F64307105F5
:1023000078F58091E602811117C080910C0381114C
:1023100027C08A2DE5E6F2E008C09091C00095FF45
:10232000FCCF8093C600319684918111F6CF8091C5
:10233000C00085FFFCCF12C0882DE8E6F2E008C09F
:102340009091C00095FFFCCF8093C6003196849198
:102350008111F6CF8091C00085FFFCCFB092C600FE
:102360008091E8039091E9030196B2010E9468729E
:102370009093E9038093E8038091E6039091E7034B
:1023800001969093E7038093E603109273051092F1
:1023900072050ACE8B3311F49092710590917105FC
:1023A000911102CE4091E8035091E903749ED0014F
:1023B000759EB00D1124A20FB31FA651BC4F8C9374
:1023C0002F5F3F4F3093730520937205EDCD8091C1
:1023D000E6039091E70304970CF42FC129C1809183
:1023E000720590917305892B09F4E8C04FC14D30F7
:1023F00081F04A3321F420917105222351F020917C
:102400007205309173052F3531051CF4019609F0E2
:10241000B8C04091DC035091DD036091DE03709100
:10242000DF038091D4039091D503A091D603B0919E
:10243000D703481759076A077B0708F46DC08F8DCB
:10244000E0EEF2E008C09091C00095FFFCCF8093D1
:10245000C600319684918111F6CF8091C00085FF2E
:10246000FCCF7092C6000E94252B60937E0570936E
:102470007F0580938005909381052091820530919E
:1024800083054091840550918505621B730B840B75
:10249000950BA70196010E947C72CA01B901A501A2
:1024A00094010E947C727F936F933F932F9380E9F6
:1024B00091E09F938F933F922F920E94E075862D1B
:1024C0000FB6F894DEBF0FBECDBFE7ECF0E008C05A
:1024D0009091C00095FFFCCF8093C6003196849107
:1024E0008111F6CFF10106C09091C00095FFFCCF9D
:1024F0008093C60081918111F7CF8091C00085FF44
:10250000FCCF7092C6008CE093E00E94FD6A61E00F
:102510008CE093E00E94F46920917205309173057C
:102520002115310519F410927105B0C08091E803AE
:102530009091E903189FF001199FF00D1124E20F0B
:10254000F31FE651FC4F1082FC01E659FA4F00835D
:102550002091E6033091E7032F5F3F4F3093E7036D
:102560002093E6030196B2010E9468729093E903FA
:102570008093E80310927105109273051092720512
:102580003BC04B3311F400937105809171058111AB
:1025900033C08091E8039091E903189FF001199FDF
:1025A000F00D1124E20FF31FE651FC4F40832F5F23
:1025B0003F4F30937305209372051EC010E601E073
:1025C00034E0432E512CE0EEF2E034913F8F4AE0AC
:1025D000742E58EEC52E53E0D52EE12CF12C6CE371
:1025E000862E912CA12CB12C22242394312C2C0E3C
:1025F0003D1EE7ECF0E064904091DC035091DD0378
:102600006091DE037091DF038091D4039091D50334
:10261000A091D603B091D703481759076A077B07E3
:10262000A8F58091E6039091E7030497A4F02EC0EB
:1026300080910D038111D3CE29C081EC95E00E94D9
:102640000A2D8093700520917205309173058A30B0
:1026500009F0BACCC5CC8091C1039091C203A0917E
:10266000C303B091C4038093DC039093DD03A09374
:10267000DE03B093DF0389EB93E00E946E31482FB5
:10268000809370058A3009F0B2CEC3CE6F960FB634
:10269000F894DEBF0FBECDBFDF91CF911F910F9198
:1026A000FF90EF90DF90CF90BF90AF909F908F9072
:1026B0007F906F905F904F903F902F9008958F92F2
:1026C0009F92AF92BF92CF92DF92EF92FF920F93C1
:1026D0001F93CF93DF93C0E4AC2EC2E0BC2E05EF76
:1026E00012E0CEE8D5E088E0882E83E0982EF50150
:1026F00081915F010E943C0F882319F10E94280FED
:102700006B017C01F4018081811103C060919E0501
:1027100001C061E070E080E090E00E944C6FF80141
:1027200020813181428153810E947F719B01AC01E4
:10273000C701B6010E94D16D688379838A839B8328
:1027400009C0F80180819181A281B3818883998336
:10275000AA83BB830C5F1F4F2496FFEF8F1A9F0A3B
:1027600084E4A81682E0B80611F686E40E943C0FC5
:102770008823D9F00E94280F6B017C016093A80583
:102780007093A9058093AA059093AB0520E030E0F3
:10279000A9010E94AD70181644F4C0922C01D09289
:1027A0002D01E0922E01F0922F01DF91CF911F9128
:1027B0000F91FF90EF90DF90CF90BF90AF909F90E0
:1027C0008F9008950E945F1389E40E943C0F882334
:1027D00059F00E94280F6093AC057093AD0580936B
:1027E000AE059093AF0508C01092AC051092AD05F0
:1027F0001092AE051092AF058AE40E943C0F882328
:1028000059F00E94280F6093B0057093B105809332
:10281000B2059093B30508951092B0051092B105DA
:102820001092B2051092B3050895CF92DF92EF9205
:10283000FF92C0900C01D0900D01E0900E01F0903D
:102840000F01A701960160918E0570918F0580910F
:102850009005909191050E94AA6E87FF08C0C092D2
:102860008E05D0928F05E0929005F0929105C09070
:102870001001D0901101E0901201F0901301A70116
:1028800096016091920570919305809194059091C5
:1028900095050E94AA6E87FF08C0C0929205D0924B
:1028A0009305E0929405F0929505C0901401D090A4
:1028B0001501E0901601F0901701A70196016091B3
:1028C00096057091970580919805909199050E94C1
:1028D000AA6E87FF08C0C0929605D0929705E09235
:1028E0009805F0929905C0900001D0900101E09008
:1028F0000201F0900301A701960160918E0570918D
:102900008F0580919005909191050E94AD701816E9
:1029100044F4C0928E05D0928F05E0929005F0921B
:102920009105C0900401D0900501E0900601F0905F
:102930000701A7019601609192057091930580911E
:102940009405909195050E94AD70181644F4C092BC
:102950009205D0929305E0929405F0929505C0906F
:102960000801D0900901E0900A01F0900B01A70145
:1029700096016091960570919705809198059091C8
:1029800099050E94AD70181644F4C0929605D09235
:102990009705E0929805F0929905FF90EF90DF90EF
:1029A000CF900895CF92DF92EF92FF920F931F93F3
:1029B0008EE895E00E9415140E94252B60938605F1
:1029C00070938705809388059093890560911A011B
:1029D00070911B01882777FD8095982F0E944C6F7E
:1029E00020912C0130912D0140912E0150912F0109
:1029F0000E947F7120E030E040E752E40E94B16E17
:102A000020E030E048EC52E40E94B16E28EEC22E85
:102A100022E0D22E7B018C012AE935E046E955E01F
:102A200062E975E08EE895E00E94904580918E0500
:102A300090918F05A0919005B09191058093F5023A
:102A40009093F602A093F702B093F802809192055A
:102A500090919305A0919405B09195058093F9020A
:102A60009093FA02A093FB02B093FC02809196052A
:102A700090919705A0919805B09199058093FD02DA
:102A80009093FE02A093FF02B093000380919A05F9
:102A900090919B05A0919C05B0919D0580930103A9
:102AA00090930203A0930303B09304031F910F912B
:102AB000FF90EF90DF90CF900895AF92BF92CF92AA
:102AC000DF92EF92FF920F931F93CF93DF93182F14
:102AD0002091B0053091B1054091B2055091B305F8
:102AE0006091AC057091AD058091AE059091AF05F8
:102AF0000E94BA70EB01082FF92E60911A017091B3
:102B00001B01882777FD8095982F0E944C6F20919C
:102B10002C0130912D0140912E0150912F010E94E6
:102B20007F7120E030E040E752E40E94B16E20E087
:102B300030E048EC52E40E94B16E2091E8022F93FD
:102B40001F93FF920F93DF93CF935B016C0132E0F1
:102B5000E32E01E020E04CEA55E06EE875E085EFF9
:102B600092E00E944E3C80918E0590918F05A0913D
:102B70009005B09191058093F5029093F602A09391
:102B8000F702B093F8028091920590919305A0917D
:102B90009405B09195058093F9029093FA02A09361
:102BA000FB02B093FC028091960590919705A0914D
:102BB0009805B09199058093FD029093FE02A09331
:102BC000FF02B093000380919A0590919B05A0911C
:102BD0009C05B0919D058093010390930203A093FF
:102BE0000303B09304030E94252B60938605709322
:102BF000870580938805909389050F900F900F901B
:102C00000F900F900F90DF91CF911F910F91FF9038
:102C1000EF90DF90CF90BF90AF900895F8940E940E
:102C2000075D5E9A5E9A159A5E9AECEBF1E007C03A
:102C30009091C00095FFFCCF8093C600319684919F
:102C40008111F6CFE3E2F6E007C09091C00095FF56
:102C5000FCCF8093C600319684918111F6CF80918C
:102C6000C00085FFFCCF8AE08093C600FFCFCF92E3
:102C7000DF92EF92FF920F931F930E94252B0091FA
:102C8000A0051091A1052091A2053091A305C09047
:102C90008605D0908705E0908805F09089056C192D
:102CA0007D098E099F09061717072807390730F491
:102CB000012B022B032B11F00E940E168091310183
:102CC00090913201A0913301B0913401892B8A2B6C
:102CD0008B2B09F10E94252B009186051091870509
:102CE0002091880530918905601B710B820B930B35
:102CF0000091310110913201209133013091340162
:102D0000061717072807390730F490915508809166
:102D10005408981741F01F910F91FF90EF90DF90AA
:102D2000CF900C946C455E9A5E9A159A5E9AF3CF9A
:102D30000E94075D8091E602811134C081E080939A
:102D4000E60280917A0590917B05A0917C05B09177
:102D50007D058093A4059093A505A093A605B09347
:102D6000A705ECEBF1E007C09091C00095FFFCCF08
:102D70008093C600319684918111F6CFE4E4F6E0A9
:102D800007C09091C00095FFFCCF8093C60031969C
:102D900084918111F6CF8091C00085FFFCCF8AE03D
:102DA0008093C60008958091E6020895EF92FF9205
:102DB0000F931F93CF93DF938C017B0184E0E80E88
:102DC000F11CEB016991F801808191819C012F5FD9
:102DD0003F4F318320830E94E977CE15DF0591F7BD
:102DE00084E090E0DF91CF911F910F91FF90EF90E1
:102DF0000895EF92FF920F931F93CF93DF938C016F
:102E00007B0180E1E80EF11CEB016991F801808102
:102E100091819C012F5F3F4F318320830E94E9778E
:102E2000CE15DF0591F780E190E0DF91CF911F9102
:102E30000F91FF90EF900895EF92FF920F931F93E1
:102E4000CF93DF938C017B0184E0E80EF11CEB0152
:102E50006991F801808191819C012F5F3F4F3183FF
:102E600020830E94E977CE15DF0591F784E090E09A
:102E7000DF91CF911F910F91FF90EF9008950F93E5
:102E80001F93CF93DF93CDB7DEB72A970FB6F89491
:102E9000DEBF0FBECDBF80E390E3A0E3B0E08D8343
:102EA0009E83AF83B88784E690E09A878987BE01C6
:102EB0006B5F7F4FCE0109960E94D61663E77DE0D7
:102EC000CE0109960E94F91663E87DE0CE010996CD
:102ED0000E94F91603E61DE0F80161918F018985D2
:102EE0009A859C012F5F3F4F3A8729870E94E97797
:102EF000FDE003371F0781F76BE57DE0CE01099602
:102F00000E941C1767E57DE0CE0109960E941C1700
:102F10006FE57DE0CE0109960E941C1767E47DE015
:102F2000CE0109960E941C1703E91DE0F80161918A
:102F30008F0189859A859C012F5F3F4F3A872987AA
:102F40000E94E977FDE007391F0781F763E57DE01F
:102F5000CE0109960E941C176FE47DE0CE01099610
:102F60000E941C176BE47DE0CE0109960E941C179D
:102F700009EE12E0F80161918F0189859A859C0123
:102F80002F5F3F4F3A8729870E94E977F2E0053F9C
:102F90001F0781F762E571E0CE0109960E941C17B8
:102FA0006EE471E0CE0109960E941C176AE471E09C
:102FB000CE0109960E941C1786E590E3A6E3B0E0D7
:102FC00089839A83AB83BC8384E690E09A87898760
:102FD000BE016F5F7F4FCE0109960E94D616E7ECC7
:102FE000F0E007C09091C00095FFFCCF8093C60031
:102FF000319684918111F6CFEAE5F4E007C0909113
:10300000C00095FFFCCF8093C6003196849181115A
:10301000F6CF8091C00085FFFCCF8AE08093C60088
:103020002A960FB6F894DEBF0FBECDBFDF91CF91C9
:103030001F910F910895EF92FF920F931F93CF93DB
:10304000DF938C017B0180E1E80EF11CEB01F801BC
:10305000808191819C012F5F3F4F318320830E94AB
:10306000E1778993CE15DF0591F780E190E0DF915C
:10307000CF911F910F91FF90EF900895EF92FF92E3
:103080000F931F93CF93DF938C017B0184E0E80EB5
:10309000F11CEB01F801808191819C012F5F3F4F72
:1030A000318320830E94E1778993CE15DF0591F764
:1030B00084E090E0DF91CF911F910F91FF90EF900E
:1030C0000895AF92BF92CF92DF92EF92FF920F934B
:1030D0001F93CF93DF93CDB7DEB7EC970FB6F8947D
:1030E000DEBF0FBECDBFD82E24E630E03AAF29AF09
:1030F00046E550E366E370E049AB5AAB6BAB7CABA3
:103100008E010B5C1F4FB8017E0189E3E80EF11CB4
:1031100089AD9AAD9C012F5F3F4F3AAF29AF6BAF9E
:103120007CAF0E94E177F80181938F016BAD7CAD9C
:10313000EE15FF0569F7D110A4C043E050E0CE01C1
:10314000C1960E94A975009709F09BC063E77DE0D6
:10315000C8010E941B1863E87DE0C8010E941B188B
:1031600003E61DE089AD9AAD9C012F5F3F4F3AAF5A
:1031700029AF0E94E177F80181938F01FDE00337C9
:103180001F0781F76BE57DE0CE01C9960E943E18CE
:1031900067E57DE0CE01C9960E943E186FE57DE0AF
:1031A000CE01C9960E943E1867E47DE0CE01C99623
:1031B0000E943E1803E91DE089AD9AAD9C012F5F86
:1031C0003F4F3AAF29AF0E94E177F80181938F0119
:1031D000FDE007391F0781F763E57DE0CE01C99661
:1031E0000E943E186FE47DE0CE01C9960E943E1811
:1031F0006BE47DE0CE01C9960E943E1809EE12E014
:1032000089AD9AAD9C012F5F3F4F3AAF29AF0E9425
:10321000E177F80181938F01F2E0053F1F0781F705
:1032200062E571E0CE01C9960E943E186EE471E03D
:10323000CE01C9960E943E186AE471E0CE01C9969B
:103240000E943E18E7ECF0E007C09091C00095FFA7
:10325000FCCF8093C600319684918111F6CFECE8C3
:10326000F1E007C09091C00095FFFCCF8093C600AD
:10327000319684918111F6CF8091C00085FFFCCFFB
:10328000DDC080E1EBE5F1E0DE01919601900D9269
:103290008A95E1F780E1EBE6F1E0DE0151960190DD
:1032A0000D928A95E1F780E1EBE7F1E0DE011196FE
:1032B00001900D928A95E1F76E0181E2C80ED11C52
:1032C00043E7E42E4DE0F42E8E010F5E1F4F63E8BE
:1032D0007DE0AE014F5F5F4FE3E6AE2EEDE0BE2E28
:1032E00024E030E0F60181919191A191B1916F01BB
:1032F000F70181939193A193B1937F01F80181919B
:103300009191A191B1918F01FB0181939193A1932F
:10331000B193BF01FA0181919191A191B191AF0156
:10332000F50181939193A193B1935F0121503109EC
:10333000C9F680E090E0AAE7B4E480935B0D909337
:103340005C0DA0935D0DB0935E0D8093570D90932F
:10335000580DA093590DB0935A0D10925F0D109215
:10336000600D1092610D1092620D80E29EE4A0E06B
:10337000B0E08093930D9093940DA093950DB0932E
:10338000960D1092470D1092480D1092490D109213
:103390004A0D80E090E0A0E7B1E48093530D909354
:1033A000540DA093550DB093560D4DEC5CEC6CECA8
:1033B0007EE340934F0D5093500D6093510D7093E9
:1033C000520D80934B0D90934C0DA0934D0DB093E7
:1033D0004E0D1092F1021092F2021092F30210922E
:1033E000F4021092ED021092EE021092EF0210928F
:1033F000F0021092E9021092EA021092EB0210928F
:10340000EC02E7ECF0E007C09091C00095FFFCCF24
:103410008093C600319684918111F6CFEFE9F1E0F7
:1034200006C09091C00095FFFCCF8093C6008191AB
:103430008111F7CF8091C00085FFFCCF8AE0809397
:10344000C600EC960FB6F894DEBF0FBECDBFDF917D
:10345000CF911F910F91FF90EF90DF90CF90BF9091
:10346000AF9008952F923F924F925F926F927F920A
:103470008F929F92AF92BF92CF92DF92EF92FF9284
:103480000F931F93CF93DF93CDB7DEB7A6970FB6F9
:10349000F894DEBF0FBECDBF87E40E943C0F8823A7
:1034A00009F40EC20E94280F0E94196F6430710542
:1034B000D9F144F46230710521F15CF577FF17C052
:1034C0000C94DF276A35710509F4A6C134F46C3118
:1034D000710511F00C94DF276AC06B35710509F492
:1034E0009FC16C35710511F00C94DF279EC180914E
:1034F000E602811106C00E945F130E94D2140C9450
:103500006F288091E602811104C00E94E21381E0DD
:1035100007C08091E602811107C00E94E21380E09B
:103520000E945D150C946F2880E50E943C0F882353
:1035300039F00E94280F0E941E6F6B017C0103C0AE
:10354000C12CD12C760183E50E943C0F882361F0C9
:103550000E94280F20E030E04AE754E40E947F7187
:103560000E941E6F6B017C010E94D4570E94252B84
:103570004B015C018C0C9D1CAE1CBF1C0E94252BBA
:1035800060938605709387058093880590938905DD
:1035900005C00E94255A81E00E9437160E94252B03
:1035A000681579058A059B05A0F30C94DF278091A7
:1035B0002C0190912D01A0912E01B0912F018093AB
:1035C0008A0590938B05A0938C05B0938D0580910F
:1035D0001A0190911B01909307038093060384E6E0
:1035E00090E090931B0180931A010E94252B609319
:1035F000860570938705809388059093890581E0FF
:103600000E946E518091F5029091F602A091F7020E
:10361000B091F80280938E0590938F05A09390054A
:10362000B09391058091F9029091FA02A091FB026A
:10363000B091FC028093920590939305A09394051A
:10364000B09395058091FD029091FE02A091FF023A
:10365000B09100038093960590939705A0939805E9
:10366000B09399058091010390910203A091030307
:10367000B091040380939A0590939B05A0939C05B9
:10368000B0939D0510922C0110922D0110922E01E5
:1036900010922F0188E50E943C0F882311F090E0E2
:1036A0000AC089E50E943C0F8111F9CF8AE50E948A
:1036B0003C0F91E098279093300191110C94E227F0
:1036C00088E50E943C0F81110C94E2278091300123
:1036D00081110C94E82789E50E943C0F81110C941C
:1036E000E8278091300181110C94EE278AE50E9431
:1036F0003C0F81110C94EE2788E50E943C0F882333
:10370000D1F00E94310F672B682B692BA1F00E942A
:10371000280F2091E9023091EA024091EB0250918A
:10372000EC020E94D16D6093F5027093F6028093D3
:10373000F7029093F80289E50E943C0F8823D1F0AC
:103740000E94310F672B682B692BA1F00E94280F74
:103750002091ED023091EE024091EF025091F00283
:103760000E94D16D6093F9027093FA028093FB027C
:103770009093FC028AE50E943C0F8823D1F00E94BE
:10378000310F672B682B692BA1F00E94280F209125
:10379000F1023091F2024091F3025091F4020E9442
:1037A000D16D6093FD027093FE028093FF029093AF
:1037B000000321E033E04DEF52E069EF72E085EF66
:1037C00092E00E941F5080E00E946E5180918A0515
:1037D00090918B05A0918C05B0918D0580932C0163
:1037E00090932D01A0932E01B0932F018091060399
:1037F0009091070390931B0180931A010E94252B3F
:10380000609386057093870580938805909389055A
:103810000E9467510C94DF2710929E050C94DF27BD
:1038200081E080939E050C94DF2785E40E943C0F85
:10383000811102C00E94D45750E4C52E52E0D52E0B
:1038400069EEE62E62E0F62E05EF12E0B12CF601ED
:1038500081916F010E943C0F882339F1F3E0BF1280
:103860000CC00E94280FF8016083718382839383C8
:1038700081E093E00E94BB5018C00E94280FF7011E
:1038800020813181428153810E94D16DF801608392
:1038900071838283938321E033E04DEF52E069EF3F
:1038A00072E085EF92E00E941F50B394F4E0EF0EB7
:1038B000F11C0C5F1F4F24E0B212C9CF0C94DF271C
:1038C0008DE40E943C0F882311F40C9432270E944F
:1038D000280F0E94196F6237710509F45FC70CF059
:1038E0006FC06C31710509F46DC19CF566317105CD
:1038F00009F425C1ACF46231710509F45EC634F4F3
:103900006131710511F00C94DF27E2C0643171055B
:1039100009F4E4C06531710511F00C94DF2709C189
:103920006931710509F434C154F46731710509F442
:103930000CC16831710511F00C94DF2719C16A318F
:10394000710509F42BC16B31710511F00C94DF275F
:1039500033C16435710509F430C6CCF46A3271059F
:1039600009F43BC254F46E31710509F460C16F3142
:10397000710511F00C94DF2798C16235710509F4C7
:1039800015C66335710511F00C94DF2712C6683631
:10399000710509F45FC254F46535710509F448C630
:1039A0006C35710511F00C94DF2758C66936710526
:1039B00009F4C6C26D36710511F00C94DF2792C36D
:1039C0006E3C710511F40C94E325D4F56C38710547
:1039D00009F4A2C2C4F46737710511F40C94B02441
:1039E00034F46337710511F00C94DF27C9C66837CA
:1039F000710511F40C94AA246937710511F00C9427
:103A0000DF270C94AC246B3C710511F40C94492510
:103A10005CF46E3B710509F42DC5693C710511F02C
:103A20000C94DF270C940F256C3C710511F40C9459
:103A300065256D3C710511F00C94DF270C948525EC
:103A4000603931E0730711F40C940E2704F56D32E0
:103A500091E0790711F40C94202664F46C3D710513
:103A600011F40C94FF256D3D710511F00C94DF27C6
:103A70000C9411266E32F1E07F0711F40C94FB26B2
:103A80006F32714011F00C94DF270C94FF26663FD3
:103A900031E0730711F40C9416276CF4643F91E045
:103AA000790711F40C941127653F714011F00C94C3
:103AB000DF270C941427673FF1E07F0711F40C9483
:103AC0001A27673E734011F00C94DF270C941D27D2
:103AD0005E985E9815985E980C94DF27E3EFF2E00D
:103AE00007C09091C00095FFFCCF8093C60031962F
:103AF00084918111F6CF8091C00085FFFCCF8AE0D0
:103B00008093C6008CE093E00E94EE64E3E0F3E073
:103B100007C09091C00095FFFCCF8093C6003196FE
:103B200084918111F6CF8091C00085FFFCCF0C9469
:103B3000DC278CE093E00E9430650C94DF278CE05A
:103B400093E00E94F6650C94DF27009174051091B4
:103B500075050C5F1F4F6AE270E0C8010E949775FF
:103B6000009719F0FC013197108241E0B80159C06B
:103B70008CE093E00E94FA650E94252B60938205F9
:103B80007093830580938405909385050C94DF27BB
:103B90008CE093E00E9401660C94DF2780910E0375
:103BA000882311F40C94DF2783E50E943C0F8111D8
:103BB0000C94F4270C94DF278CE093E00E94316989
:103BC0000C94DF2780917405909175056AE270E08E
:103BD00004960E9497758C010097E1F020916E0584
:103BE00030916F0540E6429FC001439F900D112424
:103BF0006EE470E086519C4F0E94977560E270E021
:103C00000E94977501969093750580937405F8014D
:103C10003197108260917405709175056C5F7F4FCC
:103C200040E08CE093E00E9406660C94DF278091D0
:103C30000E03882311F40C94DF278CE093E00E949C
:103C4000E86A80917405909175056AE270E00496C7
:103C50000E9497758C010097E1F020916E053091DC
:103C60006F0540E6429FC001439F900D11246EE412
:103C700070E086519C4F0E94977560E270E00E9450
:103C8000977501969093750580937405F8013197A7
:103C9000108260917405709175056C5F7F4F8CE0A8
:103CA00093E00E94F5670C94DF270E94252B609318
:103CB0007E0570937F058093800590938105009128
:103CC0008205109183052091840530918505601B44
:103CD000710B820B930B28EE33E040E050E00E9422
:103CE0007C72CA01B9012CE330E040E050E00E9450
:103CF0007C727F936F933F932F9380E991E09F9322
:103D00008F93CE0101969F938F930E94E075E7EC0D
:103D1000F0E084910FB6F894DEBF0FBECDBFE7ECA4
:103D2000F0E008C09091C00095FFFCCF8093C600E2
:103D3000319684918111F6CFFE01319606C09091A3
:103D4000C00095FFFCCF8093C60081918111F7CF11
:103D50008091C00085FFFCCF8AE08093C6008091EF
:103D6000260D882311F40C94DF271092260D609104
:103D7000E802E62FF0E0EE0FFF1FE050F24F8081E7
:103D800091810E9459592091390130913A01409115
:103D90003B0150913C010E94AD70181614F00C9438
:103DA000DF276091E802062F10E080E090E00E949B
:103DB0008958F801EE0FFF1FE050F24F9183808386
:103DC000F801EE0FFF1FEE0FFF1FEA50F24F1082B7
:103DD0001182128213820C94DF2783E50E943C0F2C
:103DE000882311F40C94DF270E94280F0E94196F7A
:103DF0007B0180E50E943C0F882311F40C94DF279F
:103E0000F7FE02C00C94DF27FFEFEF16F10409F074
:103E100014F40C9405280C94DF278191919180175C
:103E2000910711F40C94DF2722E0E83BF207A9F791
:103E300017FF02C00C94DF2761E0802F0E944D2CF9
:103E40006E2D802F0E94692CB701802F0E94C22BFB
:103E50000C94DF278091E80280939F0584E50E94FF
:103E60003C0F882379F10E94280F0E941E6F6093F7
:103E70009F05662339F1E7ECF0E007C09091C000A0
:103E800095FFFCCF8093C600319684918111F6CFC7
:103E9000EDEBF1E006C09091C00095FFFCCF809360
:103EA000C60081918111F7CF40E050E060919F05FD
:103EB00081EC95E00E94D02D8091C00085FFFCCF61
:103EC0000C94DC2783E50E943C0F882309F1B09015
:103ED0009F050E94280F6B017C010B2D10E00E94B2
:103EE000196FDC01CB016B2D0E948958F801EE0F90
:103EF000FF1FE050F24F91838083F801EE0FFF1F08
:103F0000EE0FFF1FEA50F24FC082D182E282F382AD
:103F10000E94065D0C94DF2783E50E943C0F8823F6
:103F200011F40C94DF270E94280F0E94196FCB0117
:103F30000E940D599093FF0D8093FE0D0C94DF2786
:103F40008091E80280939F0584E50E943C0F8823BE
:103F500079F10E94280F0E941E6F60939F056623CF
:103F600039F1E7ECF0E007C09091C00095FFFCCF7D
:103F70008093C600319684918111F6CFE4EDF1E093
:103F800006C09091C00095FFFCCF8093C600819140
:103F90008111F7CF40E050E060919F0581EC95E002
:103FA0000E94D02D8091C00085FFFCCF0C94DC27AF
:103FB000E1E1F3E007C09091C00095FFFCCF809352
:103FC000C600319684918111F6CF60919F05E62F4E
:103FD000F0E0EE0FFF1FE450F24F808191810E94CC
:103FE0005959AB01BC0121E030E081EC95E00E9421
:103FF000E12EE7E1F3E007C09091C00095FFFCCF10
:104000008093C600319684918111F6CF60919F050F
:10401000E62FF0E0EE0FFF1FE050F24F808191811C
:104020000E945959AB01BC0121E030E081EC95E0E0
:104030000E94E12EEAE1F3E007C09091C00095FFF5
:10404000FCCF8093C600319684918111F6CF809188
:10405000FA0D9091FB0D0E94135CAB01BC0121E0B5
:1040600030E081EC95E00E94E12EEEE1F3E007C044
:104070009091C00095FFFCCF8093C600319684914B
:104080008111F6CF8091FE0D9091FF0D0E94135C7F
:10409000AB01BC0121E030E081EC95E00E94E12E13
:1040A000E1E2F3E007C09091C00095FFFCCF809360
:1040B000C600319684918111F6CF80919F0590E0E2
:1040C0000E9483584AE050E0BC0181EC95E00E94D8
:1040D000E82D8091C00085FFFCCF8AE08093C60068
:1040E0000C946F288091E80280939F0584E50E94DC
:1040F0003C0F882371F10E94280F0E941E6F60936D
:104100009F05662331F1E7ECF0E007C09091C00015
:1041100095FFFCCF8093C600319684918111F6CF34
:10412000EBEEF1E006C09091C00095FFFCCF8093CC
:10413000C60081918111F7CF40E050E060919F056A
:1041400081EC95E00E94D02D8091C00085FFFCCFCE
:1041500033C71092260D83E50E943C0F882309F196
:10416000B0909F050E94280F6B017C010B2D10E081
:104170000E94196FDC01CB016B2D0E948958F80158
:10418000EE0FFF1FE050F24F91838083F801EE0F96
:10419000FF1FEE0FFF1FEA50F24FC082D182E28272
:1041A000F38283E50E943C0F882351F00E94280F80
:1041B0006093390170933A0180933B0190933C01E5
:1041C00082E40E943C0F882351F00E94280F6093E4
:1041D0003D0170933E0180933F019093400186E43E
:1041E0000E943C0F882369F00E94280F60933501DC
:1041F00070933601809337019093380181E080936A
:10420000260D0E94065D0E94252B4B015C018091CA
:104210009F0590E0880F991FFC01E050F24F20812C
:10422000318138A32F8FFC01E450F24F80819181BE
:104230009EA38DA3CC24CA94DC2C7601E5E2F3E0A6
:104240002490E8E2F3E03490ECE2F3E0049148EEED
:10425000442E43E0542E612C712C1AE0F9C6822DB5
:10426000E5E2F3E008C09091C00095FFFCCF809399
:10427000C600319684918111F6CF60919F05E62F9B
:10428000F0E0EE0FFF1FE450F24F808191810E9419
:104290005959AB01BC0121E030E081EC95E00E946E
:1042A000E12E832DE8E2F3E008C09091C00095FF75
:1042B000FCCF8093C600319684918111F6CF609136
:1042C0009F054AE050E070E081EC95E00E94E82D07
:1042D000802FECE2F3E008C09091C00095FFFCCF86
:1042E0008093C600319684918111F6CFF7FE03C00A
:1042F000E2E0F2E027C00E94252B4B015C01C701E0
:10430000B601605F784D8F4F9F4F681979098A0910
:104310009B09A30192010E947C7249015A012AE083
:1043200030E0B501A40181EC95E00E94C42D80919C
:10433000C00085FFFCCF0DC09091C00095FFFCCF61
:104340008093C60081918111F7CF8091C00085FFD5
:10435000FCCF1093C6000E94252B4B015C010E94EC
:10436000255A81E00E9437169FEFC916D906E90643
:10437000F906A9F560919F05EF8DF8A12DA13EA149
:104380002E173F070CF07FC6E62FF0E0EE0FFF1F61
:10439000E450F24F808191810E94595969A37AA318
:1043A0008BA39CA360919F05E62FF0E0EE0FFF1F0B
:1043B000E050F24F808191810E94595920E030E015
:1043C00040E85FE30E94D06D9B01AC0169A17AA136
:1043D0008BA19CA10E94AD7087FF20C639C0F7FC5D
:1043E00037C060919F05E62FF0E0EE0FFF1FE4500D
:1043F000F24F808191810E94595969A37AA38BA3BE
:104400009CA360919F05E62FF0E0EE0FFF1FE050A8
:10441000F24F808191810E9459599B01AC0169A1A1
:104420007AA18BA19CA10E94D06D0E94196FAB0153
:10443000BC0177FF07C070956095509541955F4F1F
:104440006F4F7F4F44305105610571050CF0E6C593
:104450003FEFC316D306E306F30609F4F9C5F7FCEC
:10446000E2C50E94252B6C197D096031774208F462
:10447000EFC5D9C583E50E943C0F882359F00E94FF
:10448000280F0E94196FCB010E940D599093FF0DC8
:104490008093FE0D0E94252B6B017C01E0E3F3E08D
:1044A000A490E3E3F3E0B490E7E3F3E014910AE0CF
:1044B00070C00E94252B6C197D098E099F09693EE9
:1044C00073408105910508F45FC06091E802A62F52
:1044D000B0E0AA0FBB1FA450B24F8D919C910E94D7
:1044E0005959AB01BC018A2DE0E3F3E008C090917B
:1044F000C00095FFFCCF8093C60031968491811156
:10450000F6CF22E030E081EC95E00E94E12E8B2D89
:10451000E3E3F3E008C09091C00095FFFCCF8093E7
:10452000C600319684918111F6CF6091E8024AE08D
:1045300050E070E081EC95E00E94E82D812FE7E3E8
:10454000F3E008C09091C00095FFFCCF8093C600B7
:10455000319684918111F6CF8091FA0D9091FB0DE7
:104560000E94135CAB01BC0121E030E081EC95E0DE
:104570000E94E12E8091C00085FFFCCF0093C60011
:104580000E94252B6B017C010E94255A81E00E942C
:1045900037162091FE0D3091FF0D8091FA0D90910C
:1045A000FB0D821793070CF484CF47C510920B03C1
:1045B00006C581E080930B0302C583E50E943C0F92
:1045C000882399F00E94280F20E030E04AE754E465
:1045D0000E947F710E941E6F6093310170933201BF
:1045E0008093330190933401EAC488E50E943C0F24
:1045F000811141C589E50E943C0F81113CC58AE5C6
:104600000E943C0F811137C585E40E943C0F811147
:1046100032C52BC55E9A89E50E943C0F81115E9AD6
:104620008AE50E943C0F882309F4C9C4159AC7C4BF
:1046300083E50E943C0F0E94280F20E030E04AE70B
:1046400054E40E947F710E941E6F6093A0057093D6
:10465000A1058093A2059093A305B1C420E432E0A4
:104660003EA32DA353E7252E5DE0352E83E89DE084
:1046700098A38F8F67E3862E6DE0962E10E0EDA154
:10468000FEA18191FEA3EDA30E943C0F882309F4B3
:1046900066C0133009F05CC00E94280F6B017C01DA
:1046A00020E030E040EA51E40E94AA6E87FF4AC051
:1046B000A7019601F10160817181828193810E943D
:1046C000B16E762EA72EB82E092F762F272F3A2DD2
:1046D0004B2D502F60914B0D70914C0D80914D0DD5
:1046E00090914E0D0E947F7160934B0D70934C0D15
:1046F00080934D0D90934E0D272D3A2D4B2D502F1D
:10470000EF8DF8A160817181828193810E947F7118
:10471000EF8DF8A16083718382839383F4016081BC
:104720007181828193810E944A6F272D3A2D4B2DF2
:10473000502F0E947F710E941E6FF401608371836D
:1047400082839383F101C082D182E282F38207C027
:104750000E94280FF10160837183828393831F5F1E
:10476000F4E02F0E311C2F8D38A12C5F3F4F38A362
:104770002F8F34E0830E911C143009F080CF1FC4BA
:10478000EBE3F3E007C09091C00095FFFCCF80936E
:10479000C600319684918111F6CF11C4E6EDF3E0A5
:1047A00007C09091C00095FFFCCF8093C600319662
:1047B00084918111F6CF4091F5025091F6026091FB
:1047C000F7027091F80222E030E081EC95E00E945F
:1047D000E12EE9EDF3E007C09091C00095FFFCCF1A
:1047E0008093C600319684918111F6CF4091F902F1
:1047F0005091FA026091FB027091FC0222E030E0DD
:1048000081EC95E00E94E12EECEDF3E007C0909181
:10481000C00095FFFCCF8093C60031968491811132
:10482000F6CF4091FD025091FE026091FF0270911F
:10483000000322E030E081EC95E00E94E12EEFEDF4
:10484000F3E007C09091C00095FFFCCF8093C600B5
:10485000319684918111F6CF40910103509102036A
:10486000609103037091040322E030E081EC95E055
:104870000E94E12EE2EEF3E007C09091C00095FFA8
:10488000FCCF8093C600319684918111F6CF0E94AF
:104890002E580E944C6F2091730D3091740D4091F1
:1048A000750D5091760D0E94B16EAB01BC0122E0F6
:1048B00030E081EC95E00E94E12EECEEF3E007C0E1
:1048C0009091C00095FFFCCF8093C60031968491F3
:1048D0008111F6CF81E00E942E580E944C6F2091EA
:1048E000770D3091780D4091790D50917A0D0E949D
:1048F000B16EAB01BC0122E030E081EC95E00E949A
:10490000E12EEFEEF3E007C09091C00095FFFCCFE1
:104910008093C600319684918111F6CF82E00E9487
:104920002E580E944C6F20917B0D30917C0D409150
:104930007D0D50917E0D0E94B16EAB01BC0122E055
:1049400030E081EC95E00E94E12E8091C00085FF6F
:10495000FCCF32C380E001C081E00E946E512FC3C2
:10496000E2EFF3E007C09091C00095FFFCCF809389
:10497000C600319684918111F6CF329B03C0E7EBDC
:10498000F1E009C0EAEBF1E006C09091C00095FFAC
:10499000FCCF8093C60081918111F7CFE9EFF3E05E
:1049A00007C09091C00095FFFCCF8093C600319660
:1049B00084918111F6CF339B03C0E7EBF1E009C08E
:1049C000EAEBF1E006C09091C00095FFFCCF809328
:1049D000C60081918111F7CFE0E0F4E007C090912B
:1049E000C00095FFFCCF8093C60031968491811161
:1049F000F6CF349B03C0E7EBF1E009C0EAEBF1E04E
:104A000006C09091C00095FFFCCF8093C6008191B5
:104A10008111F7CF8091C00085FFFCCFCDC240E46B
:104A2000E42E42E0F42E00E010E0F70181917F01D6
:104A30000E943C0F882339F10E94280F23E6C22EE2
:104A40002DE0D22EC00ED11E0E941E6FF601608393
:104A50007183828393830E94280F37E3C32E3DE046
:104A6000D32EC00ED11EF801ED58F24F20813181B6
:104A7000428153810E947F710E941E6FF601608304
:104A80007183828393830C5F1F4F0031110569F698
:104A900096C200E412E093E8E92E9DE0F92EF801B9
:104AA00081918F010E943C0F882339F00E94280FCA
:104AB000F7016083718382839383F4E0EF0EF11C2E
:104AC00022E00434120759F77AC283E50E943C0FB2
:104AD000882351F00E94280F60935B0D70935C0D4A
:104AE00080935D0D90935E0D84E50E943C0F8823BA
:104AF00009F465C20E94280F6093570D7093580DFA
:104B00008093590D90935A0D5AC283E50E943C0F31
:104B1000882351F00E94280F60935F0D7093600D01
:104B20008093610D9093620D84E50E943C0F882371
:104B300051F00E94280F6093470D7093480D8093A9
:104B4000490D90934A0D82E40E943C0F882361F046
:104B50000E94280F0E941E6F6093930D7093940D16
:104B60008093950D9093960D88E50E943C0F8823C5
:104B700051F00E94280F6093530D7093540D809351
:104B8000550D9093560D8AE50E943C0F882351F0F5
:104B90000E94280F60934F0D7093500D8093510D1C
:104BA0009093520D85E40E943C0F882309F407C2BC
:104BB0000E94280F60934B0D70934C0D80934D0D08
:104BC00090934E0DFCC100E412E089EEE82E82E0E5
:104BD000F82EF80181918F010E943C0F882339F053
:104BE0000E94280FF7016083718382839383F4E02E
:104BF000EF0EF11C22E00334120759F7E0C183E500
:104C00000E943C0F882309F4DAC10E94280F0E94F9
:104C1000196F70931B0160931A0181E08093050363
:104C2000CEC183E50E943C0F882309F4C8C10E94CD
:104C3000280F0E94196F7093190160931801BFC16A
:104C400080E50E943C0F882351F00E94280F60935A
:104C5000520170935301809354019093550189E45C
:104C60000E943C0F882381F00E94280F2DEB37E330
:104C700046E05EE30E947F7160934E0170934F01A6
:104C8000809350019093510184E40E943C0F88234B
:104C900081F00E94280F2DEB37E346E05EE30E948F
:104CA000B16E60934A0170934B0180934C019093D5
:104CB0004D0183E40E943C0F882351F00E94280F8D
:104CC0006093460170934701809348019093490196
:104CD0000E946C58E4E0F2E006C09091C00095FF9D
:104CE000FCCF8093C60081918111F7CFE7E0F2E01D
:104CF00006C09091C00095FFFCCF8093C6008191C3
:104D00008111F7CF409152015091530160915401AC
:104D10007091550122E030E081EC95E00E94E12E97
:104D2000EBE0F2E006C09091C00095FFFCCF8093CD
:104D3000C60081918111F7CF2DEB37E346E05EE3AA
:104D400060914E0170914F018091500190915101FD
:104D50000E94B16EAB01BC0122E030E081EC95E035
:104D60000E94E12EEFE0F2E006C09091C00095FFB6
:104D7000FCCF8093C60081918111F7CF2DEB37E3F3
:104D800046E05EE360914A0170914B0180914C01D5
:104D900090914D010E947F71AB01BC0122E030E097
:104DA00081EC95E00E94E12EE3E1F2E006C09091F3
:104DB000C00095FFFCCF8093C60081918111F7CF91
:104DC0002DEB37E346E05EE36091460170914701C9
:104DD00080914801909149010E947F71AB01BC0113
:104DE00022E030E081EC95E00E94E12E8091C0004D
:104DF00085FFFCCFE1C081E00E94D550E0C083E593
:104E00000E943C0F882319F00E94280F04C060E024
:104E100070E086E193E40E94295DD1C00E94D457DE
:104E2000CEC00E943F17CBC080E001C081E00E944D
:104E30006118C5C00E94BE0BC2C01092E6028091EC
:104E4000A4059091A505A091A605B091A705809312
:104E50007A0590937B05A0937C05B0937D050E9415
:104E60007F0FADC084E50E943C0F882309F463C026
:104E70000E94280F0E941E6F60939F05662391F188
:104E8000E7ECF0E007C09091C00095FFFCCF809365
:104E9000C600319684918111F6CFE7E1F2E006C0B9
:104EA0009091C00095FFFCCF8093C6008191811145
:104EB000F7CF40E050E060919F0581EC95E00E94C3
:104EC000D02DE9E1F2E006C09091C00095FFFCCF43
:104ED0008093C60081918111F7CF8091C00085FF3A
:104EE000FCCF6AC01092E802E7ECF0E007C09091B6
:104EF000C00095FFFCCF8093C6003196849181114C
:104F0000F6CFEAE2F2E006C09091C00095FFFCCF38
:104F10008093C60081918111F7CF6091E8024AE049
:104F200050E070E081EC95E00E94E82D8091C00097
:104F300085FFFCCF41C0E7ECF0E007C09091C000D6
:104F400095FFFCCF8093C600319684918111F6CFF6
:104F5000E7E0F4E007C09091C00095FFFCCF80939C
:104F6000C600319684918111F6CF80916E059091A3
:104F70006F0520E6289FF001299FF00D1124E651CE
:104F8000FC4F06C09091C00095FFFCCF8093C600F7
:104F900081918111F7CFE9E1F4E007C09091C00061
:104FA00095FFFCCF8093C600319684918111F6CF96
:104FB0008091C00085FFFCCF8AE08093C6000E94EC
:104FC000570F8DC080E090E00E94140A0C94661B7D
:104FD00081E090E00E94140A0C94711B82E090E042
:104FE0000E94140A0C947C1B0E94310FAB01609349
:104FF000DC035093DD038093DE039093DF03BC0159
:1050000089EB93E00E94F931DACF0E94280F0E94C9
:10501000196F8B01E4E4F2E00C940D1F0E94252B24
:105020006B017C0115CA0E94252B60938205709349
:10503000830580938405909385050E94252B6093BA
:105040008605709387058093880590938905B7CF6F
:105050000E94252B681979098A099B09693E7340CA
:105060008105910508F0FBC87AC90E94D4575E9A61
:105070000E944258A4CF0E94D45788E50E943C0F5A
:105080008111C8CAC8CAE62FF0E0EE0FFF1FE45036
:10509000F24F808191810E94595969A37AA38BA311
:1050A0009CA360919F05E62FF0E0EE0FFF1FE050FC
:1050B000F24F808191810E94595920E030E040E810
:1050C0005FE30E94D16D9B01AC0169A17AA18BA124
:1050D0009CA10E94AA6E18160CF0A0CFB9C9A69682
:1050E0000FB6F894DEBF0FBECDBFDF91CF911F91F9
:1050F0000F91FF90EF90DF90CF90BF90AF909F9077
:105100008F907F906F905F904F903F902F90089579
:10511000CF93DF938091E6039091E703039714F414
:105120000E94AB0F60E08CE093E00E94F4698091F4
:10513000E6039091E703892B09F460C080910C038A
:10514000882309F443C080916E0590916F0520E695
:10515000289FE001299FD00D1124C651DC4F6CE33C
:1051600072E0CE010E94C675892BB9F4BE018CE0B5
:1051700093E00E948669E7EAF1E007C09091C000E1
:1051800095FFFCCF8093C600319684918111F6CFB4
:105190008091C00085FFFCCF15C08CE093E00E9499
:1051A000E86AEAEAF1E007C09091C00095FFFCCF01
:1051B0008093C600319684918111F6CF8091C00012
:1051C00085FFFCCF8AE08093C60002C00E94321A9D
:1051D0008091E6039091E70301979093E703809312
:1051E000E60380916E0590916F05019664E070E092
:1051F0000E94687290936F0580936E050E94255AF5
:1052000081E00E943716DF91CF910C94D850CF9255
:10521000DF92EF92FF920F931F93CF93DF9300D013
:1052200000D0CDB7DEB740E052EC61E070E081EC39
:1052300095E00E94D22CEAEDF0E007C09091C0000A
:1052400095FFFCCF8093C600319684918111F6CFF3
:105250008091C00085FFFCCF8AE08093C60087EC78
:1052600090E0FC0107C03091C00035FFFCCF2093D7
:10527000C600319624912111F6CF24B720FF14C027
:10528000E0EEF0E007C04091C00045FFFCCF309356
:10529000C600319634913111F6CF3091C00035FF00
:1052A000FCCF3AE03093C60021FF14C0E8EEF0E0F6
:1052B00007C04091C00045FFFCCF3093C600319637
:1052C00034913111F6CF3091C00035FFFCCF3AE078
:1052D0003093C60022FF14C0E8EFF0E007C0409111
:1052E000C00045FFFCCF3093C60031963491311198
:1052F000F6CF3091C00035FFFCCF3AE03093C600C6
:1053000023FF14C0E9E0F1E007C04091C00045FF71
:10531000FCCF3093C600319634913111F6CF3091E5
:10532000C00035FFFCCF3AE03093C60025FF14C023
:10533000E9E1F1E007C03091C00035FFFCCF2093D8
:10534000C600319624912111F6CF2091C00025FF8F
:10535000FCCF2AE02093C60014BEE9E2F1E007C0CA
:105360003091C00035FFFCCF2093C60031962491C8
:105370002111F6CFE1E3F1E007C03091C00035FF25
:10538000FCCF2093C600319624912111F6CF2091B5
:10539000C00025FFFCCF2AE02093C600FC01249129
:1053A000E7ECF0E008C03091C00035FFFCCF20935F
:1053B000C600319624912111F6CFEBE3F1E007C04E
:1053C0003091C00035FFFCCF2093C6003196249168
:1053D0002111F6CFEBE4F1E007C03091C00035FFBA
:1053E000FCCF2093C600319624912111F6CFE6E53B
:1053F000F1E007C03091C00035FFFCCF2093C6001C
:10540000319624912111F6CFE2E6F1E007C0309108
:10541000C00035FFFCCF2093C600319624912111A6
:10542000F6CF2091C00025FFFCCF2AE02093C600D4
:10543000FC018491E7ECF0E008C09091C00095FF7A
:10544000FCCF8093C600319684918111F6CFE6E6B9
:10545000F1E007C09091C00095FFFCCF8093C6009B
:10546000319684918111F6CF0E94990E4AE050E066
:10547000BC0181EC95E00E94E82DE5E7F1E007C072
:105480009091C00095FFFCCF8093C6003196849127
:105490008111F6CF4AE050E060ED74E081EC95E0D8
:1054A0000E94E82D8091C00085FFFCCF8AE08093A8
:1054B000C60010926A0510926B0510926C0510924E
:1054C0006D0580E00E94611873E6C72E7DE0D72E3F
:1054D000E3E7EE2EEDE0FE2E07E31DE0F60161911D
:1054E0007191819191916F01F701219131914191D8
:1054F00051917F0129833A834B835C830E944A6FD9
:1055000029813A814B815C810E947F710E941E6FCC
:10551000F80161937193819391938F01F3E7CF1613
:10552000FDE0DF06D9F60E94AA5C0E94F3430F90CB
:105530000F900F900F90DF91CF911F910F91FF90DF
:10554000EF90DF90CF900C9488570E94872B0E9499
:1055500007290E948828FDCF24E832E0FC0131832E
:1055600020832581222319F002960C94E0320895BD
:10557000CF93DF93EC0185559F4F0E94AC2ACE015B
:1055800085599F4F0E94AC2ACE01825B9F4F0E949B
:10559000AC2ACE01C1960E94AC2ACE014296DF9180
:1055A000CF910C94AC2A8CE093E00C9412638CE0C5
:1055B00093E00C94B82A1F920F920FB60F92112409
:1055C0002F933F938F939F93AF93BF938091B80591
:1055D0009091B905A091BA05B091BB053091C00575
:1055E000232F2D5F2D3720F40196A11DB11D05C07D
:1055F000232F2A570296A11DB11D2093C005809329
:10560000B8059093B905A093BA05B093BB058091F6
:10561000BC059091BD05A091BE05B091BF05019656
:10562000A11DB11D8093BC059093BD05A093BE053F
:10563000B093BF05BF91AF919F918F913F912F91F3
:105640000F900FBE0F901F9018950F931F938FB759
:10565000F8940091B8051091B9052091BA053091E0
:10566000BB058FBFB801C9011F910F9108950F931A
:105670001F939FB7F8940091BC051091BD05209130
:10568000BE053091BF0586B5A89B06C08F3F21F0AF
:105690000F5F1F4F2F4F3F4F9FBF322F212F102FD4
:1056A0000027080F111D211D311D42E0000F111FA1
:1056B000221F331F4A95D1F7B801C9011F910F91DD
:1056C0000895CF92DF92EF92FF92CF93DF936B0119
:1056D0007C010E94372BEB010EC00E94372B6C1B04
:1056E0007D0B683E734038F081E0C81AD108E108AC
:1056F000F108C851DC4FC114D104E104F10469F789
:10570000DF91CF91FF90EF90DF90CF900895789444
:1057100084B5826084BD84B5816084BD85B58260B6
:1057200085BD85B5816085BDEEE6F0E08081816054
:105730008083E1E8F0E01082808182608083808154
:1057400081608083E0E8F0E0808181608083E1EB2C
:10575000F0E0808184608083E0EBF0E08081816014
:105760008083EAE7F0E080818460808380818260CA
:1057700080838081816080838081806880831092B3
:10578000C10008951F93CF93DF93182FEB0161E0C1
:105790000E944D2C209711F460E004C0CF3FD1054A
:1057A00039F461E0812FDF91CF911F910C94692C26
:1057B000E12FF0E0E05FFC4EE491E330B9F028F433
:1057C000E13051F0E230B1F50CC0E63019F1E730CC
:1057D00049F1E43079F514C084B5806884BDC7BD53
:1057E0002EC084B5806284BDC8BD29C08091800070
:1057F000806880938000D0938900C09388001FC088
:1058000080918000806280938000D0938B00C09351
:105810008A0015C08091B00080688093B000C0936A
:10582000B3000DC08091B00080628093B000C0933F
:10583000B40005C0C038D1050CF0B3CFADCFDF91B7
:10584000CF911F910895833069F028F48130A1F041
:10585000823011F514C08630B1F08730C1F0843049
:10586000D9F404C0809180008F7703C080918000BC
:105870008F7D80938000089584B58F7702C084B5B2
:105880008F7D84BD08958091B0008F7703C0809193
:10589000B0008F7D8093B000089590E0FC01E05D42
:1058A000FC4E2491FC01E05BFC4EE491EE2381F080
:1058B000F0E0EB58FC4EA491B0E09FB7F8948C91C7
:1058C000611103C02095822301C0822B8C939FBF5E
:1058D00008950F931F93CF93DF931F92CDB7DEB739
:1058E000A82FB0E0FD01E05FFC4E8491FD01E05D7A
:1058F000FC4E1491FD01E05BFC4E04910023B9F0D5
:10590000882321F069830E94232C6981E02FF0E035
:10591000E059FC4EA491B0E09FB7F8948C916111CE
:1059200003C01095812301C0812B8C939FBF0F90E2
:10593000DF91CF911F910F9108951F920F920FB693
:105940000F9211242F933F934F935F936F938F93F5
:105950009F93EF93FF936091C60020914206309190
:105960004306C90101968F779927409144065091CB
:1059700045068417950741F0F901EE53FA4F60830D
:105980009093430680934206FF91EF919F918F91F0
:105990006F915F914F913F912F910F900FBE0F909C
:1059A0001F9018959A01AB01211581EE380741052A
:1059B0005105A9F42AC03093C5002093C4008091FA
:1059C000C10080618093C1008091C1008860809394
:1059D000C1008091C10080688093C100089582E079
:1059E0008093C00060E079E08DE390E00E949E72B9
:1059F0002150310941095109CA01B90122E030E0C1
:105A000040E050E00E949E72D6CF1092C00020E18C
:105A100030E0D1CF80914406909145062091420616
:105A2000309143062817390769F0FC01EE53FA4F0D
:105A3000208101968F77992790934506809344069D
:105A400030E002C02FEF3FEFC90108958091440676
:105A500090914506909343068093420608956F9275
:105A60007F928F929F92AF92BF92CF92DF92EF92EE
:105A7000FF920F931F93CF93DF93CDB7DEB7A0971D
:105A80000FB6F894DEBF0FBECDBF8C014115510596
:105A900061057105E1F420E030E040E350E060E0B2
:105AA00070E0A0960FB6F894DEBF0FBECDBFDF91B9
:105AB000CF911F910F91FF90EF90DF90CF90BF900B
:105AC000AF909F908F907F906F900C94D72D66240D
:105AD0006394712C6C0E7D1EC12CD12C7601822E0C
:105AE000912CA12CB12CCB01BA01A50194010E94EB
:105AF0007C72FA01D3016D933D01BFEFCB1ADB0A33
:105B0000EB0AFB0AA901BF014115510561057105A9
:105B100051F781E0C81AD108E108F1081AC0E1E0A4
:105B2000F0E0EC0FFD1FEC0DFD1D8081482F8A3049
:105B300010F4405D01C0495C50E060E070E020E09E
:105B400030E0C8010E94D72DA1E0CA1AD108E108AF
:105B5000F108BFEFCB16DB06EB06FB0601F7A096BC
:105B60000FB6F894DEBF0FBECDBFDF91CF911F916E
:105B70000F91FF90EF90DF90CF90BF90AF909F90EC
:105B80008F907F906F9008952115310539F48091A1
:105B9000C00085FFFCCF4093C60008950C942F2DC4
:105BA0009A01462F50E060E070E00C94C42D21155E
:105BB000310539F48091C00085FFFCCF4093C600C9
:105BC00008952A30310511F40C94142E0C942F2DC5
:105BD0009A01AB01662757FD6095762F0C94D72D5F
:105BE000CF93DF93EC0120E030E04DE050E060E047
:105BF00070E00E94D72D20E030E04AE050E060E005
:105C000070E0CE01DF91CF910C94D72DCF93DF932D
:105C1000EC019A01AB0160E070E00E94C42DCE015E
:105C2000DF91CF910C94F02DCF92DF92EF92FF9203
:105C3000CF93DF93EC016A017B0177FF10C020E076
:105C400030E04DE250E060E070E00E94D72DF0942B
:105C5000E094D094C094C11CD11CE11CF11C2AE03A
:105C6000B701A601CE01DF91CF91FF90EF90DF90B9
:105C7000CF900C942F2D8F929F92AF92BF92CF9284
:105C8000DF92EF92FF920F931F93CF93DF938C01DC
:105C90004A015B01C22F20E030E0A901C501B40137
:105CA0000E94AA6E87FF0DC020E030E04DE250E078
:105CB00060E070E0C8010E94D72DB7FAB094B7F841
:105CC000B094D0E060E070E080E09FE307C020E0A7
:105CD00030E040E251E40E94B16EDF5FDC13F7CFA9
:105CE000262F372F482F592FC501B4010E94D16D9F
:105CF000D62EE72EF82ED92F0E941E6F962EA72E95
:105D0000B82EC92E0E944A6F9B01AC016D2D7E2DCD
:105D10008F2D9D2F0E94D06DD62FF72EE82ED92ED5
:105D20002AE0492D5A2D6B2D7C2DC8010E942F2D64
:105D3000CC23C1F1EEE7F2E006C09091C00095FFE0
:105D4000FCCF8093C60081918111F7CF2BC020E05A
:105D500030E040E251E46D2F7F2D8E2D9D2D0E946D
:105D60007F714B015C01792D9B2D0E94196F6B0196
:105D7000EE24D7FCE094FE2CB701A601C8010E94D6
:105D8000142EC701B6010E944C6F9B01AC01682D17
:105D9000792D8A2D9B2D0E94D06DD62FF72EE82EBF
:105DA000D92EC150C111D3CFDF91CF911F910F9147
:105DB000FF90EF90DF90CF90BF90AF909F908F902B
:105DC00008950C943B2ECF93DF93EC019C012C5F44
:105DD0003F4F41E050E060E070E0898D9A8D0E9475
:105DE000AC398823A1F04D895E896F89788D452B68
:105DF000462B472B71F44C815D816E817F814D8BE9
:105E00005E8B6F8B788F89818068898302C080E088
:105E100001C081E0DF91CF910895CF92DF92EF92A0
:105E2000FF921F93CF93DF93EC0149895A896B89C5
:105E30007C89403E5F4F6F41710508F06DC00E9444
:105E4000E32E882309F468C00E94B737882309F439
:105E500063C0E98DFA8DCC80DD80EE80FF8032E07A
:105E6000C31AD108E108F108058404C0CC0CDD1C7C
:105E7000EE1CFF1C0A94D2F746855785608971890C
:105E8000C40ED51EE61EF71E81E080934C06C0921C
:105E90004F08D0925008E0925108F092520880E0EA
:105EA00092E0EFE4F6E0DF019C011D9221503040CA
:105EB000E1F711E011C0B701A601410F511D611DAD
:105EC000711D2FE436E080914D0690914E060E94A0
:105ED000866D882309F11F5FE98DFA8D848118177B
:105EE00050F3C12C82E0D82EE12CF12C058404C0A3
:105EF000CC0CDD1CEE1CFF1C0A94D2F749895A8990
:105F00006B897C894C0D5D1D6E1D7F1D498B5A8BE5
:105F10006B8B7C8B81E001C080E0DF91CF911F9182
:105F2000FF90EF90DF90CF900895CF93DF93EC0137
:105F300041E0611101C040E06C857D858E859F85C3
:105F40000E94F237882341F0288980E2289F90013F
:105F50001124215B394F02C020E030E0C901DF91FC
:105F6000CF910895CF93FB0120E030E231932F5F72
:105F70002B30E1F7DC0130E0C7E01CC0CA3051F142
:105F800038E0CAE017C0E21729F1FC010196E4915C
:105F9000E111F9CFC317F0F02132E0F02F37D0F440
:105FA000FB01E30FF11D822F81568A3108F4205244
:105FB00020833F5FCD012D91211109C0FA0180831B
:105FC000918381E0FB019081903259F403C02F321C
:105FD00019F4F4CF80E005C02E3281F28CEB96E00C
:105FE000D4CFCF9108950F931F93CF93DF93EC01FC
:105FF0008B018B81882311F080E044C0FB018789ED
:10600000803131F528C083E08B83F801428D538DB8
:10601000648D758D4D8B5E8B6F8B788F9E012F5E9F
:106020003F4FC8010E94AC38882331F31A8F098F83
:1060300081E089831C821D821E821F821886198638
:106040001A861B861C861D861E861F86188A1AC005
:10605000803291F6D8CF82E08B831D8A1E8A1F8AF8
:10606000188EFB01408D518D60E070E095E0440F8B
:10607000551F661F771F9A95D1F7498B5A8B6B8BEB
:106080007C8BD4CFDF91CF911F910F9108952F92E8
:106090003F924F925F926F927F928F929F92AF92B8
:1060A000BF92CF92DF92EF92FF920F931F93CF9305
:1060B000DF9300D000D0CDB7DEB79C838B831A016D
:1060C000DC0113968C91811103C02FEF3FEFEEC0DE
:1060D000EB81FC81818180FFF8CFBCC01601201AC2
:1060E000310A21015B018B819C8104969A8389830B
:1060F000ABC0AB81BC8118960D911D912D913C9147
:106100001B97D901C8019170AA27BB273C01EB81DD
:10611000FC8143816801790159E0F694E794D794B2
:10612000C7945A95D1F7818D928D423061F4DC018C
:106130005A966D917D918D919C915D976C0D7D1D11
:106140008E1D9F1D4BC0FC0194809A949C2061146D
:10615000710401F591101EC0012B022B032B59F481
:10616000EB81FC8185899689A789B08D848395838D
:10617000A683B7830FC0AB81BC8114964D915D910E
:106180006D917C91179729813A810E942B38882341
:1061900009F49BCFAB81BC815996ED91FC915A9744
:1061A00014966D917D918D919C9117976250710914
:1061B00081099109058404C0660F771F881F991F04
:1061C0000A94D2F70685178520893189600F711FDF
:1061D000821F931F690D711D811D911D20E032E00A
:1061E0002619370972012415350508F47901E114DF
:1061F000B2E0FB0609F054C000914F08109150081E
:106200002091510830915208601771078207930757
:10621000D9F546C0C301815B994FA701BC01C501F7
:106220000E948375AE0CBF1CEB81FC81008511853B
:10623000228533850E0D1F1D211D311D00871187FD
:10624000228733874E185F084114510409F051CF5B
:1062500091012CC0EB81FC81C188D288E388F4884D
:1062600000851185228533852A01612C712C460118
:106270005701801A910AA20AB30A481459046A0401
:106280007B0408F02BCF2DCF9501AB01BC01809191
:106290004D0690914E060E94636C8111C3CF15CFBD
:1062A00040E00E94F2378111B5CF0FCFC9010F90A6
:1062B0000F900F900F90DF91CF911F910F91FF9052
:1062C000EF90DF90CF90BF90AF909F908F907F9096
:1062D0006F905F904F903F902F900895CF93DF93F2
:1062E0001F92CDB7DEB741E050E0BE016F5F7F4F38
:1062F0000E944730019719F4298130E002C02FEF46
:106300003FEFC9010F90DF91CF9108950F931F9335
:10631000CF93DF938C01EB01FC018381823028F164
:1063200040855185628573854F715527662777278C
:10633000452B462B472BC9F440E250E0BE01C80173
:106340000E9447308032910521F0892B71F480E062
:106350000DC088818823D9F3853E71F38E3261F3B5
:106360008B8583FDE9CF80E201C08FEFDF91CF9174
:106370001F910F910895CF92DF92EF92FF92CF93EA
:10638000DF93EC018B81823018F420E030E029C0EB
:10639000C884D984EA84FB8475E0F694E794D794A2
:1063A000C7947A95D1F78FE0C822DD24EE24FF242C
:1063B000CE010E946E3197FDE8CF488559856A85E8
:1063C0007B85415E5F4F6F4F7F4F488759876A8754
:1063D0007B87960165E0220F331F6A95E1F7215B09
:1063E000394FC901DF91CF91FF90EF90DF90CF90AF
:1063F00008958F929F92AF92BF92CF92DF92EF92C9
:10640000FF920F931F93CF93DF93EC014A015B013F
:106410002B81222309F475C089899A89AB89BC89AB
:1064200084179507A607B70708F46BC06CC08114E2
:106430009104A104B10449F41C821D821E821F82B2
:10644000188619861A861B865AC0088519852A85DA
:106450003B85E98DFA8D858590E00996B901A80103
:106460004150510961097109082E04C0769567955C
:10647000579547950A94D2F7CC24CA94DC2C760120
:10648000C80CD91CEA1CFB1C04C0F694E794D794F2
:10649000C7948A95D2F7C416D506E606F70620F00B
:1064A000012B022B032B49F44D895E896F89788D6E
:1064B0004C835D836E837F8316C0C41AD50AE60AB7
:1064C000F70A11C04C815D816E817F819801898DB1
:1064D0009A8D0E942B3891E0C91AD108E108F10881
:1064E000811104C014C08E010C5F1F4FC114D10470
:1064F000E104F10439F788869986AA86BB8681E093
:1065000006C080E004C0223009F091CFF4CFDF91C3
:10651000CF911F910F91FF90EF90DF90CF90BF90A0
:10652000AF909F908F9008950F931F93CF93DF9319
:10653000EC018B818823E1F1898187FF33C061E021
:10654000CE010E94952F8C01009791F1FC01808172
:10655000853E71F18B81823040F449895A896B897B
:106560007C89448F558F668F778F4D895E896F89BF
:10657000788DF801538F428F758B648BE0914606BE
:10658000F0914706309759F0B8016A5E7F4FC80115
:1065900048960995F801808D918D938B828B898126
:1065A0008F778983DF91CF911F910F910C94B7372B
:1065B00081E0888380E0DF91CF911F910F91089552
:1065C000CF93DF93EC010E9494321B82DF91CF9135
:1065D0000895FC01238121110C94E03208956F92FB
:1065E0007F928F929F92AF92BF92CF92DF92EF9263
:1065F000FF920F931F93CF93DF9300D000D0CDB7BE
:10660000DEB73C016A017B01FC018381813009F026
:1066100083C0818181FF80C081C0452B462B472BE1
:1066200009F478C0F30180849184A284B384B70113
:10663000A601C3010E94F931811101C06DC0F301AF
:10664000818D928DC114D104E104F10479F445895E
:1066500056896789708D0E94BD3A882309F45CC011
:10666000F301158A168A178A108E3AC0F301448105
:106670005581668177819E012F5F3F4F0E942B38A5
:10668000882309F449C049815A816B817C81F301D7
:10669000818D928DFC012789203139F4483FFFEF2D
:1066A0005F0761057105E0F407C0483F2FEF52070F
:1066B00062072FE07207A0F40E94BD3A882361F1BF
:1066C000F30144815581668177810FEF1FEF2FEF32
:1066D0003FE0818D928D0E941439811101C01CC050
:1066E000F301C18AD28AE38AF48A81818068818336
:1066F000C3010E949432882379F0B701A6018C145B
:106700009D04AE04BF0410F4B501A401C3010E94AE
:10671000F93110C081E00EC080E00CC0F301418966
:106720005289638974894C155D056E057F0508F0F3
:1067300074CFF2CF0F900F900F900F90DF91CF9109
:106740001F910F91FF90EF90DF90CF90BF90AF908F
:106750009F908F907F906F900895CF93DF93EC017F
:1067600040E050E0BA010E94EF32882371F061E00E
:10677000CE010E94952F009741F025EEFC01208369
:106780001B82DF91CF910C94B73780E0DF91CF91DE
:106790000895FF920F931F93CF93DF93EC01F42E94
:1067A00080E2689FF0011124E15BF94F83858171DC
:1067B00021F0842F827109F05CC000914F08109184
:1067C000500820915108309152080C871D872E8760
:1067D0003F87688B4489558960E070E0BA0155278E
:1067E0004427028D138D20E030E0402B512B622B8B
:1067F000732B4D8B5E8B6F8B788F8385887151F4F3
:10680000048D158D268D378D098B1A8B2B8B3C8B28
:1068100081E00CC0803169F59E012F5E3F4F898D6C
:106820009A8D0E94AC38882321F184E08B838F2DD0
:106830008F7089831C821D821E821F821886198692
:106840001A861B86F4FE18C040E050E0BA01CE0163
:106850000E94EF32811110C012C049895A896B8998
:106860007C89CE01DF91CF911F910F91FF900C9405
:10687000F9311B8280E003C0F5FCEFCF81E0DF91AE
:10688000CF911F910F91FF9008956F927F928F92F9
:106890009F92AF92BF92CF92DF92EF92FF920F93AF
:1068A0001F93CF93DF935C01EB014A01722E898D18
:1068B0009A8DF501928F818F40E050E0BA01CE01B0
:1068C0000E94F931612C33C045E036952795179524
:1068D00007954A95D1F70F70CE010E94BB31DC01BC
:1068E000009709F495C08C91882311F0853EB1F48E
:1068F000611010C0C0904F08D0905008E09051082F
:10690000F0905208F501C486D586E686F786008B9E
:10691000662463948C9181110AC075C04BE050E0ED
:10692000BD01C4010E947675009709F46FC0088507
:1069300019852A853B85C988DA88EB88FC880C157F
:106940001D052E053F0508F4BFCF5DC071FE60C078
:10695000662051F0F501008961E0C5010E94952F84
:10696000EC01009771F454C08B81823009F450C05F
:10697000CE010E940D2F882309F44AC0CFE4D6E04F
:1069800000E080E2FE0111928A95E9F78BE0F401C4
:10699000DE0101900D928A95E1F7E0914606F091B3
:1069A0004706309739F0BE01625F7F4FCE014096B7
:1069B000099508C081E298E2998B888B80E098E085
:1069C0009F878E87888999899B8B8A8B998F888FDF
:1069D0008E859F859F8B8E8B0E94B7378823C1F051
:1069E000472D602FC501DF91CF911F910F91FF902F
:1069F000EF90DF90CF90BF90AF909F908F907F905F
:106A00006F900C94C93376FCA1CF02C077FEE8CF1B
:106A100080E0DF91CF911F910F91FF90EF90DF9079
:106A2000CF90BF90AF909F908F907F906F90089580
:106A30005F926F927F928F929F92AF92BF92CF920E
:106A4000DF92EF92FF920F931F93CF93DF93CDB717
:106A5000DEB7C354D1090FB6F894DEBF0FBECDBF69
:106A60005C016B0124965FAF4EAF2497522E1C8EB3
:106A70001F8E19821C826115710511F410E075C01A
:106A8000FC0183818111FACF2496EEADFFAD2497EE
:106A900080818F3239F0760117C031962496FFAF8E
:106AA000EEAF24972496EEADFFAD249780818F3210
:106AB000A1F3F60183818250823060F4ECCFEE24A2
:106AC000E394F12CEC0EFD1E8E01045E1F4F480175
:106AD00038010CC0F601618D728DCE0101960E94C5
:106AE000F32F8111ECCFCACF78018301AE014E5B49
:106AF0005F4FBE01695C7F4F24968EAD9FAD24979A
:106B00000E94B22F811106C0B9CF31962496FFAFF3
:106B1000EEAF24972496EEADFFAD249780818F329F
:106B2000A1F38823C9F021E0AE01495C5F4FB701B2
:106B3000C8010E944534882309F4A0CFEC14FD0459
:106B400019F0C7010E94E0320815190569F68E0197
:106B50000F5F1F4F7301CACF252DAE01495C5F4FF8
:106B6000B701C5010E944534182FCE0101960E943D
:106B7000E932CE014C960E94E932812FCD5BDF4F86
:106B80000FB6F894DEBF0FBECDBFDF91CF911F913E
:106B90000F91FF90EF90DF90CF90BF90AF909F90BC
:106BA0008F907F906F905F9008951F93CF93DF93A6
:106BB000CDB7DEB76B970FB6F894DEBF0FBECDBF73
:106BC000AB0119821C8222E0BC01CE0101960E9419
:106BD0001835882331F0CE0101960E94AD33182F6D
:106BE00001C010E0CE0101960E94E932812F6B9620
:106BF0000FB6F894DEBF0FBECDBFDF91CF911F91CE
:106C000008952F923F924F925F927F928F929F9220
:106C1000AF92BF92CF92DF92EF92FF920F931F93AA
:106C2000CF93DF9300D000D000D0CDB7DEB71C01EA
:106C3000162F072F5E834D83DC0113968C911397DB
:106C4000813009F054C111968C9181FF50C155C11A
:106C5000F101418952896389748980859185A28572
:106C6000B38584179507A607B70729F4AD80BE80C2
:106C7000812E902E07C1C1010E94F9318111F6CFFA
:106C800036C1D10159968D919C915A97FC0174801F
:106C90007A94B701A601E9E07695679557954795EF
:106CA000EA95D1F77422F1E0DF22EE24FF242601D9
:106CB00071104AC0C114D10409F046C014964D9118
:106CC0005D916D917C911797411551056105710595
:106CD00061F455960D911D912D913C915897011598
:106CE00011052105310549F522C09E012F5F3F4F57
:106CF0000E942B38882309F4FAC009811A812B815C
:106D00003C81D1015996ED91FC915A978789803148
:106D100039F4083FBFEF1B072105310540F40DC0D2
:106D2000083FEFEF1E072E07EFE03E0730F0C101EE
:106D30000E94E32E811108C0DAC0D10114960D9390
:106D40001D932D933C93179780E092E08419950949
:106D500085018A159B0508F48C01D1015996ED91A6
:106D6000FC915A971496CD90DD90ED90FC9017977A
:106D7000B2E0CB1AD108E108F108058404C0CC0CBC
:106D8000DD1CEE1CFF1C0A94D2F786859785A0892E
:106D9000B189C80ED91EEA1EFB1EC70CD11CE11C0E
:106DA000F11C0115E2E01E0731F580914F0890912A
:106DB0005008A0915108B09152088C159D05AE0560
:106DC000BF0569F410924C068FEF9FEFDC018093B2
:106DD0004F0890935008A0935108B0935208940123
:106DE000B701A60180914D0690914E060E94866DD6
:106DF000811137C07CC04114510419F5D101189696
:106E00004D915D916D917C911B9751968D919D91C6
:106E10000D90BC91A02D481759076A077B0788F091
:106E20000E94B737882309F462C081E080934C0642
:106E3000C0924F08D0925008E0925108F092520848
:106E400008C041E0C701B6010E94F237882309F467
:106E50004EC09201215B394FA801B401C9010E94C3
:106E60008375F101C084D184E284F384C00ED11E05
:106E7000E11CF11CC086D186E286F386800E911E4D
:106E8000A01AB10AF101C084D184E284F384A11470
:106E9000B10409F0F6CE01891289238934890C15D1
:106EA0001D052E053F0530F4D101C18AD28AE38A3F
:106EB000F48A0BC08091460690914706892B59F0C1
:106EC000ED81FE81EF2B39F0D10111968C91119754
:106ED000806811968C93F101818183FD03C02D811F
:106EE0003E810EC0C1010E9494328111F8CF81E031
:106EF000D1018C932FEF3FEF03C082FDA9CEB6CE18
:106F0000C90126960FB6F894DEBF0FBECDBFDF9144
:106F1000CF911F910F91FF90EF90DF90CF90BF9096
:106F2000AF909F908F907F905F904F903F902F9069
:106F30000895DB010D900020E9F7AD0141505109A2
:106F4000461B570B02960C940136CF93DF931F928A
:106F5000CDB7DEB7698341E050E0BE016F5F7F4F80
:106F600002960E9401360F90DF91CF910895809193
:106F70004C068823A9F140914F0850915008609128
:106F80005108709152082FE436E080914D0690919F
:106F90004E060E94866D811102C080E008954091E6
:106FA00048065091490660914A0670914B0641157A
:106FB00051056105710591F02FE436E080914D0691
:106FC00090914E060E94866D882339F310924806F0
:106FD0001092490610924A0610924B0610924C06E7
:106FE00081E00895CF92DF92EF92FF92CF936B01F1
:106FF0007C01C42F80914F0890915008A0915108B6
:10700000B09152088C159D05AE05BF05D1F00E94C8
:10701000B737811102C080E018C02FE436E0B70115
:10702000A60180914D0690914E060E94636C8823C4
:1070300091F3C0924F08D0925008E0925108F0921C
:10704000520881E0C11180934C06CF91FF90EF90E0
:10705000DF90CF900895AF92BF92CF92DF92EF92E0
:10706000FF920F931F93CF93DF935C016A017B0123
:10707000E901FC0141855285638574854F5F5F4F4F
:107080006F4F7F4F4C155D056E057F0510F480E056
:1070900058C0FC018789803129F499278F2D7E2DD6
:1070A0006D2D0CC0803299F7C701B60127E0969587
:1070B0008795779567952A95D1F7F5010389148906
:1070C00025893689600F711F821F931F00914F0819
:1070D00010915008209151083091520860177107A3
:1070E0008207930729F4F50187898031A1F406C04E
:1070F00040E00E94F2378111F6CFC9CFDD24EE24A3
:10710000FF24F601EE0FFF1FE15BF94F80819181B3
:10711000A0E0B0E011C0E894C7F8DD24EE24FF241D
:10712000F601EE0FFF1FEE0FFF1FE15BF94F8081AD
:107130009181A281B381BF7088839983AA83BB8325
:1071400081E0DF91CF911F910F91FF90EF90DF9041
:10715000CF90BF90AF9008956F927F928F929F9241
:10716000AF92BF92CF92DF92EF92FF920F931F9355
:10717000CF93DF9300D000D0CDB7DEB78C01498329
:107180005A836B837C833901C12CD12C7601812CED
:1071900042E0942EA12CB12C49815A816B817C81D3
:1071A0009E012F5F3F4FC8010E942B38882341F179
:1071B000D501C401F801058404C0880F991FAA1FD6
:1071C000BB1F0A94D2F7C80ED91EEA1EFB1E4981C6
:1071D0005A816B817C818789803131F4483F5F4FD0
:1071E0006105710530F4D8CF483F5F4F6F4F7F4046
:1071F00098F2F301C082D182E282F38281E001C081
:1072000080E00F900F900F900F90DF91CF911F9122
:107210000F91FF90EF90DF90CF90BF90AF909F9035
:107220008F907F906F9008956F927F928F929F9230
:10723000AF92BF92CF92DF92EF92FF920F931F9384
:10724000CF93DF9300D0CDB7DEB73C014A015B019D
:10725000423051056105710508F46CC0F3014185A8
:107260005285638574854F5F5F4F6F4F7F4F481521
:1072700059056A057B0508F45DC08789803129F4CA
:10728000FF24EB2CDA2CC92C0DC0803209F052C03F
:107290007501640177E0F694E794D794C7947A95E2
:1072A000D1F7F30183899489A589B689C80ED91EBF
:1072B000EA1EFB1E41E0C701B60129833A830E9402
:1072C000F23729813A818823A9F1F3018789803136
:1072D00059F49924AA24BB24F401EE0FFF1FE15BAB
:1072E000F94F1183008310C0E89487F89924AA24E9
:1072F000BB24F401EE0FFF1FEE0FFF1FE15BF94F00
:107300000083118322833383F3018289823080F0EA
:1073100085819681A781B0858C0D9D1DAE1DBF1DF9
:107320008093480690934906A0934A06B0934B0673
:1073300081E001C080E00F900F90DF91CF911F910D
:107340000F91FF90EF90DF90CF90BF90AF909F9004
:107350008F907F906F9008952F923F924F925F92FF
:107360006F927F928F929F92AF92BF92CF92DF9255
:10737000EF92FF920F931F93CF93DF93CDB7DEB7BA
:107380002F970FB6F894DEBF0FBECDBF1C014C8700
:107390005D876E877F873B872A87DC0119964D9032
:1073A0005D906D907C901C97BFEF4B1A5B0A6B0A47
:1073B0007B0AF90180809180A280B38081149104BE
:1073C000A104B10431F0FFEF8F1A9F0AAF0ABF0A80
:1073D00010C0DC018D909D90AD90BC90B1E0BD835C
:1073E0002C853D854E855F85213031054105510550
:1073F00009F01D82750164011E821F82188619869C
:10740000F10181859285A385B4852E813F814885D0
:107410005985281739074A075B0708F052C04C14F2
:107420005D046E047F0450F4B2E0CB2ED12CE12C2D
:10743000F12C12E0812E912CA12CB12C9E012F5FFA
:107440003F4FB701A601C1010E942B388823C9F123
:1074500049815A816B817C81D701C6010196A11DAA
:10746000B11D452B462B472B19F04C015D010DC07A
:1074700088199909AA09BB092C853D854E855F8528
:1074800082179307A407B50789F08E819F81A8858D
:10749000B9850196A11DB11D8E839F83A887B987E9
:1074A0009FEFC91AD90AE90AF90AAACF0FEF1FEF0D
:1074B0002FEF3FE0A601B701C1010E9414398111ED
:1074C00015C080E041C044244A94542C32014C0C35
:1074D0005D1C6E1C7F1C97018601B301A201C101D6
:1074E0000E941439882369F3730162018C149D048E
:1074F000AE04BF0440F3AA85BB854D915D916D91AB
:107500007C91411551056105710551F4EA85FB85B2
:1075100080829182A282B382FD81F11109C013C0E1
:1075200095018401C1010E9414398111EFCFC9CFA7
:107530002FEF821A920AA20AB20AD1018D929D926D
:10754000AD92BC92139781E02F960FB6F894DEBFF0
:107550000FBECDBFDF91CF911F910F91FF90EF90A4
:10756000DF90CF90BF90AF909F908F907F906F9063
:107570005F904F903F902F900895AF92BF92CF921F
:10758000DF92EF92FF920F931F93CF93DF9300D080
:1075900000D0CDB7DEB75C016A017B0142E050E06C
:1075A00060E070E0FC0140835183628373839E013D
:1075B0002F5F3F4FB701A601C5010E942B388111F3
:1075C00002C080E023C000E010E09801B701A601EE
:1075D000C5010E9414398823A1F3C980DA80EB80A9
:1075E000FC80F5018789803141F4F8EFCF16FFEF79
:1075F000DF06E104F10448F4DACF88EFC8168FEF14
:10760000D806E8068FE0F80690F281E00F900F9020
:107610000F900F90DF91CF911F910F91FF90EF90FE
:10762000DF90CF90BF90AF9008958F929F92AF92CE
:10763000BF92CF92DF92EF92FF920F931F93CF935F
:10764000DF93EC01142F70934E0660934D061F8A52
:1076500052E0C52ED12CE12CF12CC882D982EA82CD
:10766000FB8210924C061092480610924906109226
:107670004A0610924B06CC24CA94DC2C7601C092A8
:107680004F08D0925008E0925108F09252084423DB
:1076900059F1453008F0DDC040E060E070E0CB011A
:1076A0000E94F237882309F4D4C020E1129FF00130
:1076B0001124E350F84F80818F7709F0CAC0C48449
:1076C000D584E684F78434E6C316D104E104F104DA
:1076D00008F4BFC0C084D184E284F384C114D1040F
:1076E000E104F10421F4B5C0C12CD12C760140E0B5
:1076F000C701B6010E94F237882309F4AAC080911D
:107700005A0690915B068115924009F0A2C0209123
:107710005F06222309F49DC080915D0690915E066C
:10772000009709F496C040915C06442309F491C087
:107730002A8B4C831D8650E061E070E006C02E2F3E
:107740002F5F2D87E83008F084C0ED859B010E2E59
:1077500002C0220F331F0A94E2F74217530779F74A
:1077600020916506309166062115310519F040E03B
:1077700050E008C020917306309174064091750660
:10778000509176062D833E834F83588746015701DB
:10779000880E991EA11CB11C8B8A9C8AAD8ABE8A58
:1077A0000091600610916106198F088FA0915F0605
:1077B000B0E00E944572680D791D8A1D9B1D6A8F7D
:1077C0007B8F8C8F9D8F980105E0220F331F0A95C8
:1077D000E1F721503E4F232F33272695DC01CB01C3
:1077E000820F931FA11DB11D8E879F87A88BB98B18
:1077F00080906206909063068114910419F0A12C88
:10780000B12C08C080906F0690907006A090710611
:10781000B0907206A7019601281B390B4A0B5B0B2F
:10782000DA01C901880D991DAA1DBB1D04C0B695BA
:10783000A79597958795EA95D2F789879A87AB8719
:10784000BC87853F3FE09307A105B10520F48CE09C
:107850008F8B80E016C0853F9F4FA105B10510F4C6
:1078600080E10DC040917B0650917C0660917D06C1
:1078700070917E064A8F5B8F6C8F7D8F80E28F8B3D
:1078800081E0DF91CF911F910F91FF90EF90DF90FA
:10789000CF90BF90AF909F908F9008952F923F927E
:1078A0004F925F926F927F928F929F92AF92BF9210
:1078B000CF92DF92EF92FF920F931F93CF93DF93BC
:1078C000CDB7DEB7CA54D1090FB6F894DEBF0FBEEC
:1078D000CDBF1C017E8B6D8B3A012BA30EA3E8A6B6
:1078E000AEAABFAAC8AED9AE34E0239F800111244E
:1078F000400F511F5BAB4AABDA018D909D90AD906C
:10790000BC90FC01E00FF11F208131814281538145
:10791000C501B4010E94D16D6AAF7BAF8CAF9DAF42
:10792000EEA1B4E0EB9F7001112493012E0D3F1DD9
:107930003DAB2CABD9014D905D906D907C90F101E9
:10794000EE0DFF1D2081318142815381C301B201BF
:107950000E94D16D6EAF7FAF21968FAF2197229697
:107960009FAF2297E8A5B4E0EB9FC0011124F1017D
:10797000E80FF91F20813181428153812B8F3C8F89
:107980004D8F5E8FED89FE89E80FF91F608171814F
:10799000828193810E94D06D462F572F682F792FB7
:1079A000498B5A8B6B8B7C8BAD89BE891C968D91D4
:1079B0009D910D90BC91A02D8AA79BA7ACA7BDA7B8
:1079C000D1011C962D913D914D915C911F972F8F68
:1079D00038A349A35AA3B7FAB094B7F8B09477FA8A
:1079E000709477F87094ED89FE89E00FF11F7AADFD
:1079F0006BAD9CAD8DAD272F362F492F582F608151
:107A00007181828193810E94D06D6F8B788F898F75
:107A10009DA3ED89FE89EE0DFF1D7EAD6FAD219614
:107A20009FAD219722968FAD2297272F362F492F72
:107A3000582F60817181828193810E94D06D162FB1
:107A4000072F382E292E7F89688D998D8DA1272F9C
:107A5000362F492F582FC501B4010E947F716B0149
:107A60007C01B801C101272F362F492F582FC301A0
:107A7000B2010E947F719B01AC01C701B6010E9457
:107A8000D16D6B017C01B801C101272F362F492F21
:107A9000582FC501B4010E947F716EA77FA788ABE4
:107AA00099AB7F89688D998D8DA1272F362F492F0E
:107AB000582FC301B2010E947F719B01AC016EA5DA
:107AC0007FA588A999A90E94D06DA70196010E945F
:107AD000446E362E272E182F092F20E030E0A90102
:107AE000D101F8016B2F7A2F8F2F9E2F0E94AA6E43
:107AF00087FF10C02BED3FE049EC50E4D101F801C5
:107B00006B2F7A2F8F2F9E2F0E94D16D362E272E0E
:107B1000182F092FA4968FADA497882381F02BED01
:107B20003FE049EC50E4D101F8016B2F722D8F2F0B
:107B3000902F0E94D06D362E272E182F092FC9881E
:107B4000DA88EB88FC88E894F7F8A3962CAD3DAD75
:107B50004EAD5FADA397D101F8016B2F722D8F2F22
:107B6000902F0E947F71A70196010E94BA706B014D
:107B70007C012FE632E143E85AE30E94AA6E87FDBA
:107B800016C2C701B6010E94876F0E941E6F7A8FCE
:107B9000698FFB01EF2B21F421E030E03A8F298F30
:107BA000498D5A8DBA0180E090E00E944A6F6B01C6
:107BB0007C019B01AC01D101F8016B2F722D8F2F3D
:107BC000902F0E94B16E6F8B788F1C01A7019601D8
:107BD00069897A898B899C890E94B16E24966FAFDE
:107BE000249725967FAF259726968FAF26972796C1
:107BF0009FAF27972F8D38A149A15AA16AA57BA5D0
:107C00008CA59DA50E94D06DA70196010E94B16E22
:107C100028966FAF289729967FAF29972A968FAF1E
:107C20002A972B969FAF2B9720E030E040E05FE350
:107C3000BF89A88D6B2F7A2F822D932D0E947F7183
:107C4000BF89A88D2B2F3A2F422D532D0E947F7173
:107C50009B01AC0160E070E080E89FE30E94D06D82
:107C60006DA37AA78EA723969FAF2397CE01019687
:107C7000FC01A8A554E0A59FE00DF11D11242B8D5A
:107C80003C8D4D8D5E8D20833183428353832F8DB8
:107C900038A149A15AA12D873E874F87588B198A51
:107CA00041E050E05C8F4B8F81E090E08C0F9D1F96
:107CB000BBA1A4E0BA9F800D911D112499A788A7AC
:107CC00021E030E02C0F3D1F5EA144E0549F200DC9
:107CD000311D11243FA32EA3FCA3EBA347C1898927
:107CE00089310CF050C07F89688D272F362F422DA7
:107CF000532DC501B4010E947F716B017C017DA1F0
:107D00006AA59EA523968FAD2397272F362F492F3F
:107D1000582FC301B2010E947F719B01AC01C701C2
:107D2000B6010E94D16D7B018C017DA16AA59EA543
:107D300023968FAD2397272F362F492F582FC50114
:107D4000B4010E947F715B016C017F89688D272FD0
:107D5000362F422D532DC301B2010E947F719B012A
:107D6000AC016A2D7B2D8C2D9D2D0E94D06D862E11
:107D7000972EA82EB92E99899F5F998B4E2C5F2C38
:107D8000602E712E72C0AB8DBC8DBD0180E090E085
:107D90000E944A6FBF89A88D2B2F3A2F422D532D59
:107DA0000E947F717B018C017F2D802F912F0E947B
:107DB000AE6E2B013C016E2D7F2D802F912F0E94E6
:107DC000E271698B7A8B8B8B9C8BEAA9FBA98081F2
:107DD0009181A281B3819C01AD0150582F8F38A3AE
:107DE00049A35AA3ACA9BDA9CD90DD90ED90FC901C
:107DF000A30192016F8D78A189A19AA10E947F7140
:107E00004B015C0129893A894B895C89C701B6011C
:107E10000E947F719B01AC01C501B4010E94D16D2C
:107E2000862E972EA82EB92E29893A894B895C89EE
:107E30006F8D78A189A19AA10E947F71698B7A8B3D
:107E40008B8B9C8BA3019201C701B6010E947F71AD
:107E50009B01AC0169897A898B899C890E94D06DCC
:107E6000462E572E682E792E198AA5019401BAAD97
:107E7000ABADFCADEDAD6B2F7A2F8F2F9E2F0E94F7
:107E8000D16DE8A5F9A56083718382839383A301F3
:107E90009201BEADAFAD2196FFAD21972296EFAD19
:107EA00022976B2F7A2F8F2F9E2F0E94D16DAEA11C
:107EB000BFA16D937D938D939C93139724967FAD73
:107EC000249725966FAD259726969FAD26972796E2
:107ED0008FAD2797272F362F492F582FEBA1FCA1C5
:107EE00060817181828193810E94D16DABA1BCA11F
:107EF0006D937D938D939C93139728967FAD2897D0
:107F000029966FAD29972A969FAD2A972B968FAD0C
:107F10002B97272F362F492F582F6D857E858F85DC
:107F200098890E94D16D6D877E878F87988BCE014F
:107F300001960E94151494E6C92ED12CCC0EDD1E9C
:107F4000EEA8FFA808AD19AD9E01235F3F4FAE011B
:107F5000475F5F4FBE016B5F7F4FCE0101960E946E
:107F60009045EB8DFC8D3196FC8FEB8F2B8D3C8DEE
:107F7000498D5A8D2417350708F4B1CE2D893E89D5
:107F8000245F3F4F4D895E89485F5F4F6D897E89D1
:107F90006C5F7F4F84E6C82ED12CCC0EDD1EEEA880
:107FA000FFA808AD19AD8D899E890E949045C65BDA
:107FB000DF4F0FB6F894DEBF0FBECDBFDF91CF917C
:107FC0001F910F91FF90EF90DF90CF90BF90AF90F7
:107FD0009F908F907F906F905F904F903F902F90E9
:107FE00008952F923F924F925F926F927F928F925D
:107FF0009F92AF92BF92CF92DF92EF92FF920F9338
:108000001F93CF93DF93CDB7DEB768970FB6F89481
:10801000DEBF0FBECDBF1C014A015B0168017901C3
:10802000DC01D8966D917D918D919C91DB970E949A
:108030004A6F69837A838B839C83A50194010E9494
:108040007F710E94976E0E941E6F6D837E838F8367
:108050009887A701960169817A818B819C810E9412
:108060007F710E94976E0E941E6F69877A878B8747
:108070009C872D813E814F815885283731054105E8
:10808000510540F488E790E0A0E0B0E08D839E8346
:10809000AF83B88729853A854B855C8528373105BC
:1080A0004105510540F488E790E0A0E0B0E0898701
:1080B0009A87AB87BC87F101EC5BFF4F4080518012
:1080C00062807380C301B2010E944C6F6B017C011E
:1080D000D101DC966D917D918D919C91DF970E94ED
:1080E0004A6F6D877E878F87988B20E030E0A901EB
:1080F000C701B6010E94AA6E882339F129813A810D
:108100004B815C81CA01B9010E947F714B015C0106
:108110002D853E854F855889CA01B9010E947F711E
:108120009B01AC01C501B4010E94D06D4B015C0103
:10813000A7019601C701B6010E94D16D9B01AC0158
:10814000C501B4010E94B16E04C060E070E080E03F
:1081500090E00E94976E0E94196F4B015C016627A8
:108160007727CB0164197509860997090E944C6F1E
:108170002B013C01F101E05CFF4F60817181828144
:1081800093810E944A6F698B7A8B8B8B9C8B20E04A
:1081900030E0A901C301B2010E94AA6E882379F1DF
:1081A00029893A894B895C89CA01B9010E947F718A
:1081B0006D8B7E8B8F8B988F29813A814B815C816F
:1081C000CA01B9010E947F719B01AC016D897E8952
:1081D0008F89988D0E94D06D69837A838B839C836D
:1081E000A3019201C301B2010E94D16D9B01AC01B8
:1081F00069817A818B819C810E94B16E04C060E0AC
:1082000070E080E090E00E94876FD10150962D9140
:108210003D914D915C91539729833A834B835C83C5
:1082200029013A01481859086A087B080E94196F09
:10823000461A570A680A790A77FE6CC020E030E0D7
:10824000A901C701B6010E94AA6E882309F445C09E
:10825000A7019601C701B6010E94D16D2B013C0117
:1082600069817A818B819C810E944A6F9B01AC015C
:10827000C301B2010E947F712B013C012D853E8517
:108280004F855889CA01B9010E947F719B01AC01D9
:10829000C301B2010E94D06D2B013C0129893A89AA
:1082A0004B895C89CA01B9010E947F719B01AC01B5
:1082B000C301B2010E94D16D4B015C0120E030E0AE
:1082C00040E850E4C701B6010E947F719B01AC01F8
:1082D000C501B4010E94B16E04C060E070E080E0AE
:1082E00090E00E94976E0E94196F4B015C01B7FEEF
:1082F00003C0812C912C540129813A814B815C81EE
:1083000082169306A406B50610F049015A01412CC5
:10831000512C32018FB7F894F101E45BFF4F90814B
:10832000911125C0D10154968D929D92AD92BC922F
:108330005797480C591C6A1C7B1CF101408E518ECA
:10834000628E738E2D813E814F815885DC962D93F0
:108350003D934D935C93DF97A05CBF4F29853A8591
:108360004B855C852D933D934D935C9313978FBF05
:1083700068960FB6F894DEBF0FBECDBFDF91CF91E8
:108380001F910F91FF90EF90DF90CF90BF90AF9033
:108390009F908F907F906F905F904F903F902F9025
:1083A0000895AF92BF92CF92DF92EF92FF920F9318
:1083B0001F93CF93DF935B017A016115710509F477
:1083C00075C04115510509F471C0FB0102A513A543
:1083D000D4A5C5A5CE01202F312F492F582F66A136
:1083E00077A180A591A50E94AA6E882309F45EC09A
:1083F000F50187A981114BC0F701C6A0D7A0E0A461
:10840000F1A4A7019601DE01602F712F8B2F9A2F07
:108410000E94AD701816DCF5A7019601C701B601E0
:108420000E947F716B017C01F50182A993A9A4A927
:10843000B5A9BC01CD0190589B01AC010E94D16D42
:10844000F50126A537A540A951A90E947F719B017E
:10845000AC01C701B6010E94D06D0E94EC716B01A6
:108460007C01762F272F3D2D4E2D5F2DFE01602F95
:10847000712F8F2F9E2F0E94AA6E87FF03C0680165
:10848000ED2EFC2E5C2D4D2D3E2D2F2D03C0502F9B
:10849000412F9E01852F942FA32FB22FF50186A384
:1084A00097A3A0A7B1A781E0F50186ABDF91CF919B
:1084B0001F910F91FF90EF90DF90CF90BF90AF9002
:1084C0000895CF92DF92EF92FF920F931F93CF9375
:1084D000DF931F92CDB7DEB7809155088FB7F89420
:1084E000F09054088FBF8091550890E08F19910942
:1084F0008F709927049704F12091550823502F700D
:1085000040E050E000E010E08DE4E82E13C02111BF
:1085100001C020E12150E29E6001112486E598E02F
:10852000C80ED91EB801C60129830E94D141A801F5
:10853000860129812F11EBCF0F90DF91CF911F91F1
:108540000F91FF90EF90DF90CF9008952F923F9280
:108550004F925F926F927F928F929F92AF92BF9253
:10856000CF92DF92EF92FF920F931F93CF93DF93FF
:10857000EC011B01009709F464C08FA9811161C04F
:108580008EA09FA0A8A4B9A4FB01C6A0D7A0E0A478
:10859000F1A42C2D3D2D4E2D5F2DC501B4010E945F
:1085A000AA6E87FF4EC0A5019401C501B4010E94C7
:1085B0007F712B013C018AA89BA8ACA8BDA8C5016E
:1085C000B40190589B01AC010E94D16D2EA53FA52E
:1085D00048A959A90E947F719B01AC01C301B20156
:1085E0000E94D06D0E94EC718B01D82FC92F762F7D
:1085F000CE01272F312F492F582F6C2D7D2D8E2DF9
:108600009F2D0E94AA6E87FF03C08601DE2DCF2D0D
:10861000CE01202F312F492F5C2F6C2D7D2D8E2DDB
:108620009F2D0E94AA6E882361F09E01802F912FBA
:10863000A32FBC2FF10186A397A3A0A7B1A781E028
:1086400086ABDF91CF911F910F91FF90EF90DF905C
:10865000CF90BF90AF909F908F907F906F905F90E2
:108660004F903F902F900895EF92FF920F931F939A
:10867000CF93DF93F0905408C0E0D0E080E090E02A
:108680002DE4E22E11C0EF9C800111240A5A174FED
:10869000A801BE010E94A6428F2D8F5F803109F490
:1086A00080E0F82ECE01E80120915508F212EBCFC0
:1086B00040E050E0BE01DF91CF911F910F91FF90FC
:1086C000EF900C94A6424F925F926F927F928F929E
:1086D0009F92AF92BF92CF92DF92EF92FF920F9351
:1086E0001F93CF93DF9350905408C0E0D0E03DE457
:1086F000432E37C0489E3001499E700C112486E5F8
:1087000098E0680E791E209731F18EA9811104C07E
:10871000F30186A98823F9F0CAA0DBA0ECA0FDA094
:10872000A7019601F30166A177A180A591A50E94FA
:10873000B16E4B015C01A70196016EA17FA188A5D6
:1087400099A50E94B16EAB01BC0195018401CE01D7
:108750000E94F13F1EAA5394F0E15F1201C0512C18
:10876000E301852D992787FD90952091550830E0EC
:108770008217930709F0BECF2097F1F0CAA0DBA0C3
:10878000ECA0FDA0A70196016DEC7CEC8CE49DE3D0
:108790000E94B16E4B015C01A70196016EA17FA101
:1087A00088A599A50E94B16EAB01BC019501840119
:1087B000CE010E94F13F1EAADF91CF911F910F9130
:1087C000FF90EF90DF90CF90BF90AF909F908F90F1
:1087D0007F906F905F904F9008950E9461420E9439
:1087E00034430C946343109255081092540880E16E
:1087F000E7E2FDE0DF011D928A95E9F71092970DFF
:108800001092980D1092990D10929A0D10929B0D46
:1088100010929C0D10929D0D10929E0D10929F0D26
:108820001092A00D1092A10D1092A20D1092A30D06
:108830001092A40D1092A50D1092A60D1092A70DE6
:108840001092A80D1092A90D1092AA0D08954F92A2
:108850005F926F927F928F929F92AF92BF92CF92D0
:10886000DF92EF92FF920F931F93CF93DF9380914C
:10887000260D882309F41FC160E08091000E9091BD
:10888000010E0E9459590091390110913A01D0917D
:108890003B01C0913C0120E030E040E050E40E9408
:1088A000D16DFE01202F312F4F2F5E2F0E94AA6E17
:1088B00087FD01C1F0905408B12CC12CD12CE12CC2
:1088C0004DE4A42E5CC02F2D30E0A29EF001A39EAB
:1088D000F00D1124EA5AF74F80819181A281B38172
:1088E000892B8A2B8B2B81F484819581A681B7817A
:1088F000892B8A2B8B2B41F480859185A285B385AA
:10890000892B8A2B8B2BC1F1A29E4001A39E900C38
:10891000112486E598E0880E991EF401648575851A
:10892000868597850E944C6F2B013C01F40160897C
:108930007189828993890E944A6F9B01AC01C301AE
:10894000B2010E94B16EF40122A133A144A155A14C
:108950000E947F713B014C012B2D3C2D4D2D5E2D36
:10896000662D772D882D992D0E94AD70181624F450
:10897000B62CC72CD82CE92CF394FFE0FF22809171
:108980005508F812A0CF2091350130913601409161
:108990003701509138016B2D7C2D8D2D9E2D0E941D
:1089A0007F719B01AC01FE01602F712F8F2F9C2FD7
:1089B0000E94D16D6B017C01CE01202F312F492FF8
:1089C0005C2F6C2D7D2D8E2D9F2D0E94AA6E87FD14
:1089D00003C08601DE2DCF2DC0903D01D0903E0119
:1089E000E0903F01F09040012C2D3D2D4E2D5F2D4C
:1089F000FE01602F712F8F2F9C2F0E94AD701816D3
:108A00001CF06801ED2EFC2E8090AB0D9090AC0D0B
:108A1000A090AD0DB090AE0D2C2D3D2D4E2D5F2DA7
:108A2000C501B4010E94AD701816F4F420E037EDD2
:108A300043EA5CE36C2D7D2D8E2D9F2D0E947F716E
:108A40008B01D82FC92F28E431EE4AE75FE3C50137
:108A5000B4010E947F71FE01202F312F4F2F5E2F16
:108A60000E94D16D6B017C018C2D9D2DAE2DBF2DF3
:108A70008093AB0D9093AC0DA093AD0DB093AE0D64
:108A80006C2D7D2D8E2D9F2D0E94196FDC01CB0149
:108A900060E00E9489589093010E8093000E8C2D07
:108AA0009D2DAE2DBF2D8093F60D9093F70DA093C5
:108AB000F80DB093F90DDF91CF911F910F91FF90B9
:108AC000EF90DF90CF90BF90AF909F908F907F906E
:108AD0006F905F904F900895909154088091550841
:108AE0009817D9F02091540830E04DE410C0429F0F
:108AF000F0011124EA5AF74F80859185A285B3854C
:108B0000892B8A2B8B2B09F03F5F2F5F2F70809171
:108B100055082813ECCF311101C0159A0C94274445
:108B20002F923F924F925F926F927F928F929F927D
:108B3000AF92BF92CF92DF92EF92FF920F931F936B
:108B4000CF93DF93CDB7DEB7C357D1090FB6F894F3
:108B5000DEBF0FBECDBF2C013B014A0159013E2CA7
:108B6000F9AA0AAB212EDDAACCAA209155082F5FC5
:108B700063962FAF6397203119F463961FAE639706
:108B800063963FAD6397032F112707FD109505C02E
:108B90000E94255A81E00E9437168091540890E087
:108BA00080179107A9F32091730D3091740D4091B6
:108BB000750D5091760DD2016D917D918D919C91A5
:108BC0000E947F710E944F7123966FAF2397249666
:108BD0007FAF249725968FAF259726969FAF269730
:108BE0002091770D3091780D4091790D50917A0D4B
:108BF000F30160817181828193810E947F710E9463
:108C00004F7127966FAF279728967FAF28972996A1
:108C10008FAF29972A969FAF2A9720917B0D30918D
:108C20007C0D40917D0D50917E0DD4016D917D9113
:108C30008D919C910E947F710E944F712B966FAF16
:108C40002B972C967FAF2C972D968FAF2D972E9626
:108C50009FAF2E9720917F0D3091800D4091810D17
:108C60005091820DF50160817181828193810E9412
:108C70007F710E944F716AAF7BAF8CAF9DAF8091C7
:108C8000330D9091340DA091350DB091360D2AAD74
:108C90003BAD4CAD5DAD281739074A075B07C1F105
:108CA0006091E802E62FF0E0EE0FFF1FE450F24F74
:108CB000808191810E94595920E030E04AE253E4DA
:108CC0000E94AA6E87FF24C080915308811120C0A2
:108CD0000C94F54F9091C00095FFFCCF8093C60097
:108CE000319684918111F6CFE2EDF6E007C09091C4
:108CF000C00095FFFCCF8093C6003196849181110E
:108D0000F6CF8091C00085FFFCCF8AE08093C6003B
:108D10008091330D9091340DA091350DB091360DA9
:108D20002AAD3BAD4CAD5DAD281B390B4A0B5B0B3F
:108D3000CA01B90157FF07C090958095709561955C
:108D40007F4F8F4F9F4F0E944C6F4B015C0120E083
:108D500030E848E953E460917F0D7091800D809177
:108D6000810D9091820D0E947F719B01AC01C50124
:108D7000B4010E94AD7018166CF58AAD9BADACAD18
:108D8000BDAD8093330D9093340DA093350DB0930A
:108D9000360DECECF6E007C09091C00095FFFCCFDB
:108DA0008093C600319684918111F6CFECEEF6E007
:108DB00007C09091C00095FFFCCF8093C60031960C
:108DC00084918111F6CF8091C00085FFFCCF8AE0AD
:108DD0008093C60080915508EDE48E9FD001112448
:108DE000AA5AB74FBCA3ABA3FD01E45BFF4F1082AF
:108DF0002091270D3091280D4091290D50912A0D79
:108E00002DA33EA34FA358A726964CAC5DAC6EACE9
:108E10007FAC2697421A530A640A750A77FE08C087
:108E20007094609450944094411C511C611C711CBE
:108E3000ABA1BCA14D925D926D927C921397209153
:108E40002B0D30912C0D40912D0D50912E0D29A7F9
:108E50003AA74BA75CA72A968CAC9DACAEACBFAC36
:108E60002A97821A930AA40AB50AB7FE08C0B094DA
:108E7000A09490948094811C911CA11CB11CABA166
:108E8000BCA114968D929D92AD92BC9217972091A1
:108E90002F0D3091300D4091310D5091320D2DA795
:108EA0003EA74FA758AB2E964CAD5DAD6EAD7FADD6
:108EB0002E978DA59EA5AFA5B8A9481B590B6A0B87
:108EC0007B0B77FF07C070956095509541955F4F7C
:108ED0006F4F7F4F142F052F6EAB78AFABA1BCA1A6
:108EE00018964C93189719965C9319971A966C9349
:108EF0001A971B967C93C090330DD090340DE09060
:108F0000350DF090360DA0911801B09119012AADE0
:108F10003BAD4CAD5DAD2C193D094E095F0957FFC6
:108F200007C050954095309521953F4F4F4F5F4F6B
:108F30000E94507224E630E040E050E00E949E72B1
:108F4000EBA1FCA12487358746875787812F902F77
:108F5000AEA9B8AD88159905AA05BB0514F4D501CD
:108F6000C40182179307A407B50714F4DA01C901F5
:108F700093018201481659066A067B0614F48C0197
:108F80009D01ABA1BCA150960D931D932D933C93D5
:108F90005397063011052105310510F40C94055046
:108FA000FD01E85BFF4F8091E70290E0A0E0B0E0B8
:108FB00080839183A283B38326962CAD3DAD4EADC5
:108FC0005FAD26978DA19EA1AFA1B8A5281739073F
:108FD0004A075B072CF0ABA1BCA190961C9204C081
:108FE00081E0EBA1FCA180A32A962CAD3DAD4EAD56
:108FF0005FAD2A9789A59AA5ABA5BCA52817390707
:109000004A075B0744F4ABA1BCA190968C91909762
:10901000826090968C932E962CAD3DAD4EAD5FAD9B
:109020002E978DA59EA5AFA5B8A9281739074A0781
:109030005B0744F4ABA1BCA190968C91909784609F
:1090400090968C932AAD3BAD4CAD5DAD2C153D0596
:109050004E055F0544F4ABA1BCA190968C9190970E
:10906000886090968C93ECA9FDA98081ABA1BCA1EE
:1090700091968C9345284628472809F05E98EBA1E5
:10908000FCA184819581A681B781892B8A2B8B2BAA
:1090900009F05E98EBA1FCA180859185A285B3853E
:1090A000892B8A2B8B2B09F01598EBA1FCA18485C9
:1090B0009585A685B785892B8A2B8B2B09F05E9821
:1090C000ABA1BCA11C962D913D914D915C911F9738
:1090D00022962CAF3DAF4EAF5FAF2297232B242BB0
:1090E000252BD9F44090470D5090480D6090490DC4
:1090F00070904A0D242D352D462D572DA9A9FAA97A
:10910000632D7A2F8F2F922D0E94AA6E87FD0EC09D
:10911000432C59A86AA8722C09C040905F0D50904A
:10912000600D6090610D7090620DE4CF26966CAD7D
:109130007DAD8EAD9FAD26972DA13EA14FA158A527
:10914000621B730B840B950B0E944C6F2091730D67
:109150003091740D4091750D5091760D0E94B16E55
:109160006DA379AB8AAB9CAB362F272F982F8CA998
:10917000432F522F692F782F498B5A8B6B8B7C8B07
:109180002A966CAD7DAD8EAD9FAD2A9729A53AA5E7
:109190004BA55CA5621B730B840B950B0E944C6F57
:1091A0002091770D3091780D4091790D50917A0D85
:1091B0000E94B16E162F072F89A79EAB9801982F9A
:1091C0008EA9432F522F692F782F4D8B5E8B6F8B7B
:1091D000788F2E966CAD7DAD8EAD9FAD2E972DA563
:1091E0003EA54FA558A9621B730B840B950B0E94DB
:1091F0004C6F20917B0D30917C0D40917D0D5091F5
:109200007E0D0E94B16E6DA778AF382E292E362FB5
:10921000272FC101432F522F692F782F498F5A8F43
:109220006B8F7C8FA0901801B09019016AAD7BAD57
:109230008CAD9DAD6C197D098E099F090E944C6F04
:1092400020917F0D3091800D4091810D5091820DC4
:109250000E94B16E6B017C01B501882777FD809576
:10926000982F0E944C6F9B01AC01C701B6010E9470
:109270007F7120E030E048EC52E40E94B16E462F4E
:10928000572F682F792FDB01CA014D8F5E8F6F8FAB
:1092900078A3EBA1FCA180809180A280B380F6E04E
:1092A0008F169104A104B104E4F4EBA1FCA1448164
:1092B00055816681778146305105610571058CF4D1
:1092C000408551856285738546305105610571057C
:1092D00044F4AC01BD017F7746A757A760AB71ABE3
:1092E0003AC05DA149A93AA92CA9652F742F832FF3
:1092F000922F0E942A726B017C01A80139A52EA928
:10930000652F702F832F922F0E942A729B01AC0130
:10931000C701B6010E94D16D162F072FF82EE92E36
:109320005DA548AD9101652F742F832F922D0E946A
:109330002A729B01AC01D801F7016B2F7A2F8F2F76
:109340009E2F0E94D16D0E94EC71EBA1FCA166A73B
:1093500077A780AB91ABABA1BCA19E962D913D911F
:109360004D915C91D197AA962CAF3DAF4EAF5FAFB8
:10937000AA9760E070E080E89FE30E94B16E9B01D5
:10938000AC01642D752D862D972D0E947F7169A7E4
:109390007DA789AB9CAB9091550880915408E92F2B
:1093A000F0E0E81BF109EF70FF27FBABEAAB762F8B
:1093B0006DA599A98CA9272F362F492F582F60E02A
:1093C00074E284E799E40E94B16E0E944F711B0120
:1093D0008C012AA93BA9223031050CF44AC069014D
:1093E000EE24D7FCE094FE2CC701B6010E944C6F1E
:1093F00020E030E040E051E40E94AA6E87FF39C0CF
:10940000210138018091930D9091940DA091950DBB
:10941000B091960D481659066A067B0650F5BC01B8
:10942000CD016419750986099709660F771F881F92
:10943000991FA70196010E947C72CA01B9010E947E
:109440004A6F0E944F71AB01BC01CB01BA01640DA0
:10945000751D861D971D0E944A6F9B01AC0160E03F
:1094600074E284E799E40E94B16E69A77DA789AB95
:109470009CAB79A56DA599A98CA9272F362F492FCB
:10948000582FAA966CAD7DAD8EAD9FADAA970E9468
:109490007F716E966FAF6E97A2967FAFA2972F9651
:1094A0008FAF2F97A6969FAFA697362F272F982F6F
:1094B000A6968FADA697432F522F692F782FABA179
:1094C000BCA192964D935D936D937C939597509626
:1094D0006D917D918D919C9153970E944A6F6B0184
:1094E0007C0179A56DA599A98CA9272F362F492F25
:1094F000582FC701B6010E947F710E94976E0E948B
:109500001E6F67966CAF7DAF8EAF9FAF6797EBA175
:10951000FCA160AF71AF82AF93AF9E012F5E3F4F52
:109520003FAB2EABAE014F5F5F4F5EA34DA383E811
:109530009DE06D969FAF8EAF6D97DE019196BAA3B9
:10954000A9A359AF48AF212C312C00E81FE3EEA9A5
:10955000FFA96191719181919191FFABEEABB9A59A
:10956000ADA5F9A9ECA92B2F3A2F4F2F5E2F0E9402
:109570007F71AB01BC01A8ADB9AD4D935D936D9307
:109580007D93B9AFA8AFDB01CA01BF776B968CAFF3
:109590009DAFAEAFBFAF6B976D96AEADBFAD6D97E4
:1095A0004D905D906D907D906D96BFAFAEAF6D9715
:1095B000A30192016B966CAD7DAD8EAD9FAD6B97A7
:1095C0000E94AD701816F4F46B962CAD3DAD4EAD07
:1095D0005FAD6B97C301B2010E94B16E2B01782E73
:1095E000692E762FC301272F352D492F582F622D35
:1095F000732D802F912F0E94AA6E87FD03C0120148
:10960000072D162DEEA9FFA929A13AA1E217F3070C
:1096100009F09DCF20E030E040E85FE3622D732D3C
:10962000802F912F0E94AA6E87FF4FC03E0131E12B
:10963000630E711C222D332D402F512FADA1BEA1E1
:109640006D917D918D919C910E947F71EDA1FEA104
:109650006193719381939193FEA3EDA3E615F705B2
:1096600049F7222D332D402F512F6E96BFAD6E97A7
:10967000A296AFADA2972F96FFAD2F97A696EFAD0E
:10968000A6976B2F7A2F8F2F9E2F0E947F71ABA1F1
:10969000BCA192966D937D938D939C9395976796BD
:1096A0006CAD7DAD8EAD9FAD67970E944A6F222D48
:1096B000332D402F512F0E947F710E941E6FEBA10E
:1096C000FCA160AF71AF82AF93AFAA962CAD3DAD58
:1096D0004EAD5FADAA97C701B6010E94B16E162FBD
:1096E000072F382E292E81149104A104B10491F57D
:1096F000EBA1FCA184819581A681B781892B8A2B5E
:109700008B2B41F580859185A285B385892B8A2B8A
:109710008B2B01F52091570D3091580D4091590D2B
:1097200050915A0DD801F1016B2F7A2F8F2F9E2F58
:109730000E947F710E94976EEBA0FCA0F4E4EF0EF4
:10974000F11C0E941E6FD7016D937D938D939C93A6
:10975000139700C120915B0D30915C0D40915D0D20
:1097600050915E0DD801F1016B2F702F8F2F922D2C
:109770000E947F710E94976E0E941E6FEBA1FCA158
:10978000EC5BFF4FFEA3EDA3608371838283938321
:109790004090370D5090380D6090390D70903A0D13
:1097A0000E944A6F69A77AA78BA79CA7C501B4013D
:1097B0000E944C6F9B01AC0169A57AA58BA59CA565
:1097C0000E947F71A70196010E94B16E4B015C015E
:1097D000C301B2010E944A6F9B01AC01C501B401F3
:1097E0000E94AD70181634F4EDA1FEA140825182A2
:1097F0006282738240903B0D50903C0D60903D0D15
:1098000070903E0DADA1BEA16D917D918D919C9109
:109810000E944A6F4B015C01EBA1FCA16481758140
:10982000868197810E944C6F9B01AC01C501B401F8
:109830000E947F71A70196010E94B16E4B015C01ED
:10984000C301B2010E944A6F9B01AC01C501B40182
:109850000E94AD7018163CF4ADA1BEA14D925D9270
:109860006D927C9213974090430D5090440D609000
:10987000450D7090460DEBA1FCA1EC5BFF4FFEA3E4
:10988000EDA360817181828193810E944A6F4B01B7
:109890005C0122966CAD7DAD8EAD9FAD22970E948E
:1098A0004C6F9B01AC01C501B4010E947F71A701FF
:1098B00096010E94B16E4B015C01C301B2010E948E
:1098C0004A6F9B01AC01C501B4010E94AD7018162E
:1098D0003CF4ADA1BEA14D925D926D927C92139726
:1098E00040903F0D5090400D6090410D7090420DA2
:1098F000EDA1FEA160817181828193810E944A6FF6
:109900004B015C01ABA1BCA118966D917D918D912D
:109910009C911B970E944C6F9B01AC01C501B40147
:109920000E947F71A70196010E94B16E6B017C01BC
:10993000C301B2010E944A6F9B01AC01C701B6018D
:109940000E94AD70181634F4EDA1FEA14082518240
:1099500062827382EBA1FCA1EC5BFF4F608171819D
:10996000828193810E944A6F6B017C01B801C10121
:10997000272F302F492F522DC701B6010E94B16EFB
:10998000462F572F682F792FE0964CAF5DAF6EAF03
:109990007FAFE097ABA1BCA1D2964D935D936D9341
:1099A0007C93D5972DEB37E346E051E4C701B60130
:1099B0000E947F710E94196FEBA1FCA1648F758FCB
:1099C000868F978F4090530D5090540D6090550D99
:1099D0007090560D20E030E040E05FE3C301B2013B
:1099E0000E947F716DA379A78DA799AB29853A85D0
:1099F0004B855C85A1962CAF3DAF4EAF5FAFA19775
:109A000080904F0D9090500DA090510DB090520D40
:109A100020E030E040E05FE3C501B4010E947F71C7
:109A2000162F072FF82EE92EA1966CAD7DAD8EADC9
:109A30009FADA1979F77D801F7012B2F3A2F4F2F7A
:109A40005E2F0E94AD701816B4F4B801C701272F1D
:109A5000362F492F582FBDA1A9A5FDA5E9A96B2F28
:109A60007A2F8F2F9E2F0E94AA6E87FD04C01DA300
:109A700009A7FDA6E9AA8D859E85AF85B889A5961B
:109A80008CAF9DAFAEAFBFAFA597C0904B0DD09040
:109A90004C0DE0904D0DF0904E0D20E030E040E098
:109AA0005FE3C701B6010E947F71162F072F382E82
:109AB000292EA5966CAD7DAD8EAD9FADA5979F77F8
:109AC000D801F1012B2F3A2F4F2F5E2F0E94AD703E
:109AD0001816B4F4B801C101272F362F492F582F7B
:109AE000BDA1A9A5FDA5E9A96B2F7A2F8F2F9E2FC8
:109AF0000E94AA6E87FD04C01DA309A73DA629AA3E
:109B0000ABA1BCA19296BC91BCABEBA1FCA1F3A113
:109B1000FEABABA1BCA19496BC91B8AFEBA1FCA1EC
:109B2000F5A1FEAF7CA96EA9272F362F4B2F5F2FF3
:109B3000BDA1A9A5FDA5E9A96B2F7A2F8F2F9E2F77
:109B40000E94AA6E87FD08C02CA92DA33EA939A7A3
:109B500048AD4DA75EAD59AB8AA99BA902970CF4FD
:109B600043C19091A70D9AABA091A80D6496AFAF99
:109B70006497B091A90D6896BFAF6897E091AA0D60
:109B80006C96EFAF6C9727E137EB41ED58E36896A1
:109B9000FFAD6897692F7A2F8F2F9E2F0E94AD708F
:109BA00018160CF021C12091970D3091980D40911D
:109BB000990D50919A0D69817A818B819C810E94C7
:109BC000D06D162F072F382E292E20919B0D309106
:109BD0009C0D40919D0D50919E0D6D817E818F81D8
:109BE00098850E94D06D2F966FAF2F97A6967FAF66
:109BF000A697AB968FAFAB97AC969FAFAC97B801DB
:109C0000C101272F362F492F582FD801F1016B2F73
:109C10007A2F8F2F9E2F0E947F71E4966CAF7DAFBD
:109C20008EAF9FAFE4972F967FAD2F97A6966FAD1F
:109C3000A697AB969FADAB97AC968FADAC97272F01
:109C4000362F492F582FDB01FC016B2F7A2F8F2FD6
:109C50009E2F0E947F719B01AC01E4966CAD7DAD9F
:109C60008EAD9FADE4970E94D16D0E94EC7162961B
:109C70006CAF7DAF8EAF9FAF6297A30192010E9440
:109C8000AD7018166CF462962CAD3DAD4EAD5FAD67
:109C90006297C301B2010E94B16E8B011C0106C024
:109CA00000E010E050E8252E6FE3362E20919F0D46
:109CB0003091A00D4091A10D5091A20DA1966CADD7
:109CC0007DAD8EAD9FADA1970E94D06D2B013C0163
:109CD000E89477F8A5019401C301B2010E94AD7028
:109CE0001816D4F4A3019201C501B4010E94B16E0B
:109CF0004B01B82EA92E762FC501272F392D492FBC
:109D0000582F602F712F822D932D0E94AA6E87FDF0
:109D100003C084012B2C3A2C2091A30D3091A40D6B
:109D20004091A50D5091A60DA5966CAD7DAD8EAD63
:109D30009FADA5970E94D06D4B015C01E894B7F8E8
:109D4000A7019601C501B4010E94AD701816D4F4A4
:109D5000A5019401C701B6010E94B16E6B01F82EF6
:109D6000E92E762FC701272F3D2D492F582F602F21
:109D7000712F822D932D0E94AA6E87FD03C086014C
:109D80002F2C3E2C202F312F422D532DBCA9AEA9B4
:109D9000F8ADEEAD6B2F7A2F8F2F9E2F0E947F7123
:109DA0004B015C01762F272F392D4A2D5B2DBAA947
:109DB0006496AFAD64976896FFAD68976C96EFAD0B
:109DC0006C976B2F7A2F8F2F9E2F0E94AA6E87FF82
:109DD0000FC08AA864969FAC64976896AFAC6897EA
:109DE0006C96BFAC6C9704C08DA099A4ADA4B9A823
:109DF000482D592D6A2D7B2DABA1BCA19A964D9370
:109E00005D936D937C939D97E0966CAD7DAD8EAD2B
:109E10009FADE09790589B01AC010E94D16DAA962E
:109E20002CAD3DAD4EAD5FADAA970E947F719B01F9
:109E3000AC016BE077ED83E29BE30E94D06D0E9462
:109E4000EC718B01F82EE92E762FC701272F312FC9
:109E5000492F582F682D792D8A2D9B2D0E94AA6E8F
:109E600087FD03C04801AF2CBE2C482D592D6A2D0B
:109E70007B2DEBA1FCA146A357A360A771A7C70147
:109E8000202F312F492F5E2DBCA9AEA9F8ADEEAD24
:109E90006B2F7A2F8F2F9E2F0E94AA6E181634F0E8
:109EA00081E0ABA1BCA1D7968C9303C0EBA1FCA130
:109EB00017AA81E0ABA1BCA1D6968C9380E1FE01EC
:109EC0003196A7E9BDE001900D928A95E1F73CA992
:109ED0002EA998AD8EAD432F522F692F782F409326
:109EE000A70D5093A80D6093A90D7093AA0D232F71
:109EF000352F492F582FBDA1A9A5FDA5E9A96B2F85
:109F00007A2F8F2F9E2F0E94B16E6B017C017CA94E
:109F10006EA998AD8EAD272F362F492F582F682D5B
:109F2000792D8A2D9B2D0E94B16EAB01BC0197014A
:109F300086018BA19CA10E94F13F6396BFAD639700
:109F4000B093550826962CAD3DAD4EAD5FAD26972E
:109F50002093270D3093280D4093290D50932A0DFF
:109F60002A968CAD9DADAEADBFAD2A9780932B0DDB
:109F700090932C0DA0932D0DB0932E0D2E962CADFD
:109F80003DAD4EAD5FAD2E9720932F0D3093300D2C
:109F90004093310D5093320D8AAD9BADACADBDAD4C
:109FA0008093330D9093340DA093350DB093360DFF
:109FB0000E94ED43CD58DF4F0FB6F894DEBF0FBEC1
:109FC000CDBFDF91CF911F910F91FF90EF90DF9068
:109FD000CF90BF90AF909F908F907F906F905F9049
:109FE0004F903F902F900C9471512AAD3BAD4CADEA
:109FF0005DAD2093330D3093340D4093350D509368
:10A00000360DECECF6E00C947146CD58DF4F0FB6F0
:10A01000F894DEBF0FBECDBFDF91CF911F910F919E
:10A02000FF90EF90DF90CF90BF90AF909F908F9078
:10A030007F906F905F904F903F902F900895EF9298
:10A04000FF920F931F93CF93DF937B018A01E90166
:10A050002091730D3091740D4091750D5091760DD6
:10A06000FC0160817181828193810E947F710E94D5
:10A070004F71E7E2FDE060837183828393832091D7
:10A08000770D3091780D4091790D50917A0DF7014F
:10A0900060817181828193810E947F710E944F71E2
:10A0A000EBE2FDE0608371838283938320917B0DDB
:10A0B00030917C0D40917D0D50917E0DF8016081B5
:10A0C0007181828193810E947F710E944F71EFE2C2
:10A0D000FDE0608371838283938320917F0D3091B3
:10A0E000800D4091810D5091820D688179818A8126
:10A0F0009B810E947F710E944F71E3E3FDE06083CA
:10A100007183828393839F014FE25DE06BE27DE088
:10A1100087E29DE00E94E1571092A70D1092A80DD2
:10A120001092A90D1092AA0D1092970D1092980DF1
:10A130001092990D10929A0D10929B0D10929C0DF9
:10A1400010929D0D10929E0D10929F0D1092A00DD9
:10A150001092A10D1092A20D1092A30D1092A40DB9
:10A160001092A50D1092A60DDF91CF911F910F9126
:10A17000FF90EF90089520917F0D3091800D4091D8
:10A18000810D5091820DFC016081718182819381EA
:10A190000E947F710E944F71E3E3FDE06083718351
:10A1A00082839383CF010C941D58809353080895A4
:10A1B0008091C10D811188C08091C00D811184C032
:10A1C0008091BF0D811180C008959091C00095FFCE
:10A1D000FCCF8093C600319684918111F6CFE0E1E7
:10A1E000F7E007C09091C00095FFFCCF8093C600B8
:10A1F000319684918111F6CF8091C10D8823D1F0E1
:10A200006091C20D7091C30D8091C40D9091C50DE8
:10A210000E944C6F2091730D3091740D4091750D1B
:10A220005091760D0E94B16EAB01BC018FE197E0B9
:10A230000E94880B8091C00D8823D1F06091C60DDB
:10A240007091C70D8091C80D9091C90D0E944C6FFF
:10A250002091770D3091780D4091790D50917A0DC4
:10A260000E94B16EAB01BC0183E297E00E94880BB3
:10A270008091BF0D8823D1F06091CA0D7091CB0DF4
:10A280008091CC0D9091CD0D0E944C6F20917B0D53
:10A2900030917C0D40917D0D50917E0D0E94B16EEC
:10A2A000AB01BC0187E297E00E94880B8091C0005F
:10A2B00085FFFCCF8AE08093C6001092C10D1092FA
:10A2C000C00D1092BF0D0895EAE0F7E085CF10921F
:10A2D000C10D1092C00D1092BF0D089580934501DD
:10A2E0000895EFE6F0E080818260808308951F92F8
:10A2F0000F920FB60F9211240F931F932F933F933A
:10A300004F935F936F937F938F939F93AF93BF937D
:10A31000EF93FF938091D20D9091D30D892B09F08B
:10A320007DC19091550880915408981771F0E09183
:10A3300054088DE4E89FF0011124EA5AF74FDF0139
:10A34000A45BBF4F81E08C9302C0E0E0F0E0F093AB
:10A35000D30DE093D20D309709F45AC1DF01A45B0D
:10A36000BF4F81E08C931092D40D1092D50D1092B6
:10A37000D60D1092D70D60AD71AD61349CE97907AF
:10A3800028F461329EE4790748F002C060E47CE979
:10A39000769567957695679584E007C0613197E279
:10A3A000790730F07695679582E08093D80D07C0E5
:10A3B0008093D80D6032710510F460E270E0605255
:10A3C0007109611588E07807D0F0872F9927880FE9
:10A3D000991F880F991F855D984FFC013296459112
:10A3E0005491AA27659F9001649F210D3A1F0694FE
:10A3F0002A1F3A1F1124FC01859194911DC09B01D5
:10A40000369527952C7F255D344FF90185919491E0
:10A410002E5F3F4FF90145915491FB01E770FF27F3
:10A420004E9F90014F9F300D5E9F300D112413E021
:10A43000369527951A95E1F7821B930B8436910583
:10A44000A0F4EAE8F2E006C09091C00095FFFCCFCE
:10A450008093C60081918111F7CF4AE050E081ECF2
:10A4600095E00E94062E84E690E09093DA0D8093AA
:10A47000D90DE091D20DF091D30D64AD75AD70930F
:10A48000DC0D6093DB0D61349CE9790728F46132BF
:10A490008EE4780748F002C060E47CE97695679521
:10A4A0007695679584E007C0613197E2790730F0CF
:10A4B0007695679582E08093D80D08C081E08093FF
:10A4C000D80D6032710510F460E270E060527109DD
:10A4D000611588E07807E0F0872F9927880F991F8A
:10A4E000880F991F855D984FFC0132962591349114
:10A4F000AA27639FA001629F410D5A1F06944A1F1D
:10A500005A1F1124FC0125913491241B350B1EC0C8
:10A51000CB01969587958C7F855D944FFC012591A5
:10A5200034910296FC0145915491FB01E770FF279D
:10A530004E9FC0014F9F900D5E9F900D112443E0F0
:10A54000969587954A95E1F7281B390B24363105F6
:10A55000A0F4EAE8F2E006C09091C00095FFFCCFBD
:10A560008093C60081918111F7CF4AE050E081ECE1
:10A5700095E00E94062E24E630E0C901A0E0B0E09C
:10A580008093DD0D9093DE0DA093DF0DB093E00D71
:10A590003093890020938800E091D20DF091D30D83
:10A5A00080899189A289B389B695A7959795879552
:10A5B000B095A095909581959F4FAF4FBF4F8093D9
:10A5C000E10D9093E20DA093E30DB093E40D809321
:10A5D000E50D9093E60DA093E70DB093E80D809301
:10A5E000E90D9093EA0DA093EB0DB093EC0D8093E1
:10A5F000ED0D9093EE0DA093EF0DB093F00D109232
:10A60000CE0D1092CF0D1092D00D1092D10D06C02C
:10A6100080ED97E09093890080938800E091D20DBF
:10A62000F091D30D309709F460C480A18093F10DAF
:10A6300080FF38C0459A8FEF80934101809145019A
:10A640008823A1F1329942C480E029C080819181A0
:10A65000A281B381181619061A061B06FCF4809114
:10A66000AF0D9091B00DA091B10DB091B20D80934E
:10A67000C20D9093C30DA093C40DB093C50D81E09E
:10A680008093C10D80899189A289B3898093CE0D71
:10A690009093CF0DA093D00DB093D10D81E0809316
:10A6A000F20D04C0459881E0809341018091F10D45
:10A6B00081FF3CC047988FEF809342018091450114
:10A6C0008823C1F1339907C480E02DC0E091D20DF9
:10A6D000F091D30D84819581A681B7811816190652
:10A6E0001A061B06FCF48091B30D9091B40DA09155
:10A6F000B50DB091B60D8093C60D9093C70DA09384
:10A70000C80DB093C90D81E08093C00D80899189F7
:10A71000A289B3898093CE0D9093CF0DA093D00DD5
:10A72000B093D10D81E08093F30D04C0479A81E08E
:10A73000809342018091F10D82FF3CC02A988FEFF7
:10A7400080934301809145018823C1F13499C8C3A6
:10A7500080E02DC0E091D20DF091D30D80859185E0
:10A76000A285B385181619061A061B06FCF48091FB
:10A77000B70D9091B80DA091B90DB091BA0D80931D
:10A78000CA0D9093CB0DA093CC0DB093CD0D81E06D
:10A790008093BF0D80899189A289B3898093CE0D62
:10A7A0009093CF0DA093D00DB093D10D81E0809305
:10A7B000F40D04C02A9A81E0809343018091F10D49
:10A7C00083FF03C0289A8FEF02C0289881E080930E
:10A7D000440120E030E081C18091C00087FF19C0B2
:10A7E000E091C6004091420650914306CA0101968D
:10A7F0008F779927609144067091450686179707D1
:10A8000041F0DA01AE53BA4FEC9390934306809334
:10A810004206E091D20DF091D30D8091E10D90911F
:10A82000E20DA091E30DB091E40D40815181628170
:10A830007381840F951FA61FB71F8093E10D90931E
:10A84000E20DA093E30DB093E40D181619061A0655
:10A850001B0644F55F9A4089518962897389841B7C
:10A86000950BA60BB70B8093E10D9093E20DA0938F
:10A87000E30DB093E40D409141018091AF0D9091B3
:10A88000B00DA091B10DB091B20D840F911DA11D1D
:10A89000B11D8093AF0D9093B00DA093B10DB09307
:10A8A000B20D5F98E091D20DF091D30D8091E50D3E
:10A8B0009091E60DA091E70DB091E80D448155818E
:10A8C00066817781840F951FA61FB71F8093E50DC2
:10A8D0009093E60DA093E70DB093E80D18161906B6
:10A8E0001A061B0644F5469A408951896289738984
:10A8F000841B950BA60BB70B8093E50D9093E60D8B
:10A90000A093E70DB093E80D409142018091B30D03
:10A910009091B40DA091B50DB091B60D840F911D1D
:10A92000A11DB11D8093B30D9093B40DA093B50DEF
:10A93000B093B60D4698E091D20DF091D30D809171
:10A94000E90D9091EA0DA091EB0DB091EC0D4085D1
:10A95000518562857385840F951FA61FB71F80934D
:10A96000E90D9093EA0DA093EB0DB093EC0D181642
:10A9700019061A061B0644F52B9A408951896289EB
:10A980007389841B950BA60BB70B8093E90D9093ED
:10A99000EA0DA093EB0DB093EC0D40914301809133
:10A9A000B70D9091B80DA091B90DB091BA0D840F6B
:10A9B000911DA11DB11D8093B70D9093B80DA0936B
:10A9C000B90DB093BA0D2B98E091D20DF091D30D43
:10A9D0008091ED0D9091EE0DA091EF0DB091F00DE5
:10A9E0004485558566857785840F951FA61FB71FFB
:10A9F0008093ED0D9093EE0DA093EF0DB093F00DBD
:10AA0000181619061A061B0644F5299A4089518919
:10AA100062897389841B950BA60BB70B8093ED0D90
:10AA20009093EE0DA093EF0DB093F00D4091440183
:10AA30008091BB0D9091BC0DA091BD0DB091BE0D4C
:10AA4000840F911DA11DB11D8093BB0D9093BC0D72
:10AA5000A093BD0DB093BE0D29988091CE0D90911D
:10AA6000CF0DA091D00DB091D10D0196A11DB11DBA
:10AA70008093CE0D9093CF0DA093D00DB093D10DB8
:10AA80004091CE0D5091CF0D6091D00D7091D10DB0
:10AA90002F5F3F4FE091D20DF091D30D80899189C6
:10AAA000A289B389481759076A077B07B0F040911C
:10AAB000CE0D5091CF0D6091D00D7091D10DE091E0
:10AAC000D20DF091D30D84899589A689B789841711
:10AAD0009507A607B70748F4E0C08091D80D90E02D
:10AAE000281739070CF478CEE2CF4091DD0D509154
:10AAF000DE0D6091DF0D7091E00D048D158D268DBA
:10AB0000378DAA27419FB12D529FC001629F900DA2
:10AB1000619F800D911D429FB00D811D9A1F519F15
:10AB2000B00D811D9A1F609FB00D811D9A1F509F0F
:10AB3000B10D8A1F9A1FB6958A1F9A1F112444AD22
:10AB400055AD480F591F5093DC0D4093DB0D80AD80
:10AB500091ADA2ADB3AD60E070E084179507A60794
:10AB6000B70720F49093DC0D8093DB0D6091DB0D33
:10AB70007091DC0D61349CE9790728F461328EE430
:10AB8000780748F002C060E47CE976956795769591
:10AB9000679584E007C0613197E2790730F07695D8
:10ABA000679582E08093D80D08C081E08093D80D2E
:10ABB0006032710510F460E270E060527109611555
:10ABC00088E07807E0F0872F9927880F991F880F72
:10ABD000991F855D984FFC01329625913491AA27E3
:10ABE000639FA001629F410D5A1F06944A1F5A1F7E
:10ABF0001124FC0125913491241B350B1EC0CB017F
:10AC0000969587958C7F855D944FFC0125913491B5
:10AC10000296FC0145915491FB01E770FF274E9F7E
:10AC2000C0014F9F900D5E9F900D1124F3E096950B
:10AC30008795FA95E1F7281B390B24363105A0F4E6
:10AC4000EAE8F2E006C09091C00095FFFCCF809347
:10AC5000C60081918111F7CF4AE050E081EC95E088
:10AC60000E94062E24E630E030938900209388006D
:10AC70008091DD0D9091DE0DA091DF0DB091E00D82
:10AC8000820F931FA11DB11D8093DD0D9093DE0DEA
:10AC9000A093DF0DB093E00DF3C04091CE0D509125
:10ACA000CF0D6091D00D7091D10D808D918DA28DC1
:10ACB000B38D84179507A607B70708F0D9C0409150
:10ACC000D40D5091D50D6091D60D7091D70D048D96
:10ACD000158D268D378DAA27419FB12D529FC0011A
:10ACE000629F900D619F800D911D429FB00D811D4F
:10ACF0009A1F519FB00D811D9A1F609FB00D811D3D
:10AD00009A1F509FB10D8A1F9A1FB6958A1F9A1FCE
:10AD100011242091DB0D3091DC0DE05CFF4F2817F2
:10AD2000390718F42081318102C0281B390B80813A
:10AD30009181A281B381A90160E070E048175907B1
:10AD40006A077B0708F49C0121349CE9390728F441
:10AD500021328EE4380748F002C020E43CE9369501
:10AD600027953695279584E007C0213197E239076A
:10AD700030F03695279582E08093D80D08C081E0A9
:10AD80008093D80D2032310510F420E230E0B90173
:10AD900060527109611588E07807E0F0872F9927E4
:10ADA000880F991F880F991F855D984FFC01329677
:10ADB00045915491AA27659F9001649F210D3A1FE8
:10ADC00006942A1F3A1F1124FC0145915491421BFD
:10ADD000530B1EC0CB01969587958C7F855D944F54
:10ADE000FC01459154910296FC0125913491FB019F
:10ADF000E770FF272E9FC0012F9F900D3E9F900D63
:10AE0000112433E0969587953A95E1F7481B590B45
:10AE100044365105A0F4EAE8F2E006C09091C00083
:10AE200095FFFCCF8093C60081918111F7CF4AE056
:10AE300050E081EC95E00E94062E44E650E05093ED
:10AE40008900409388008091D40D9091D50DA091F8
:10AE5000D60DB091D70D840F951FA11DB11D809304
:10AE6000D40D9093D50DA093D60DB093D70D08C0F7
:10AE70008091D90D9091DA0D90938900809388008C
:10AE80004091CE0D5091CF0D6091D00D7091D10DAC
:10AE9000E091D20DF091D30D80899189A289B38977
:10AEA000481759076A077B0700F11092D30D1092DB
:10AEB000D20D90915508809154089817B1F0809167
:10AEC00054088F5F8F70809354080FC08091F20DEB
:10AED0008111BCCBE3CB8091F30D8111F7CB22CC58
:10AEE0008091F40D811136CC61CCFF91EF91BF912F
:10AEF000AF919F918F917F916F915F914F913F9112
:10AF00002F911F910F910F900FBE0F901F901895CA
:10AF10003D9A3F9A229A209A569A5E9A569A5E9A3B
:10AF20000D9A159A569A5E9A3A98429A3B98439A85
:10AF30003C98449A579A5F985E9A3E9A46985E9AD1
:10AF4000239A2B98159A219A29985E9AA1E8B0E045
:10AF50008C918F7E8C938C9188608C93E0E8F0E0EC
:10AF600080818D7F808380818E7F808380818F73BD
:10AF7000808380818F7C80838C91887F82608C939A
:10AF800080E090E49093890080938800109285007F
:10AF900010928400EFE6F0E080818260808381E09F
:10AFA00080934501789408959091550880915408B4
:10AFB000981731F00E94255A81E00E943716F4CF8D
:10AFC0000895CF93DF93EFB7F894EC0188819981CE
:10AFD000AA81BB818093AF0D9093B00DA093B10D6A
:10AFE000B093B20DEB0188819981AA81BB818093D6
:10AFF000B30D9093B40DA093B50DB093B60DEA01C7
:10B0000088819981AA81BB818093B70D9093B80DF7
:10B01000A093B90DB093BA0DE90188819981AA81F5
:10B02000BB818093BB0D9093BC0DA093BD0DB093DD
:10B03000BE0DEFBFDF91CF9108952FB7F894FC01BB
:10B0400080819181A281B3818093BB0D9093BC0DCF
:10B05000A093BD0DB093BE0D2FBF08950F931F9306
:10B060009FB7F89424E0829FF0011124E155F24F3C
:10B0700000811181228133819FBFB801C9011F91D5
:10B080000F9108950E94D4575E9A5E9A159A5E9A1F
:10B09000089580916F008D7F80936F0006C080912E
:10B0A00054088F5F8F708093540890915508809159
:10B0B000540898130AC01092D30D1092D20D8091AB
:10B0C0006F00826080936F00089590915508809181
:10B0D0005408981751F3E3CF20914E0130914F015E
:10B0E000409150015091510160E070E08FE793E48E
:10B0F0000E94B16E6093030E7093040E8093050E50
:10B100009093060E08958E5F914FFC01808190E030
:10B1100008950F931F93CF93DF93EC01662309F4F7
:10B1200061C0E2E1F0E107C09091C00095FFFCCF63
:10B130008093C600319684918111F6CF4AE050E0A9
:10B1400070E081EC95E00E94E82DE9E1F0E107C0B4
:10B150009091C00095FFFCCF8093C60031968491FA
:10B160008111F6CF8091C00085FFFCCF8AE08093EB
:10B17000C6000E940E1636C0C901880F991F880F9D
:10B18000991FFC01E95CFF4E659174916C177D0776
:10B190003CF521503109220F331F220F331FF901D3
:10B1A000EB5CFF4E05911491295C3F4EF9014591EE
:10B1B0005491FC01EB5CFF4E25913491C41BD50BDF
:10B1C000201B310BC29FC001C39F900DD29F900DD9
:10B1D0001124641B750B0E946872600F711F13C0ED
:10B1E0004F5F01C041E0242F30E04D3309F0C4CF60
:10B1F0002D33310531F4E5E2F1E185919491BC0103
:10B2000002C060E070E020EF3FE3261B370BC9016E
:10B21000DF91CF911F910F910895CF93DF9321E09C
:10B2200030E0D901AA0FBB1FAA0FBB1FFD01E95CCB
:10B23000FF4E659174916817790744F521503109E3
:10B24000220F331F220F331FF901EB5CFF4EC59114
:10B25000D491295C3F4EF90145915491FD01EB5C7D
:10B26000FF4E25913491FC01E41BF50B2C1B3D0B8B
:10B27000E29FC001E39F900DF29F900D1124641B8B
:10B28000750B0E9468726C0F7D1F0BC02F5F3F4FC4
:10B290002D33310509F0C5CFE5E2F1E185919491B7
:10B2A000BC0120EF3FE3261B370BC901DF91CF9193
:10B2B00008952F923F924F925F926F927F928F925A
:10B2C0009F92AF92BF92CF92DF92EF92FF920F9335
:10B2D0001F93CF93DF938C01662351F1E2E1F0E1FC
:10B2E00007C09091C00095FFFCCF8093C6003196B7
:10B2F00084918111F6CF4AE050E070E081EC95E056
:10B300000E94E82DE9E2F1E107C09091C00095FFAD
:10B31000FCCF8093C600319684918111F6CF809145
:10B32000C00085FFFCCF8AE08093C6000E940E1605
:10B33000C0EFDFE3C01BD10B41E05EC09C01220FD8
:10B34000331F220F331FF901EB5CFF4E65907490A1
:10B35000C615D7050CF04FC00197880F991F880FAD
:10B36000991FFC01E95CFF4E259034908B5C9F4E49
:10B37000FC0105911491F901E95CFF4E4590549050
:10B38000B101882777FD8095982F0E944C6F6B0143
:10B390007C01BE01601B710B882777FD8095982F7B
:10B3A0000E944C6F4B015C01B2016219730988273E
:10B3B00077FD8095982F0E944C6F9B01AC01C501D1
:10B3C000B4010E947F714B015C01B301601B710BE2
:10B3D000882777FD8095982F0E944C6F9B01AC01C8
:10B3E000C501B4010E94B16E9B01AC01C701B60159
:10B3F0000E94D16D17C04F5F842F90E04D3309F04C
:10B400009DCFCD9759F4E7E2F1E1659174918827DA
:10B4100077FD8095982F0E944C6F04C060E070E02B
:10B4200080E090E0DF91CF911F910F91FF90EF901E
:10B43000DF90CF90BF90AF909F908F907F906F9054
:10B440005F904F903F902F9008952F923F924F9290
:10B450005F926F927F928F929F92AF92BF92CF92A4
:10B46000DF92EF92FF920F931F93CF93DF9300D061
:10B47000CDB7DEB78091F50D882309F4BFC18FB732
:10B48000F8941092F50D8FBF60E08091FC0D9091C3
:10B49000FD0D0E9459596B017C019B01AC0160912B
:10B4A000F60D7091F70D8091F80D9091F90D0E94B5
:10B4B000D06DB62EA72E182F092FA5019801852F24
:10B4C000942FA32FB22F8093070E9093080EA09372
:10B4D000090EB0930A0E20E030E040E251E4D501BD
:10B4E000F8016B2F7A2F8F2F9E2F0E94AD701816A8
:10B4F0000CF41DC120E030E040E251ECD501F80130
:10B500006B2F7A2F8F2F9E2F0E94AA6E87FD0BC163
:10B5100080910B0E8111FCC020915201309153019A
:10B520004091540150915501D501F8016B2F7A2DAE
:10B530008F2F902F0E947F71762E672E89839A839A
:10B54000A301382F292F852F942FA32FB22F80935B
:10B55000100E9093110EA093120EB093130E209123
:10B560000C0E30910D0E40910E0E50910F0ED50124
:10B57000F8016B2F7A2D8F2F902F0E94D16D8B01A8
:10B580002C018090140E9090150EA090160EB09085
:10B59000170E282D392D4A2D5B2D602F712F842DEC
:10B5A000952D0E94AA6E87FF9DC084012501802FE2
:10B5B000912FA42DB52D80930C0E90930D0EA0937A
:10B5C0000E0EB0930F0E20914E0130914F0140911D
:10B5D000500150915101602F712F842D952D0E94A3
:10B5E0007F714B015C01862F992DAA2DBB2D809375
:10B5F000180E9093190EA0931A0EB0931B0E209163
:10B600001C0E30911D0E40911E0E50911F0EC70151
:10B61000B6010E94D06D20914A0130914B014091BA
:10B620004C0150914D010E947F7120ED3CEC4CE4A7
:10B630005DE30E947F711B012C0123E333E343E7A9
:10B640005FE36091200E7091210E8091220E909107
:10B65000230E0E947F719B01AC01C201B1010E94C7
:10B66000D16D8B012C01862F912FA42DB52D8093A8
:10B67000200E9093210EA093220EB093230EC09221
:10B680001C0ED0921D0EE0921E0EF0921F0E282D61
:10B69000392D4A2D5B2DD301F980EA806B2F762D51
:10B6A0008F2D9E2D0E94D16D202F312F442D552D91
:10B6B0000E94D06D8B017C0120E030E0A901712F48
:10B6C0009F2D0E94AA6E87FD3CC020E030E04FE72E
:10B6D00053E4602F712F8E2D9F2D0E94AD70181690
:10B6E000A4F528C08090030E9090040EA090050E43
:10B6F000B090060E282D392D4A2D5B2D602F712F0D
:10B70000842D952D0E94AD7018160CF050CF4DCFA2
:10B7100010920C0E10920D0E10920E0E10920F0E33
:10B7200010920B0EF9CE81E080930B0E0AC081E0DF
:10B7300080930B0E00E010E08FE7E82E93E4F92EE3
:10B7400004C000E010E0E12CF12C2091FC0D3091C0
:10B75000FD0D4091240E5091250E421753071CF009
:10B760001092020E11C040915601509157012417BA
:10B770003507B4F7602F712F8E2D9F2D0E94196F02
:10B78000759567956093020E0E94252B0091260EF9
:10B790001091270E2091280E3091290E601B710BFD
:10B7A000820B930B683873418105910538F10E9433
:10B7B000252B6093260E7093270E8093280E90936E
:10B7C000290E8091FA0D9091FB0D20912A0E309157
:10B7D0002B0E281739078CF420915801309159010C
:10B7E0008217930754F42091FE0D3091FF0D8217BC
:10B7F00093070CF002C05A9A01C05A980F900F900C
:10B80000DF91CF911F910F91FF90EF90DF90CF903C
:10B81000BF90AF909F908F907F906F905F904F9070
:10B820003F902F9008952F923F924F925F926F9288
:10B830007F928F929F92AF92BF92CF92DF92EF92C0
:10B84000FF920F931F93CF93DF93C0EFDFE3C81BEB
:10B85000D90B81E090E09C01220F331F220F331F90
:10B86000F901EB5CFF4E65907490C615D7050CF09E
:10B870004FC00197880F991F880F991FFC01E95C41
:10B88000FF4E259034908B5C9F4EFC0105911491E6
:10B89000F901E95CFF4E45905490B101882777FD8E
:10B8A0008095982F0E944C6F6B017C01BE01601B3C
:10B8B000710B882777FD8095982F0E944C6F4B0164
:10B8C0005C01B20162197309882777FD8095982F72
:10B8D0000E944C6F9B01AC01C501B4010E947F71B5
:10B8E0004B015C01B301601B710B882777FD8095CC
:10B8F000982F0E944C6F9B01AC01C501B4010E94BE
:10B90000B16E9B01AC01C701B6010E94D16D0FC0A1
:10B9100001968D33910509F09ECFE7E2F1E1659143
:10B920007491882777FD8095982F0E944C6FDF9146
:10B93000CF911F910F91FF90EF90DF90CF90BF902C
:10B94000AF909F908F907F906F905F904F903F90BF
:10B950002F9008951092140E1092150E1092160E3C
:10B960001092170E20914E0130914F0140915001DD
:10B970005091510160E070E08FE793E40E94B16E56
:10B980006093030E7093040E8093050E9093060E41
:10B99000559A529A87ED80937A00EEE7F0E0108294
:10B9A00080818068808380818064808380E888BD16
:10B9B000EEE6F0E08081846080836AEF70E080E0F2
:10B9C00090E00E94612B60E085E090E00E94895841
:10B9D0009093250E8093240E60E083E191E00E9415
:10B9E0008958909357018093560185E090E00E941A
:10B9F0000D5990932B0E80932A0E86E990E00E94B9
:10BA00000D5990935901809358010895089560E06D
:10BA100080E090E00E9489581092F60D1092F70D88
:10BA20001092F80D1092F90D80E090E00E940D59EF
:10BA30009093FF0D8093FE0D1092010E1092000E58
:10BA40001092020E5D981092FF0D1092FE0D5A9802
:10BA500008952F923F924F925F926F927F928F92B2
:10BA60009F92AF92BF92CF92DF92EF92FF920F938D
:10BA70001F93CF93DF93CDB7DEB7E1970FB6F8945E
:10BA8000DEBF0FBECDBF688B798B8A8B9B8B0E94EC
:10BA9000252B6C8B7D8B8E8B9F8BEEE9F2E006C0A5
:10BAA0009091C00095FFFCCF8093C60081918111D9
:10BAB000F7CF8091C00085FFFCCF8AE08093C6005D
:10BAC0000E94075D8FE78093020E4C885D886E8828
:10BAD0007F884C865D866E867F86AFE7CA2ED12C26
:10BAE000E12CF12CBFE78B2E912CA12CB12C8EA632
:10BAF0009FA6A8AAB9AA11E01B861A86EBE2FFE06E
:10BB000094909FA2E3E3FFE0A490A8A6E8E3FFE0FF
:10BB1000B490B9A6EFE3FFE084908AA6E6E4FFE0E4
:10BB200094909BA6ECE4FFE0A490ACA68091F50D68
:10BB3000882309F4BBC28FB7F8941092F50D8FBF1C
:10BB400060E08091FC0D9091FD0D0E9459596E832B
:10BB50007F8388879987762F6F81982F8985272FF4
:10BB6000362F492F582FB88DA98DEA8DFB8D6B2F5D
:10BB70007A2FCF010E94AD70181644F0BE80B88EA7
:10BB80008F80898E98849A8EA984AB8E7E816F81F6
:10BB900098858985272F362F492F582FECA1602FA4
:10BBA000722D832D9E2F0E94AA6E87FD05C00E81E7
:10BBB0002F803884B984BCA2112309F43FC378894B
:10BBC00069899A898B89272F362F492F582FBE8153
:10BBD000AF81E885F9856B2F7A2FCF010E94AD7078
:10BBE00018160CF063C20E94252B6419750986098A
:10BBF0009709693873418105910508F457C28EA5EC
:10BC00009FA5A8A9B9A98C199D09AE09BF09B59529
:10BC1000A795979587958093020E0E94252B6C8798
:10BC20007D878E879F874B015C0184189508A60845
:10BC3000B70888A299A2AAA2BBA29888988EA988C0
:10BC4000A98EBA88BA8E8B888B8EF8C20E94252B5B
:10BC50008C849D84AE84BF84681979098A099B0904
:10BC6000693873418105910508F41FC20E94252B94
:10BC70002B013C018A849B84892809F4FCC1DC01E6
:10BC8000CB018C849D84AE84BF8488199909AA094C
:10BC9000BB0988A099A0AAA0BBA0880E991EAA1EC5
:10BCA000BB1E28A139A14AA15BA1281B390B4A0B55
:10BCB0005B0BCA01B901A70196010E945872A50148
:10BCC00094010E949E728EA59FA5A8A9B9A9280FCC
:10BCD000391F4A1F5B1F243131054105510524F1ED
:10BCE0002EA73FA748AB59AB2C3E31054105510566
:10BCF00044F02BEE30E040E050E02EA73FA748ABE9
:10BD000059AB8EA59FA5A8A9B9A980389105A10511
:10BD1000B105C4F0EEEFCE2ED12CE12CF12CC81AD7
:10BD2000D90AEA0AFB0A12C024E130E040E050E000
:10BD30002EA73FA748AB59AB74E1C72ED12CE12CFD
:10BD4000F12C04C0CEA4DFA4E8A8F9A88FA1EBE2EF
:10BD5000FFE008C09091C00095FFFCCF8093C60023
:10BD6000319684918111F6CF2AE030E04EA55FA58F
:10BD700068A979A981EC95E00E94D72D88A5E3E315
:10BD8000FFE008C09091C00095FFFCCF8093C600F3
:10BD9000319684918111F6CF2AE030E0B701A601F7
:10BDA00081EC95E00E94D72D89A5E8E3FFE008C06B
:10BDB0009091C00095FFFCCF8093C600319684918E
:10BDC0008111F6CF22E030E08CA1402F522D632D5F
:10BDD000782F81EC95E00E94E12E8AA5EFE3FFE049
:10BDE00008C09091C00095FFFCCF8093C6003196AB
:10BDF00084918111F6CF22E030E0F88DE98D9A8DA3
:10BE00008B8D4F2F5E2F692F782F81EC95E00E944C
:10BE1000E12E8091C00085FFFCCF8AE08093C600B0
:10BE20004A855B85433051050CF425C1C701B60135
:10BE30000E944C6F20E030E040E850E40E947F71A7
:10BE40006C8F7D8F8E8F9F8F8CA1202F322D432D55
:10BE5000582FB88DA98DEA8D1B8D6B2F7A2F8E2FC1
:10BE6000912F0E94D06D20ED3FE049E450E40E9404
:10BE70007F7120E030E040E05FE30E947F719B0132
:10BE8000AC016C8D7D8D8E8D9F8D0E94B16E362E96
:10BE9000072F182F9C8FC501B4010E944C6F20E022
:10BEA00030E04AE754E40E94B16EA62E972E282E69
:10BEB000892E8BA5E6E4FFE008C09091C00095FFB5
:10BEC000FCCF8093C600319684918111F6CF22E099
:10BED00030E08C8D432D502F612F782F81EC95E031
:10BEE0000E94E12E8CA5ECE4FFE008C09091C00018
:10BEF00095FFFCCF8093C600319684918111F6CFD7
:10BF000022E030E04A2D592D622D782D81EC95E00C
:10BF10000E94E12E8091C00085FFFCCF8AE08093D3
:10BF2000C6002AE939E949E15FE3EC8D632D702F02
:10BF3000812F9E2F0E947F71362E072F182FB92E2A
:10BF4000762F272F302F412F5B2D632D702F812FC0
:10BF50009B2D0E94D16D2A2D392D422D582D0E94E6
:10BF6000B16E6C8F7CA38DA39EA32A2D392D422DFB
:10BF7000582D632D702F812F9B2D0E947F7120E003
:10BF800030E040E05EE30E947F71A62E972E282EBF
:10BF9000892EE2E5FFE007C09091C00095FFFCCF3D
:10BFA0008093C600319684918111F6CF8091C000B4
:10BFB00085FFFCCF8AE08093C600EFE5FFE007C075
:10BFC0009091C00095FFFCCF8093C600319684917C
:10BFD0008111F6CF22E030E0432D502F612F7B2DD1
:10BFE00081EC95E00E94E12E8091C00085FFFCCF9E
:10BFF0008AE08093C600E5E6FFE007C09091C000AC
:10C0000095FFFCCF8093C600319684918111F6CFC5
:10C0100022E030E0FC8DECA19DA18EA14F2F5E2F80
:10C02000692F782F81EC95E00E94E12E8091C0006D
:10C0300085FFFCCF8AE08093C600EBE6FFE007C0F7
:10C040009091C00095FFFCCF8093C60031968491FB
:10C050008111F6CF22E030E04A2D592D622D782D46
:10C0600081EC95E00E94E12E8091C00085FFFCCF1D
:10C070008AE08093C6008EA59FA5A8A9B9A98C0DBA
:10C080009D1DAE1DBF1DB595A7959795879580936E
:10C09000020E8A859B8501969B878A870889298855
:10C0A0003A888B888CA211E001C010E020E030E0DB
:10C0B00040EA51E4B889A989EA89FB896B2F7A2F74
:10C0C000CF010E94D16D9B01AC01BE81AF81E8859B
:10C0D000F9856B2F7A2FCF010E94AD70181694F45A
:10C0E000E1E7FFE007C09091C00095FFFCCF80938F
:10C0F000C600319684918111F6CF8091C00085FFF2
:10C10000FCCF98C00E94252B8C889D88AE88BF8864
:10C11000681979098A099B09613D77408105910574
:10C1200008F43FC00E94252B6C8B7D8B8E8B9F8BE0
:10C13000EAE9FFE007C09091C00095FFFCCF809333
:10C14000C600319684918111F6CF60E08091FC0D9C
:10C150009091FD0D0E945959AB01BC0122E030E0E5
:10C1600081EC95E00E94E12EE0EAFFE007C09091AB
:10C17000C00095FFFCCF8093C60031968491811159
:10C18000F6CF6091020E4AE050E070E081EC95E05D
:10C190000E94E82D8091C00085FFFCCF8AE080934B
:10C1A000C6000E94252B6A837B838C839D830E941B
:10C1B000252B8C849D84AE84BF84840C951CA61C86
:10C1C000B71C2A813B814C815D81281939094A09B4
:10C1D0005B09260F371F481F591F21383F44424132
:10C1E000510590F0E4EAFFE007C09091C00095FF90
:10C1F000FCCF8093C600319684918111F6CF809157
:10C20000C00085FFFCCF16C0AA85BB8516970CF42D
:10C210008DCCE1ECFFE007C09091C00095FFFCCF12
:10C220008093C600319684918111F6CF8091C00031
:10C2300085FFFCCF8AE08093C60015C078896989A4
:10C240009A898B89272F362F492F582FBE81AF818E
:10C250001885F9856B2F7A2F812F9F2F0E94AA6E48
:10C2600087FDF4CC22CFE1960FB6F894DEBF0FBE67
:10C27000CDBFDF91CF911F910F91FF90EF90DF9095
:10C28000CF90BF90AF909F908F907F906F905F9076
:10C290004F903F902F900895CF93DF931F92CDB78B
:10C2A000DEB789830E94075D0E94D31669818111E0
:10C2B0002FC0E2E1F0E107C08091C00085FFFCCF14
:10C2C0009093C600319694919111F6CF4AE050E0D8
:10C2D00070E081EC95E00E94E82D8091C00085FF20
:10C2E000FCCF8AE08093C600E6E4F1E107C09091BC
:10C2F000C00095FFFCCF8093C600319684918111D8
:10C30000F6CF8091C00085FFFCCF8AE08093C60005
:10C310000F90DF91CF910895CF93DF931F92CDB708
:10C32000DEB789830E94075D0E94D316698181115F
:10C330002FC0E2E1F0E107C08091C00085FFFCCF93
:10C340009093C600319694919111F6CF4AE050E057
:10C3500070E081EC95E00E94E82D8091C00085FF9F
:10C36000FCCF8AE08093C600E3E7F1E107C090913B
:10C37000C00095FFFCCF8093C60031968491811157
:10C38000F6CF8091C00085FFFCCF8AE08093C60085
:10C390000F90DF91CF9108955A980E94D316811182
:10C3A00021C0E2E1F0E107C09091C00095FFFCCF11
:10C3B0008093C600319684918111F6CFE0EAF1E1D5
:10C3C00007C09091C00095FFFCCF8093C6003196C6
:10C3D00084918111F6CF8091C00085FFFCCF8AE067
:10C3E0008093C60008951F920F920FB60F921124EA
:10C3F0002F933F934F935F936F937F938F939F936D
:10C40000AF93BF93EF93FF9380915A01811106C0C0
:10C410008091020E80932C0E81115D9A90912C0ECA
:10C4200080915A01891708F05D988F5F8F7780930C
:10C430005A0180912D0E833009F443C020F48130DD
:10C44000D1F0A8F50CC0853009F457C008F453C0EA
:10C45000863009F454C0873009F05AC052C0109297
:10C460007B0087E480937C0080917A0080648093D5
:10C470007A0081E019C02091780030917900809194
:10C480002E0E90912F0EA091300EB091310E820F92
:10C49000931FA11DB11D80932E0E90932F0EA0937C
:10C4A000300EB093310E82E080932D0E31C086E4C1
:10C4B00080937C0080917A00806480937A0083E08E
:10C4C000F3CF20917800309179008091320E9091D5
:10C4D000330EA091340EB091350E820F931FA11D23
:10C4E000B11D8093320E9093330EA093340EB0930F
:10C4F000350E84E0D9CF85E0D7CF86E0D5CF87E071
:10C50000D3CF10922D0E8091360E8F5F8093360E12
:10C510008091360E803108F474C02FEF3FE3809194
:10C520002E0E90912F0EA901481B590BCA01509352
:10C53000FD0D4093FC0D4091320E5091330E241BA3
:10C54000350B3093FB0D2093FA0D21E02093F50D70
:10C550001092360E10922E0E10922F0E1092300E58
:10C560001092310E1092370E1092380E1092390E32
:10C5700010923A0E10923B0E10923C0E10923D0E0D
:10C5800010923E0E1092320E1092330E1092340E14
:10C590001092350E20915601309157018217930762
:10C5A0004CF01092010E1092000E80E00E944C613F
:10C5B0000E9498162091FC0D3091FD0D8091240E63
:10C5C0009091250E821793074CF01092010E109255
:10C5D000000E80E00E948C610E9498162091FA0D56
:10C5E0003091FB0D8091580190915901281739071E
:10C5F00044F01092FF0D1092FE0D0E94CC610E943B
:10C600009816FF91EF91BF91AF919F918F917F917C
:10C610006F915F914F913F912F910F900FBE0F90AF
:10C620001F901895CF93DF93FC01148A178A84E832
:10C6300092E0938B828B13AA16AA92AB81ABDF0197
:10C64000A05BBF4F1C9213961C92DF01A25BBF4FF1
:10C650008D939C93DF01A359BF4F1C9213961C929C
:10C66000DF01A559BF4F8D939C93DF01A857BF4FA2
:10C6700029E111962C93119714961C92DF01A35770
:10C68000BF4F57961C92DF01A355BF4F1C921396C4
:10C690001C92DF01A555BF4F8D939C93DF01A853DA
:10C6A000BF4F1D921D921D921C921397DF01A05344
:10C6B000BF4F1D921D921D921C92139711821282E0
:10C6C0001082EF01C453DF4F188219821A821B8235
:10C6D000DF01AC52BF4F81E08C93118A108A0E9417
:10C6E000252B68577C4E8F4F9F4F688379838A83B1
:10C6F0009B83DF91CF910895DB01FC0120E03EE2B6
:10C700004C91403229F0283009F431934C914193F7
:10C710002F5F11962B30A1F7108208952F923F9230
:10C720004F925F926F927F928F929F92AF92BF9241
:10C73000CF92DF92EF92FF920F931F93CF93DF93ED
:10C74000CDB7DEB7C158D1090FB6F894DEBF0FBE22
:10C75000CDBF8C017B01212C4A0182E0880E911C07
:10C760006801E5EDCE0ED11C5801F6EDAF0EB11CFF
:10C770008EE3482E512C4C0E5D1E82E0480E511C5B
:10C78000EAEDF1E13490F3C09C85292F2871203126
:10C7900009F007C1F6018081813009F402C18230BD
:10C7A00009F0EFC0FEC061EB72E0CE01855A9F4FE9
:10C7B0000E948C75B701CE01855A9F4F0E948C75DF
:10C7C000BE016B587F4FCE01855A9F4F0E948C75DA
:10C7D00061EB72E0CE01855A9F4F0E948C752196C5
:10C7E0001FAE219724961FAE249784E892E09FAF56
:10C7F0008EAF21E0AE014B585F4FB401C2010E94E1
:10C800001835811139C0F6018081811135C0832D21
:10C81000EAEDF1E108C09091C00095FFFCCF809354
:10C82000C600319684918111F6CFA3EBB2E006C029
:10C830009091C00095FFFCCF8093C6008D9181112F
:10C84000F7CF8091C00085FFFCCF8AE08093C600BF
:10C85000DE01AB58BF4F06C09091C00095FFFCCFE2
:10C860008093C6008D918111F7CF8091C00085FF24
:10C87000FCCF8AE08093C6008BE1FE01E05CFF4FB5
:10C88000DE01939601900D928A95E1F784E892E09B
:10C890009AA389A3AE014F5D5F4FBE01655A7F4FDA
:10C8A000C8010E948E63CE0181960E94AC2ACE01FF
:10C8B000CE960E94AC2A5BC0853E09F458C08E32E9
:10C8C00009F455C08F3509F452C093FD50C081E082
:10C8D000203109F080E0F8018787811108C089853F
:10C8E000873409F044C08A858E3709F440C0380186
:10C8F000F3E06F0E711CBE016F5F7F4FC3010E949A
:10C900007C63F601808181111EC0D70106C0909121
:10C91000C00095FFFCCF8093C6008D918111F7CFA9
:10C92000D30106C09091C00095FFFCCF8093C60054
:10C930008D918111F7CF8091C00085FFFCCF8AE0F7
:10C940008093C60014C0813039F4F5018081918153
:10C950000196918380830BC0823049F4222D30E010
:10C96000F5018081918128173907F1F02394BE01E8
:10C970006F5F7F4FC4010E94863118160CF404CFFC
:10C9800013C0BE016F5F7F4FCE018B589F4F0E9437
:10C990007C636C961FAE6C97F701808181110ACF82
:10C9A00002CF8981811188CFCF57DF4F0FB6F8941E
:10C9B000DEBF0FBECDBFDF91CF911F910F91FF90D2
:10C9C000EF90DF90CF90BF90AF909F908F907F902F
:10C9D0006F905F904F903F902F900895EF92FF924D
:10C9E0000F931F93CF93DF93CDB7DEB76D970FB63D
:10C9F000F894DEBF0FBECDBF8C01FC01EB52FF4FA0
:10CA000010827C0184E1E80EF11C40E050E0BA01A4
:10CA1000C7010E94F9318BE1F701DE011396019005
:10CA20000D928A95E1F784E892E09A838983AE01BA
:10CA30004F5F5F4F6DE972E0C8010E948E63CE01C7
:10CA400001960E94AC2A6D960FB6F894DEBF0FBE19
:10CA5000CDBFDF91CF911F910F91FF90EF9008957F
:10CA6000EF92FF920F931F93CF93DF93EC011A8203
:10CA70008F89882321F0CE0144960E94E0327E0106
:10CA800088E8E80EF11C4FE160E0C7010E94906C5D
:10CA900081111FC0EAEDF1E107C09091C00095FF40
:10CAA000FCCF8093C600319684918111F6CFE0EEE1
:10CAB000F1E107C09091C00095FFFCCF8093C600C4
:10CAC000319684918111F6CF8091C00085FFFCCF13
:10CAD00076C08E0103571F4F41E0B701C8010E9485
:10CAE000153B811126C040E0B701C8010E94153BEB
:10CAF00081111FC0EDEEF1E107C09091C00095FFDC
:10CB0000FCCF8093C600319684918111F6CFE4EF7B
:10CB1000F1E107C09091C00095FFFCCF8093C60063
:10CB2000319684918111F6CF8091C00085FFFCCFB2
:10CB300046C0B801CE0144960E94F32F81111FC058
:10CB4000EDEEF1E107C09091C00095FFFCCF80931E
:10CB5000C600319684918111F6CFE7E0F2E107C07B
:10CB60009091C00095FFFCCF8093C60031968491D0
:10CB70008111F6CF8091C00085FFFCCF20C081E0FD
:10CB80008A83EAEDF1E107C09091C00095FFFCCFE8
:10CB90008093C600319684918111F6CFE7E1F2E1EE
:10CBA00007C09091C00095FFFCCF8093C6003196DE
:10CBB00084918111F6CF8091C00085FFFCCF8AE07F
:10CBC0008093C6008BE1FE017496DE01D39601903E
:10CBD0000D928A95E1F7CE01429698AB8FA7DF912F
:10CBE000CF911F910F91FF90EF900895FC0111825A
:10CBF00012820895FC012281222311F021E0218379
:10CC00000895FC0121812111118208952F923F92F4
:10CC10004F925F926F927F928F929F92AF92BF924C
:10CC2000CF92DF92EF92FF920F931F93CF93DF93F8
:10CC3000CDB7DEB7AA970FB6F894DEBF0FBECDBF53
:10CC40007C016B01342EFC018281882309F4B4C17C
:10CC50004701FDEA8F0E911CC4010E94E032F701EA
:10CC600011821B821E8284E892E09A838983C70125
:10CC7000429690AB87A7F60180818F3209F08CC075
:10CC80006FE270E0C6010E9497758C010F5F1F4F25
:10CC90009AE0292E44244394512C4C0E5D1E77C0FB
:10CCA0006FE270E0C8010E9497755C01009709F47B
:10CCB0007BC00817190708F077C03C01601A710A99
:10CCC000A301B801CE014E960E94B775EEE1F0E0E7
:10CCD000EC0FFD1FE60DF71D10828E01025E1F4F47
:10CCE000F80106C09091C00095FFFCCF8093C6006C
:10CCF00081918111F7CF8091C00085FFFCCF2092F8
:10CD0000C600F70167A570A96115710519F06E5F7E
:10CD10007F4F02C060E070E021E0AE01425E5F4FF5
:10CD2000CE0103960E94183581112BC0E2E2F2E198
:10CD300007C09091C00095FFFCCF8093C60031964C
:10CD400084918111F6CF06C09091C00095FFFCCF71
:10CD50008093C600F80181918F018111F5CFE6E340
:10CD6000F2E107C09091C00095FFFCCF8093C60010
:10CD7000319684918111F6CF8091C00085FFFCCF60
:10CD800014C1F70150AA47A685010F5F1F4F011577
:10CD9000110509F085CF05C0C701C196F70190AB19
:10CDA00087A7BC2CAD2C02C0B02EA12EF70167A521
:10CDB00070A9332009F49FC06115710519F06E5FE9
:10CDC0007F4F02C060E070E021E04B2D5A2DC4017E
:10CDD0000E941835882309F463C0F701E853FF4F18
:10CDE000D701A355BF4F51960D911D912D913C91A7
:10CDF00054970083118322833383E8E3F2E107C071
:10CE00009091C00095FFFCCF8093C600319684912D
:10CE10008111F6CFEB2DFA2D06C09091C00095FF41
:10CE2000FCCF8093C60081918111F7CFE5E4F2E158
:10CE300007C09091C00095FFFCCF8093C60031964B
:10CE400084918111F6CFF701E853FF4F4081518162
:10CE5000628173812AE030E081EC95E00E94C42D6C
:10CE60008091C00085FFFCCF8AE08093C600F70167
:10CE7000E053FF4F1082118212821382ECE4F2E140
:10CE800007C09091C00095FFFCCF8093C6003196FB
:10CE900084918111F6CF8091C00085FFFCCF85C0C1
:10CEA000EAE5F2E107C09091C00095FFFCCF8093C6
:10CEB000C600319684918111F6CFEB2DFA2D06C074
:10CEC0009091C00095FFFCCF8093C60081918111A5
:10CED000F7CFEEE6F2E107C09091C00095FFFCCFDE
:10CEE0008093C600319684918111F6CF8091C00065
:10CEF00085FFFCCF5AC06115710519F06E5F7F4F39
:10CF000002C060E070E026E54B2D5A2DC4010E945E
:10CF1000183581112BC0E0E7F2E107C09091C00005
:10CF200095FFFCCF8093C600319684918111F6CF96
:10CF3000EB2DFA2D06C09091C00095FFFCCF809399
:10CF4000C60081918111F7CFE4E8F2E107C090912A
:10CF5000C00095FFFCCF8093C6003196849181116B
:10CF6000F6CF8091C00085FFFCCF1FC081E0F701A4
:10CF70008083E6E8F2E107C09091C00095FFFCCF06
:10CF80008093C600319684918111F6CFF60106C0D8
:10CF90009091C00095FFFCCF8093C60081918111D4
:10CFA000F7CF8091C00085FFFCCF8AE08093C60058
:10CFB000CE0101960E94AC2AAA960FB6F894DEBF65
:10CFC0000FBECDBFDF91CF911F910F91FF90EF90DA
:10CFD000DF90CF90BF90AF909F908F907F906F9099
:10CFE0005F904F903F902F9008955F926F927F9245
:10CFF0008F929F92AF92BF92CF92DF92EF92FF9269
:10D000000F931F93CF93DF93CDB7DEB7AA970FB6D9
:10D01000F894DEBF0FBECDBF8C016B01FC01828195
:10D02000882309F408C1C80183559F4F0E94E0324C
:10D03000F80111821B821E8284E892E09A83898320
:10D04000C801429690AB87A7F60180818F3209F024
:10D050008EC06FE270E0C6010E94977501967C0158
:10D060004AE0542E66246394712C6C0E7D1E7AC0A7
:10D070006FE270E0C7010E9497755C01009709F4A8
:10D080007CC0E816F90608F078C04C018E189F089D
:10D09000A401B701CE014E960E94B775EEE1F0E013
:10D0A000EC0FFD1FE80DF91D10823EE1E32EF12C7F
:10D0B000EC0EFD1EF70106C09091C00095FFFCCF5D
:10D0C0008093C60081918111F7CF8091C00085FFC8
:10D0D000FCCF5092C600F80167A570A961157105D3
:10D0E00019F06E5F7F4F02C060E070E021E0AE019A
:10D0F000425E5F4FCE0103960E94183581112BC00E
:10D10000E8E9F2E107C09091C00095FFFCCF809361
:10D11000C600319684918111F6CF06C09091C0006F
:10D1200095FFFCCF8093C600F70181917F018111AB
:10D13000F5CFECEAF2E107C09091C00095FFFCCF7B
:10D140008093C600319684918111F6CF8091C00002
:10D1500085FFFCCF69C0F80170AA67A67501FFEFD3
:10D16000EF1AFF0AE114F10409F082CF05C0C801EB
:10D17000C196F80190AB87A77601F80187A590A921
:10D18000009711F0029602C080E090E0B7010E9483
:10D19000D535882301F1EEEAF2E107C09091C00095
:10D1A00095FFFCCF8093C600319684918111F6CF14
:10D1B000F70106C09091C00095FFFCCF8093C60098
:10D1C00081918111F7CFF801E053FF4F1082118256
:10D1D000128213822CC0ECEBF2E107C09091C000E8
:10D1E00095FFFCCF8093C600319684918111F6CFD4
:10D1F000F70106C09091C00095FFFCCF8093C60058
:10D2000081918111F7CFE4EDF2E107C09091C00068
:10D2100095FFFCCF8093C600319684918111F6CFA3
:10D220008091C00085FFFCCF8AE08093C600CE01CC
:10D2300001960E94AC2AAA960FB6F894DEBF0FBEE4
:10D24000CDBFDF91CF911F910F91FF90EF90DF90B5
:10D25000CF90BF90AF909F908F907F906F905F9096
:10D260000895CF93DF93EC018A818823C1F1E6ED25
:10D27000F2E107C09091C00095FFFCCF8093C600FB
:10D28000319684918111F6CFFE01E053FF4F40812A
:10D290005181628173812AE030E081EC95E00E9447
:10D2A000C42DE8EEF2E107C09091C00095FFFCCFDD
:10D2B0008093C600319684918111F6CFC853DF4F19
:10D2C000488159816A817B812AE030E081EC95E0D8
:10D2D0000E94C42D8091C00085FFFCCF11C0EAEEF2
:10D2E000F2E107C09091C00095FFFCCF8093C6008B
:10D2F000319684918111F6CF8091C00085FFFCCFDB
:10D300008AE08093C600DF91CF910895CF92DF929B
:10D31000EF92FF920F931F93CF93DF937C01EB016A
:10D32000EC2FFD2FDF010D900020E9F78D0101505A
:10D3300011090E1B1F0BF701E355FF4F10826EE41E
:10D3400070E0CE010E9497756C01009729F4F801F6
:10D350003197EC0FFD1F0DC060E270E00E949775E1
:10D36000EC0121966AE270E0C6010E949775FC010B
:10D3700031978DE081838AE082831382BE01C701E9
:10D3800085559F4F0E949937F701E355FF4F8081E4
:10D39000882309F1EDEEF1E107C09091C00095FFFF
:10D3A000FCCF8093C600319684918111F6CFEAEFCD
:10D3B000F2E107C09091C00095FFFCCF8093C600BA
:10D3C000319684918111F6CF8091C00085FFFCCF0A
:10D3D0008AE08093C600DF91CF911F910F91FF905B
:10D3E000EF90DF90CF9008953F924F925F926F92AF
:10D3F0007F928F929F92AF92BF92CF92DF92EF92E5
:10D40000FF920F931F93CF93DF93CDB7DEB7CC5529
:10D41000D1090FB6F894DEBF0FBECDBF8C016623D5
:10D4200049F0F801EC52FF4F1082F801828181111E
:10D4300018C030C0FC01EC52FF4F8081882309F4F2
:10D44000AEC0F801E453FF4FC080D180E280F3808A
:10D450000E94252BC616D706E806F90608F49FC0D9
:10D46000E0CFF80181898F9380898F9386EC92E0D9
:10D470009F938F937E01FFE3EF0EF11CFF92EF92DB
:10D480000E94E0750F900F900F900F900F900F90EB
:10D49000670110C0C8010E943065F80182818111C6
:10D4A000E0CF7DC0F701808190E00E945675F701C2
:10D4B00081937F01F60101900020E9F73197EC1983
:10D4C000FD09C7018C199D098E179F075CF3380170
:10D4D000F4E16F0E711C40E050E0BA01C3010E94FC
:10D4E000F931312CEE24E394F12CEC0EFD1E5E019B
:10D4F0008FE3A80EB11C7FEC472E72E0572E4E0131
:10D50000E1E28E0E911C37C0F601808190E00E940E
:10D510005675F60181936F01F70101900020E9F73C
:10D520003197EE19FF09C6018E199F098E179F07C3
:10D530005CF38A858E37F9F045E050E0B501C7010C
:10D540000E94A9750097B9F4BF92AF925F924F9273
:10D550009F928F920E94E075C4010E94B50E86EDE5
:10D5600092E00E94B50E0F900F900F900F900F90C9
:10D570000F9033243394B701C3010E9486311816EB
:10D5800014F46701C9CF311004C08FEF9FEFF80189
:10D5900004C0F801808991890196918B808BC45ACF
:10D5A000DF4F0FB6F894DEBF0FBECDBFDF91CF9136
:10D5B0001F910F91FF90EF90DF90CF90BF90AF90B1
:10D5C0009F908F907F906F905F904F903F900895C5
:10D5D0000F931F93CF93DF938C01EC01C355DF4F63
:10D5E000CE010E949432CE010E94E032F8011082F6
:10D5F000DF91CF911F910F910895CF93DF93EC01AD
:10D600000E94D4570E94495819828AED92E00E94E4
:10D61000B50E8091260D8823A1F11092260D609100
:10D62000E802E62FF0E0EE0FFF1FE050F24F80819E
:10D6300091810E9459592091390130913A014091CC
:10D640003B0150913C010E94AD701816D4F46091DA
:10D65000E802C62FD0E080E090E00E948958FE01E9
:10D66000EE0FFF1FE050F24F91838083FE01EE0F1B
:10D67000FF1FEE0FFF1FEA50F24F1082118212823D
:10D680001382DF91CF910895EF92FF920F931F9332
:10D69000CF93DF937C01EB018A01060F171F09C0AE
:10D6A0006991D701ED91FC910190F081E02DC701C6
:10D6B0000995C017D107A1F7DF91CF911F910F9165
:10D6C000FF90EF9008958FEF8EBD0DB407FEFDCF54
:10D6D0008EB508958EBD0DB407FEFDCF089561E0AF
:10D6E000FC0180810C94692CFC014281242F30E0E4
:10D6F0003595279520652CBD40FD03C021E04630BF
:10D7000009F420E02DBD60E0FC0180810C94692CBF
:10D71000CF92DF92EF92FF920F931F93CF93DF93FD
:10D72000EC018B017A010E94252B6B0109C00E943C
:10D73000252B6C197D096D32714010F081E108C014
:10D740000E94636B8B838F3F91F38E3F19F08FE0C4
:10D75000898328C0E114F104E1F081E0E81AF108BE
:10D760008FEF8EBDF8012FEF06C00DB407FEFDCF81
:10D770008EB581932EBDCF01801B910B8E159F0519
:10D78000A0F30DB407FEFDCF8EB5F801EE0DFF1D21
:10D7900080830E94636B0E94636BCE010E946F6B5B
:10D7A00081E004C0CE010E946F6B80E0DF91CF91D9
:10D7B0001F910F91FF90EF90DF90CF9008950F93FE
:10D7C0001F93CF93DF938B010E94252BEB0107C0A2
:10D7D0000E94252B6C1B7D0B6017710730F40E9493
:10D7E000636B8F3FA9F781E001C080E0DF91CF91AB
:10D7F0001F910F910895CF92DF92FF920F931F9385
:10D80000CF93DF9300D000D0CDB7DEB78C01F62EDA
:10D8100029833A834B835C830E94746B6CE271E0D2
:10D82000C8010E94DF6B8F2D80640E946A6B68E1E3
:10D83000C62ED12C5C814B813A812981DA01C90144
:10D840000C2C04C0B695A795979587950A94D2F7A6
:10D8500029833A834B835C830E946A6B68E0C61A13
:10D86000D10829813A814B815C8188EFC8168FEFFE
:10D87000D80621F7FF2029F098E0F91621F08FEF64
:10D8800003C085E901C087E80E946A6BECE0FE12E4
:10D8900002C00E94636BF12C0E94636BF8018383CA
:10D8A00087FF05C0FFEFFF1611F0F394F5CF0F903F
:10D8B0000F900F900F90DF91CF911F910F91FF90DC
:10D8C000DF90CF9008950F931F93CF93DF93EC01D8
:10D8D00089018C81833039F0B9E0440F551F661FF0
:10D8E000771FBA95D1F79A01AB0161E1CE010E9491
:10D8F000FB6B81110AC040E052E0B801CE01DF911C
:10D90000CF911F910F910C94886B84E08983CE0195
:10D910000E946F6B80E0DF91CF911F910F9108956E
:10D92000BF92CF92DF92EF92FF920F931F93CF930C
:10D93000DF93EC01B62E1C82198248830E94252BAE
:10D940008B0161E088810E944D2CCE010E946F6B9B
:10D9500060E086E00E944D2C61E085E00E944D2C45
:10D9600061E087E00E944D2C61E084E00E944D2C34
:10D9700061E084E00E94692C85E08A8382E58CBDA9
:10D980001DBC2AE0F22E8FEF0E946A6BFA94D9F741
:10D9900009C00E94252B601B710B613D774010F080
:10D9A00081E058C020E030E0A90160E0CE010E9493
:10D9B000FB6BF82E8B8381E0F812EBCF2AEA31E083
:10D9C00040E050E068E0CE010E94FB6B82FF02C0A5
:10D9D000FC820DC094E0F92E0E94636B8B83FA9455
:10D9E000D9F78A3A11F082E035C082E08C838C81CD
:10D9F000823031F4C12CD12CE12C80E4F82E0DC002
:10DA0000C12CD12C760109C00E94252B601B710B03
:10DA1000613D774010F08AE01DC020E030E0A901B0
:10DA200067E3CE010E94FB6BA701960169E2CE017C
:10DA30000E94FB6B8B838111E7CF8C818230C9F40C
:10DA400020E030E0A9016AE3CE010E94FB6B88234D
:10DA500019F088E0898319C00E94636B807C803C48
:10DA600011F483E08C830E94636B0E94636B0E94BD
:10DA7000636BCE010E946F6B86E08B1518F488E112
:10DA8000898306C0BA8281E004C0CE010E946F6B18
:10DA900080E0DF91CF911F910F91FF90EF90DF9089
:10DAA000CF90BF900895CF93DF93EC016EBD20E03F
:10DAB00030E00DB407FEFDCFFA01E20FF31F8081C5
:10DAC0008EBD0DB407FEFDCF81818EBD2E5F3F4F11
:10DAD000211582E0380769F70DB407FEFDCF8FEFFF
:10DAE0000E946A6B8FEF0E946A6B0E94636B8B834C
:10DAF0008F71853039F083E18983CE010E946F6B8D
:10DB000080E001C081E0DF91CF9108950F931F93D2
:10DB1000CF93DF93EC0189018C81833039F0E9E008
:10DB2000440F551F661F771FEA95D1F79A01AB0185
:10DB300068E1CE010E94FB6B882311F086E029C0CA
:10DB4000A8016EEFCE010E94536D8823B9F068E5FD
:10DB500072E0CE010E94DF6B811102C087E119C023
:10DB600020E030E0A9016DE0CE010E94FB6B811145
:10DB70000FC00E94636B81110BC005C0CE010E94D3
:10DB80006F6B80E008C0CE010E946F6B81E003C024
:10DB900086E18983F3CFDF91CF911F910F91089593
:10DBA0005058BB27AA270ED076C23FD230F044D2BD
:10DBB00020F031F49F3F11F41EF40FC20EF4E095F3
:10DBC000E7FBDCC1E92F89D280F3BA17620773073C
:10DBD0008407950718F071F49EF5B8C20EF4E0952D
:10DBE0000B2EBA2FA02D0B01B90190010C01CA0117
:10DBF000A0011124FF27591B99F0593F50F4503EC2
:10DC000068F11A16F040A22F232F342F4427585FB3
:10DC1000F3CF469537952795A795F0405395C9F7CB
:10DC20007EF41F16BA0B620B730B840BBAF0915083
:10DC3000A1F0FF0FBB1F661F771F881FC2F70EC022
:10DC4000BA0F621F731F841F48F4879577956795F5
:10DC5000B795F7959E3F08F0B3CF9395880F08F0DE
:10DC60009927EE0F979587950895DFD158F080E8B2
:10DC700091E009F49EEFE0D128F040E851E059F43A
:10DC80005EEF09C0AAC162C2E92FE07826D268F32C
:10DC9000092E052AC1F3261737074807590738F018
:10DCA0000E2E07F8E02569F0E025E0640AC0EF6376
:10DCB00007F8009407FADB01B9019D01DC01CA01F4
:10DCC000AD01EF935DD0E7D10AD05F91552331F0DC
:10DCD0002BED3FE049E450FD49EC63CF0895DF931D
:10DCE000DD27B92FBF7740E85FE316161706480710
:10DCF0005B0710F4D92F96D29F938F937F936F93E6
:10DD0000A9D3ECE7F0E06CD1C6D12F913F914F91B0
:10DD10005F9101D3DD2349F09058A2EA2AED3FE05C
:10DD200049EC5FE3D0785D274DDFDF91B4C1F7D1D7
:10DD300080F09F3740F491110EF409C260E070E06A
:10DD400080E89FE3089526F01B16611D711D811D5B
:10DD50001BC135C1EFD008F481E0089575D1E3957A
:10DD6000ABC10CD098C168D140F05FD130F021F444
:10DD70005F3F19F003C15111EAC12FC1AED198F331
:10DD80009923C9F35523B1F3951B550BBB27AA273C
:10DD900062177307840738F09F5F5F4F220F331FAE
:10DDA000441FAA1FA9F333D00E2E3AF0E0E830D07A
:10DDB00091505040E695001CCAF729D0FE2F27D07D
:10DDC000660F771F881FBB1F261737074807AB074B
:10DDD000B0E809F0BB0B802DBF01FF2793585F4FC0
:10DDE0002AF09E3F510568F0C9C0B1C15F3FECF316
:10DDF000983EDCF3869577956795B795F7959F5F85
:10DE0000C9F7880F911D9695879597F90895E1E0D8
:10DE1000660F771F881FBB1F621773078407BA0737
:10DE200020F0621B730B840BBA0BEE1F88F7E09592
:10DE3000089504D06894B1118AC1089556D188F02C
:10DE40009F5790F0B92F9927B751A0F0D1F0660FE6
:10DE5000771F881F991F1AF0BA95C9F712C0B13001
:10DE600081F074D1B1E0089571C1672F782F8827B0
:10DE7000B85F39F0B93FCCF3869577956795B39540
:10DE8000D9F73EF490958095709561957F4F8F4FAF
:10DE90009F4F0895E89409C097FB3EF490958095B4
:10DEA000709561957F4F8F4F9F4F9923A9F0F92F60
:10DEB00096E9BB279395F695879577956795B795DE
:10DEC000F111F8CFFAF4BB0F11F460FF1BC06F5FC4
:10DED0007F4F8F4F9F4F16C0882311F096E911C0D6
:10DEE000772321F09EE8872F762F05C0662371F0F7
:10DEF00096E8862F70E060E02AF09A95660F771F0B
:10DF0000881FDAF7880F9695879597F9089507D1B6
:10DF100080F09F3740F491110EF019C160E070E07D
:10DF200080E89FEB089526F41B16611D711D811D6D
:10DF30002BC045C0990F0008550FAA0BE0E8FEEF73
:10DF400016161706E807F907C0F012161306E407BD
:10DF5000F50798F0621B730B840B950B39F40A26B6
:10DF600061F0232B242B252B21F408950A2609F494
:10DF7000A140A6958FEF811D811D089597F99F6798
:10DF800080E870E060E00895882371F4772321F041
:10DF90009850872B762F07C0662311F499270DC060
:10DFA0009051862B70E060E02AF09A95660F771FFB
:10DFB000881FDAF7880F9695879597F908959F3F00
:10DFC00031F0915020F4879577956795B795880F34
:10DFD000911D9695879597F908959FEF80EC089588
:10DFE000DF93CF931F930F93FF92EF92DF927B010A
:10DFF0008C01689405C0DA2EEF018DD1FE01E89402
:10E00000A5912591359145915591AEF3EF01DADD5A
:10E01000FE019701A801DA9479F7DF90EF90FF9065
:10E020000F911F91CF91DF91089500240A94161645
:10E03000170618060906089500240A9412161306F6
:10E04000140605060895C9CF50D0E8F3E894E0E03F
:10E05000BB279F57F0F02AED3FE049EC06C0EE0FDA
:10E06000BB0F661F771F881F28F0B23A620773073D
:10E07000840728F0B25A620B730B840BE3959A95D0
:10E0800072F7803830F49A95BB0F661F771F881F90
:10E09000D2F7904896CF092E0394000C11F48823F0
:10E0A00052F0BB0F40F4BF2B11F460FF04C06F5F50
:10E0B0007F4F8F4F9F4F0895EF93E0FF06C0A2EA76
:10E0C0002AED3FE049EC5FEB7DDDE5DF0F90039447
:10E0D00001FC9058E9EAF0E0C7C157FD9058440FA1
:10E0E000551F59F05F3F71F04795880F97FB991FB7
:10E0F00061F09F3F79F08795089512161306140674
:10E10000551FF2CF4695F1DF08C016161706180600
:10E11000991FF1CF86957105610508940895E5DF93
:10E12000A0F0BEE7B91788F4BB279F3860F4161635
:10E13000B11D672F782F8827985FF7CF8695779541
:10E140006795B11D93959639C8F30895E894BB2758
:10E1500066277727CB0197F90895ECDE08F48FEF57
:10E16000089563DF19F068DF09F037CF07CFB901F1
:10E17000CA0125CF9F775F77B0DF98F39923B9F372
:10E180005523B9F3FF27951758F4E52FE91BED3018
:10E1900070F75E3B10F0F1E41CC09034E0F40AC06C
:10E1A000E92FE51BED3028F79E3B10F0F1E411C09C
:10E1B000503488F4F9EA88232AF09A95660F771F7D
:10E1C000881FDAF744232AF05A95220F331F441F81
:10E1D000DAF79F1B5F1BFF931F930F93FF92EF9242
:10E1E00079018A01BB27AB2F9B01AC0196D0970127
:10E1F000A801BF937B018C01AA27BA2FB901CA01DC
:10E200008CD0AF919701A801EF90FF900F911F91D3
:10E21000D9DC41DFE1D04F9140FF0895552747FDFC
:10E22000509509C09B01AC0160E070E080E89FE37D
:10E2300098CDA4CEC4CE59DFE8F39923D9F3940F37
:10E24000511DBBF39150504094F059F0882332F0A7
:10E25000660F771F881F91505040C1F79E3F5105B0
:10E2600044F7880F911D9695879597F908955F3F1C
:10E27000ACF0983E9CF0BB27869577956795B7954F
:10E2800008F4B1609395C1F7BB0F58F711F460FF24
:10E29000E8CF6F5F7F4F8F4F9F4FE3CF58CF25DF82
:10E2A00058F19E5758F19851A0F0E9F0983020F5B8
:10E2B000092E9927660F771F881F991F0A94D1F797
:10E2C00012C0062E672F782F8827985F11F4000C54
:10E2D00007C0993FB4F38695779567959395D9F7DD
:10E2E000611D711D811D3EF490958095709561951D
:10E2F0007F4F8F4F9F4F0895689429CF27CF0BD022
:10E30000CACE93DE28F098DE18F0952309F036CEB9
:10E3100064CE11241CCFE1DEA0F3959FD1F3950FBD
:10E3200050E0551F629FF001729FBB27F00DB11D99
:10E33000639FAA27F00DB11DAA1F649F6627B00D29
:10E34000A11D661F829F2227B00DA11D621F739F12
:10E35000B00DA11D621F839FA00D611D221F749F20
:10E360003327A00D611D231F849F600D211D822F67
:10E37000762F6A2F11249F5750408AF0E1F08823AE
:10E380004AF0EE0FFF1FBB1F661F771F881F9150BB
:10E390005040A9F79E3F510570F0F0CDD8CE5F3FB9
:10E3A000ECF3983EDCF3869577956795B795F795EE
:10E3B000E7959F5FC1F7FE2B880F911D9695879576
:10E3C00097F908959F9340DE0F9007FCEE5F74CE9F
:10E3D00011F40EF402CEF3CD88DED0F39923D9F3F5
:10E3E000CEF39F57550B87FF38D00024A0E640EAB4
:10E3F000900180585695979528F4805C660F771F9A
:10E40000881F20F026173707480730F4621B730B6C
:10E41000840B202931294A2BA6951794079420258F
:10E4200031254A2758F7660F771F881F20F02617D7
:10E430003707480730F4620B730B840B200D311D36
:10E44000411DA09581F7B901842F9158880F9695A9
:10E45000879508959B01AC0152CF91505040660FB3
:10E46000771F881FD2F708959F938F937F936F93A1
:10E47000FF93EF939B01AC0142DFEF91FF91B0DD81
:10E480002F913F914F915F913ACF0E94BA72A59F11
:10E49000900DB49F900DA49F800D911D112408959F
:10E4A000B7FF0C9445720E944572821B930B08952E
:10E4B000DB018F939F930E944572BF91AF91A29F02
:10E4C000800D911DA39F900DB29F900D1124089572
:10E4D00097FB072E16F4009407D077FD09D00E9411
:10E4E000C67207FC05D03EF4909581959F4F089524
:10E4F000709561957F4F0895A1E21A2EAA1BBB1B50
:10E50000FD010DC0AA1FBB1FEE1FFF1FA217B307FF
:10E51000E407F50720F0A21BB30BE40BF50B661F15
:10E52000771F881F991F1A9469F7609570958095D9
:10E5300090959B01AC01BD01CF010895052E97FB7D
:10E5400016F4009407D057FD0DD00E947C7207FC92
:10E5500009D07EF490958095709561957F4F8F4F8F
:10E560009F4F089550954095309521953F4F4F4FBF
:10E570005F4F0895A29FB001B39FC001A39F01D038
:10E58000B29F700D811D1124911D0895AA1BBB1B04
:10E5900051E107C0AA1FBB1FA617B70710F0A61BA3
:10E5A000B70B881F991F5A95A9F780959095BC01C4
:10E5B000CD010895EE0FFF1F0590F491E02D099411
:10E5C000A0E0B0E0E6EEF2E70C94A0788B016115D4
:10E5D000710519F0FB01808391837C01F701C190E3
:10E5E0007F01EF018C2D90E00E944E75892BB1F7D1
:10E5F000FDE2CF1204C0C990DD24D39405C02BE204
:10E60000C21201C0C990D12C7E0141E0E41AF10888
:10E6100043E050E06AE773E1C7010E945E75892B11
:10E62000E9F47E0182E0E80EF11C45E050E06DE780
:10E6300073E1C7010E945E75892B21F47E01E7E03A
:10E64000EE0EF11C0115110519F0F801F182E082BE
:10E6500010E0D0E0C0E8D110FBC0FFC043E050E0C4
:10E6600062E873E1C7010E945E75892B49F40115C8
:10E67000110509F4EFC02296F801D183C083EAC0E6
:10E6800060E070E0CB01E12CF12CEC2DE053EA309E
:10E6900048F5FD2DF2602D2D2870D2FE06C0211107
:10E6A00027C02FEFE21AF20A23C0222319F041E01B
:10E6B000E41AF108A5E0B0E09B01AC010E944572AC
:10E6C000660F771F881F991F6E0F711D811D911D89
:10E6D0006839E9E97E078E07E9E19E0748F0FD2DDC
:10E6E000F66006C0EE3F39F4D3FC3DC0FD2DF86066
:10E6F000C990DF2ECACFE53311F0E531A1F5A8812D
:10E70000AD3219F4F0E1DF2A06C0AB3221F02196D8
:10E7100021E030E004C0A981229622E030E0A0533D
:10E72000AA3018F0C21BD30B1EC0FE0120E030E05F
:10E7300020384CE034075CF4A901440F551F440F06
:10E74000551F240F351F220F331F2A0F311DA19192
:10E75000A053EF01AA3060F3D4FE03C03195219598
:10E760003109E20EF31ED1FE07C00115110521F09B
:10E770002197F801D183C0830E944A6F2D2D237009
:10E78000233029F0162FD72FC82F092F07C0DC01FF
:10E79000CB01B058182FD92FCA2F0B2F20E030E013
:10E7A000A901612F7D2F8C2F902F0E94AA6E8823A4
:10E7B00009F454C0F7FE08C0F194E194F10831EB7C
:10E7C000C32E33E1D32E04C029E9C22E23E1D22E79
:10E7D0004601F8E18F1A910890E2A92EB12C15C0DC
:10E7E000F6014591559165917491242F352F462F4F
:10E7F000572F612F7D2F8C2F902F0E947F71162F06
:10E80000D72FC82F092FEA18FB08EA14FB0444F796
:10E8100024E0C21AD108B594A794C814D904A9F762
:10E82000612F7D2F8C2F902F282F220F292F221F11
:10E830002F3F39F020E030E0A9010E94AA6E81113B
:10E840000DC082E290E09093440E8093430E06C088
:10E850000FEF04C010E0D0E0C0EC0FE7612F7D2F78
:10E860008C2F902FCDB7DEB7ECE00C94BC78A0E0F5
:10E87000B0E0EDE3F4E70C949C782B018A0161157C
:10E88000710519F0FB01808391830115110539F0A1
:10E890009801225031092332310508F0E6C07C018D
:10E8A000F701C1917F013F018C2F90E00E944E75CE
:10E8B000892BB1F7CD3229F4F701C1913F01D1E0A5
:10E8C00006C0CB3219F4F701C1913F01D0E0011528
:10E8D000110509F4D8C00031110581F4D0C0F3014D
:10E8E0008081883719F0883509F0C3C0F301C181F0
:10E8F000F2E06F0E711CD26000E110E008301105EB
:10E90000D9F024F402301105F9F407C00A301105DA
:10E9100051F000311105C1F425C0C12CD12CE12CDE
:10E9200030E4F32E24C00AE010E02CECC22EDC2CE4
:10E93000EC2C2CE0F22E1BC008E010E0C12CD12CF6
:10E94000E12C90E1F92E13C09801442737FD409542
:10E95000542F60E070E080E090E80E947C726901D2
:10E960007A0105C0C12CD12CE12C88E0F82E40E0C2
:10E9700060E070E0CB014801AA2497FCA094BA2C77
:10E98000EC2FE053EA3060F02C2F21542A3110F4A0
:10E99000E75006C02C2F21562A3128F5EC2FE755D9
:10E9A0002E2F30E020173107F4F447FD18C0C616AB
:10E9B000D706E806F90680F09B01AC01C501B40159
:10E9C0000E9458726E0F711D811D911D613071057D
:10E9D000810520E8920710F04FEF01C041E0F301FC
:10E9E000C1913F01CDCF4114510491F0442339F03E
:10E9F000F1E06F1A7108F2017182608209C0D1FFE3
:10EA00001BC0F2E06F1A7108F2017182608214C0BB
:10EA100047FF12C0D0FF05C060E070E080E090E8E2
:10EA200004C06FEF7FEF8FEF9FE722E230E030937B
:10EA3000440E2093430E16C0D0FF08C090958095D9
:10EA4000709561957F4F8F4F9F4F0CC097FF0AC005
:10EA500082E290E09093440E8093430E6FEF7FEF3D
:10EA60008FEF9FE76B017C0112C0C12CD12C760186
:10EA70000EC0C0E30115110509F45ECF3FCFC033CE
:10EA800009F03CCF2CCFC03309F04DCF28CFB601D1
:10EA9000C701CDB7DEB7E0E10C94B8789111A7C2F9
:10EAA000803219F089508550D0F70895911108955A
:10EAB00081548A5108F4805E855A0895FB01DC0177
:10EAC0004150504088F08D9181341CF08B350CF40E
:10EAD000805E659161341CF06B350CF4605E861BC2
:10EAE000611171F3990B0895881BFCCFFB01DC01C8
:10EAF00004C08D910190801921F441505040C8F715
:10EB0000881B990B0895FB01DC0102C001900D9256
:10EB100041505040D8F70895FB01DC010D900020D2
:10EB2000E9F7119701900D920020E1F70895FC019B
:10EB30008191861721F08823D9F799270895319775
:10EB4000CF010895FB01DC0101900D920020E1F757
:10EB50000895FB01DC014150504030F08D9101904F
:10EB6000801919F40020B9F7881B990B0895FB014F
:10EB7000DC014150504048F001900D920020C9F74F
:10EB800001C01D9241505040E0F70895FB015191A2
:10EB90005523A9F0BF01DC014D9145174111E1F763
:10EBA00059F4CD010190002049F04D9140154111DB
:10EBB000C9F3FB014111EFCF81E090E00197089587
:10EBC000A0E1B0E0E6EEF5E70C94A8780F89188D87
:10EBD00086E08C831A8309838FEF9FE79E838D8362
:10EBE000AE01455E5F4F588B4F87698D7A8DCE01A0
:10EBF00001960E940476EF81F885E00FF11F1082E4
:10EC00006096E4E00C94C478ACE0B0E0EAE0F6E7AB
:10EC10000C949A787C016B018A01FC0117821682A0
:10EC2000838181FFC7C188248394912C8C0E9D1E03
:10EC3000F7019381F60193FD859193FF81916F0117
:10EC4000882309F4B3C1853239F493FD859193FF8C
:10EC500081916F01853229F4B70190E00E9410780C
:10EC6000E7CF712C312C20E02032A8F48B3261F0F8
:10EC700028F4803251F0833271F40BC08D3239F0B8
:10EC8000803349F4216028C02260246025C02860B8
:10EC900023C0206121C027FD27C0382F30533A30D0
:10ECA00078F426FF06C0FAE07F9E300D1124732E03
:10ECB00013C08AE0389E300D1124332E20620CC020
:10ECC0008E3221F426FD72C1206406C08C3611F408
:10ECD000206802C0883641F4F60193FD859193FFC8
:10ECE00081916F018111C0CF982F9554933018F006
:10ECF0009052933028F40C5F1F4FFFE3F9830DC04F
:10ED0000833631F0833771F0833509F05EC023C05C
:10ED1000F801808189830E5F1F4F66246394712CF4
:10ED2000540115C02801F2E04F0E511CF801A080DB
:10ED3000B18026FF03C0672D70E002C06FEF7FEF48
:10ED4000C5012C870E9405783C0182012C856FE764
:10ED5000262E222218C02801F2E04F0E511CF80185
:10ED6000A080B18026FF03C0672D70E002C06FEF66
:10ED70007FEFC5012C870E94FA773C012C8550E873
:10ED8000252E222A820123FC1CC006C0B70180E286
:10ED900090E00E9410783A94832D90E068167906EE
:10EDA000A8F30FC0F50127FC859127FE81915F0133
:10EDB000B70190E00E94107831103A94F1E06F1A98
:10EDC00071086114710471F7EEC0843611F0893650
:10EDD00041F5F80127FF07C060817181828193812D
:10EDE0000C5F1F4F08C060817181882777FD809577
:10EDF000982F0E5F1F4F4FE6642E622297FF09C0C7
:10EE000090958095709561957F4F8F4F9F4FF0E85B
:10EE10006F2A2AE030E0A4010E943C78A82EA818AE
:10EE200044C0853731F43FEEB32EB2222AE030E001
:10EE300024C099EFB92EB2228F36B9F020F488356C
:10EE400009F0B4C00DC0803721F0883709F0AEC09A
:10EE500002C020E1B22AB4FE0BC084E0B82A08C088
:10EE600024FF09C0E6E0BE2A06C028E030E005C065
:10EE700020E130E002C020E132E0F801B7FE07C037
:10EE800060817181828193810C5F1F4F06C0608118
:10EE9000718180E090E00E5F1F4FA4010E943C78DA
:10EEA000A82EA8188FE7682E6B2066FE0BC0362DA3
:10EEB0003E7FA71450F464FE0AC062FC08C0362DE1
:10EEC0003E7E05C0BA2C362D03C0BA2C01C0B72C2B
:10EED00034FF0DC0FE01EA0DF11D8081803311F475
:10EEE000397E09C032FF06C0B394B39404C0832FA7
:10EEF000867809F0B39433FD14C030FF0FC07A2C2C
:10EF0000B31460F4730C7B18B32C08C0B70180E213
:10EF100090E03C870E941078B3943C85B314B0F322
:10EF200004C0B31410F43B1801C0312C34FF12C0DC
:10EF3000B70180E390E03C870E9410783C8532FF67
:10EF40001EC031FF03C088E590E002C088E790E072
:10EF5000B7010CC0832F867891F031FD02C080E2AA
:10EF600001C08BE237FD8DE2B70190E00E9410787E
:10EF700006C0B70180E390E00E9410787A94A7144D
:10EF8000C0F3AA94F401EA0DF11DB701808190E06D
:10EF90000E941078A110F5CF06C0B70180E290E082
:10EFA0000E9410783A943110F8CF42CEF7012681B2
:10EFB000378102C02FEF3FEFC9012C96E2E10C949C
:10EFC000B678F999FECF92BD81BDF89A992780B5A0
:10EFD0000895262FF999FECF1FBA92BD81BD20BD9D
:10EFE0000FB6F894FA9AF99A0FBE019608959927E8
:10EFF00088270895FC010590615070400110D8F7F2
:10F00000809590958E0F9F1F0895FC016150704070
:10F0100001900110D8F7809590958E0F9F1F08954D
:10F020000F931F93CF93DF938C01EB018B8181FDB5
:10F0300003C00FEF1FEF1AC082FF0DC02E813F816A
:10F040008C819D812817390764F4E881F981019347
:10F05000F983E88306C0E885F985802F0995892B17
:10F0600041F78E819F8101969F838E83C801DF9136
:10F07000CF911F910F910895FA01AA27283051F1DD
:10F08000203181F1E8946F936E7F6E5F7F4F8F4FD9
:10F090009F4FAF4FB1E03ED0B4E03CD0670F781F38
:10F0A000891F9A1FA11D680F791F8A1F911DA11D1D
:10F0B0006A0F711D811D911DA11D20D009F4689456
:10F0C0003F912AE0269F11243019305D3193DEF6FE
:10F0D000CF010895462F4770405D4193B3E00FD0B4
:10F0E000C9F7F6CF462F4F70405D4A3318F0495D9F
:10F0F00031FD4052419302D0A9F7EACFB4E0A69582
:10F100009795879577956795BA95C9F700976105A3
:10F11000710508959B01AC010A2E069457954795F9
:10F1200037952795BA95C9F7620F731F841F951FEE
:10F13000A01D08952F923F924F925F926F927F92FF
:10F140008F929F92AF92BF92CF92DF92EF92FF92F7
:10F150000F931F93CF93DF93CDB7DEB7CA1BDB0BA3
:10F160000FB6F894DEBF0FBECDBF09942A88398848
:10F1700048885F846E847D848C849B84AA84B9844F
:10F18000C884DF80EE80FD800C811B81AA81B9815B
:10F19000CE0FD11D0FB6F894DEBF0FBECDBFED016F
:10F1A000089513E1C8EBD3E104C0FE010E94DC72B4
:0CF1B0002296CA3BD107C9F7F894FFCFA4
:10F1BC0000001B43000016430000B4420000000096
:10F1CC0000000000000080BF6400640000803B452C
:10F1DC0000803B4500007043000000000080BB44F1
:10F1EC000160EA0000CDCCCC3D0000524300007A17
:10F1FC004301010101010000803FE7849145AECF3E
:10F20C001A3D00004041FF3FFF3F0171DBB64271E8
:10F21C00DBB64200007A4500C05A440000FA4300B5
:10F22C0000FA430000A04000003442E8030000E86C
:10F23C0003000032000000FA0000004D31313000B4
:10F24C002569206D696E2C20256920736563005536
:10F25C0073696E672044656661756C7420736574A0
:10F26C0074696E67733A004820004C20004D3130B1
:10F27C003420496E76616C696420657874727564AB
:10F28C00657220004D31303520496E76616C6964B1
:10F29C0020657874727564657220004D31303920A8
:10F2AC00496E76616C6964206578747275646572F8
:10F2BC0020003F006F6B0020703A0020693A00205C
:10F2CC00643A0020633A005400496E76616C6964BC
:10F2DC002065787472756465720041637469766533
:10F2EC002045787472756465723A20004D3239008D
:10F2FC0058595A45000001000F0015000E0012006D
:10F30C00FFFF160017000E001300FFFF03000200A2
:10F31C001A001400FFFFFFFFFFFF0A00FFFF0100B0
:10F32C0000000E000D000700FFFFFFFF06002E007F
:10F33C0000000000A5379937446B537465707261F7
:10F34C00746520746F2068696768203A2000504902
:10F35C0044204175746F74756E652073746172749A
:10F36C00002F0043616E6E6F74206F70656E20739A
:10F37C007562646972006175746F25692E67004D42
:10F38C003233202573004D3234004D383420582050
:06F39C0059205A20450033
:00000001FF
